:020000040800F2
:10000000F8160020850100088B0500081D04000873
:1000100089050008F10100089B0E0008000000009F
:10002000000000000000000000000000AB0C000811
:10003000F301000800000000A90500087D0D00087C
:100040009F0100089F0100089F0100089F01000810
:100050009F0100089F0100089F0100089F01000800
:100060009F0100089F0100089F0100089F010008F0
:100070009F0100089F0100089F0100089F010008E0
:100080009F0100089F0100089F0100089F010008D0
:100090009F0100089F0100089F0100089F010008C0
:1000A0009F0100089F0100089F0100089F010008B0
:1000B0009F010008490E00089F0100089F010008E9
:1000C0009F0100089F0100089F0100089F01000890
:1000D0009F0100089F0100089F0100089F01000880
:1000E0009F0100089F0100089F0100080000000018
:1000F0000000000000000000000000000000000000
:1001000000000000000000009F0100089F0100089F
:100110009F0100089F0100089F0100089F0100083F
:100120009F0100089F0100089F0100089F0100082F
:100130009F0100089F0100089F0100089F0100081F
:100140009F0100089F0100089F0100089F0100080F
:10015000DFF80CD000F03AF800480047012400080E
:10016000F8160020EFF30980704780F30988704784
:10017000EFF30880704780F30888704740BA7047F3
:10018000C0BA70470648804706480047FEE7FEE7CA
:10019000FEE7FEE7FEE7FEE7FEE7FEE7FEE7FEE737
:1001A000ED0D000851010008D2B201E000F8012B6A
:1001B000491EFBD270470022F6E710B513460A46E7
:1001C00004461946FFF7F0FF204610BD064C074DC8
:1001D00006E0E06840F0010394E807009847103417
:1001E000AC42F6D3FFF7B8FF342F0008542F0008B5
:1001F000FEE7704701B50098411E00910028FAD132
:1002000008BD00000149C86070470000002002409E
:1002100070B50D4E0546304600F088F8042811D11F
:100220000A4C206940F0020020616561206940F0BD
:1002300040002061304600F079F8216941F6FD72F6
:100240001140216170BD0000FFFF0F00002002403F
:1002500008490420CA68D20701D001207047CA6843
:10026000520701D502207047C968C906FBD5032093
:1002700070470000002002400248016941F08001FF
:100280000161704700200240F0B506464FF6FF7747
:100290000D46384600F04AF804280DD1074C206975
:1002A00040F0010020613580384600F03FF82169B8
:1002B00041F6FE7211402161F0BD000000200240B5
:1002C0002DE9F841064600204FF6FF7700900D46D5
:1002D000384600F02BF8042817D10D4C206940F067
:1002E000010020613580B846384600F01FF841F61D
:1002F000FE77042806D1B61C280C009630804046B4
:1003000000F014F8216939402161BDE8F88100004E
:1003100000200240034802494160034941607047A0
:100320002301674500200240AB89EFCD00B50346AD
:10033000FFF78EFF02E0FFF78BFF5B1E012803D063
:10034000002B00D1052000BD002BF4D1FAE7F0B559
:10035000CC78002204F00F03E40601D58C78234307
:100360000C784FF00F0C4FF0010EDCB105680E88D1
:100370000EFA02F42640A64210D196000CFA06F7B7
:1003800025EA070703FA06F5CE783D43282E02D06A
:10039000482E02D002E0446100E00461521C082AA9
:1003A000E5D305600A88FF2A1CD94468002202F1BF
:1003B00008060EFA06F50E882E40AE420ED19600C3
:1003C0000CFA06F7BC4303FA06F7CE783C43282E16
:1003D00000D14561CE78482E00D10561521C082A13
:1003E000E5D34460F0BD41617047016170470AB1D7
:1003F0000161704741617047064801680648016025
:100400000449091F09684160024908390968816087
:1004100070470000F0F7FF1F80000020FEE700009B
:100420002DE9F047DFF878A0DAF800001D4988428E
:1004300034D10AF104000068A0F52051B1F5BC3FA9
:100440002CD84FEA9008800701D008F10108164E19
:10045000164DFFF75FFF002717E0D6F80090002445
:10046000680502D12846FFF7D3FE49462846FFF724
:1004700027FF042803D0641CE4B2032CF5D32868BA
:10048000814504D1361D2D1D7F1C4745E5D35046BF
:10049000FFF7BEFEBDE8F047FFF7EEBEBDE8F08710
:1004A000005802084433221100600208008000084E
:1004B000F8B501211C2000F079F84FF40076ADF872
:1004C000006010242D4F8DF8034003258DF8025055
:1004D00069463846FFF73BFF31463846FFF785FF50
:1004E0000120ADF800008DF803408DF802506946F8
:1004F0003846FFF72CFF01213846FFF776FF022030
:10050000ADF800008DF803408DF80250694638467A
:10051000FFF71DFF02213846FFF767FF2020ADF8E7
:100520000000174E8DF803408DF8025069463046A2
:10053000FFF70DFF20213046FFF755FF44F207007B
:10054000ADF800008DF803400E4C8DF8025069465E
:100550002046FFF7FCFE01212046FFF744FF022161
:100560002046FFF740FF04212046FFF73CFF4FF4F1
:1005700080412046FFF737FFF8BD0000000801402A
:1005800000100140000C0140FEE770474FF4A060EE
:10059000AFF3008002490843024908607047000039
:1005A0000000FA050CED00E070470000044A002945
:1005B000916901D0014300E08143916170470000DF
:1005C00000100240F0B52B4C61682B4A11F00C0171
:1005D0004FF00F0603D0042901D0082901D0026092
:1005E00026E06168636806EA914103F480330D29CF
:1005F00001D0891C00E00621BBB1E36A13F4803FFF
:10060000E36A03F00F0303F101030AD0E56AC5F3BF
:100610000317E56A7F1CB2FBF7F2C5F30325AD1C97
:100620006A43B2FBF3F24A43D9E7144A51430160EB
:100630006168134A06EA1111535C0168D9404160B0
:100640006368072505EA1323D35C21FA03F383606B
:10065000636805EAD323D25CD140C160626803239A
:1006600003EA9232064B1B1F9A5CB1FBF2F1016167
:10067000F0BD00000010024000127A0000093D00A9
:100680006400002010B5012210210448FFF7AFFEDE
:10069000BDE81040FF2000F09DBA000000080140B6
:1006A00070B5054601220021092000F0CFF90400B1
:1006B00004D11021284600F047F90446FFF7E2FF75
:1006C0000CB1012070BD002070BD70B505464FF61D
:1006D000FF7401E0641EA4B2FF2000F07DF9A8427F
:1006E00002D0002CF6D102E00CB1002070BDFF203A
:1006F00070BD1FB56846FFF7D3FF10B1002004B0EE
:1007000010BD9DF800100120B0EB911F09D19DF89C
:1007100008209DF8091000EB02200844000480091D
:10072000EDE79DF805009DF80A1000F00F0000EBC2
:10073000D1109DF809109DF8072001F0030100EB8E
:1007400041019DF80800800900EB82009DF8062019
:1007500002F0030200EB8220401CC91F8840CEE754
:100760002DE9F84300F00CF9382000F05FFA00F0B2
:1007700035F900204FF47061401C80B28842FBD3F1
:100780000024FF2000F026FA641CA4B20A2CF8D33F
:10079000C82400219522084600F058F90546012892
:1007A00004D02000A4F10104A4B2F2D14A4E0027E3
:1007B000012D377068D187224FF4D571082000F0E1
:1007C00045F94FF6FE78012820D00122002137207C
:1007D00000F03CF901220021292000F037F901281E
:1007E00053D802203070444601220021372000F007
:1007F0002DF901220021292000F028F9050053D00D
:100800002000A4F10104A4B2EED14DE000246F4613
:10081000FF2000F0E1F83855641CA4B2042CF7D393
:100820009DF80200012847D19DF80300AA2843D172
:1008300044464FF0804801220021372000F006F99D
:1008400001224146292000F001F9050004D02000D2
:10085000A4F10104A4B2EED1B4B1012200213A20E6
:1008600000F0F4F880B90024FF2000F0B5F8385506
:10087000641CA4B2042CF7D39DF80000400601D5F7
:10088000062000E00420307016E00120307044465D
:1008900001220021104600F0D9F8050004D0200004
:1008A000A4F10104A4B2F3D12CB101225102102011
:1008B00000F0CCF800B13770FFF7E4FE102000F034
:1008C000B5F9307810B10020BDE8F8830DB12846A5
:1008D000FAE7AA20F8E70000180000202DE9F0410F
:1008E0000646184815460078062800D049024FF4FD
:1008F0000077012D4FF0010219D0122000F0A6F868
:100900003946304600F020F86D1E044606F50076A4
:1009100015F0FF0501D0002CF2D0012200210C209F
:1009200000F094F8FFF7AEFE2046BDE8F0811120FC
:1009300000F08CF80400F5D13946304600F004F898
:100940000446EFE71800002070B504460D46FE206F
:10095000FFF7BBFE28B1012070BD00F03BF904F8A1
:10096000010B2800A5F10105ADB24FF0FF00F4D155
:1009700000F030F9FF2000F02DF9002070BD0000DC
:1009800038B501210420FFF711FE01211020FFF7E7
:100990000DFE1024ADF8004014208DF80300032054
:1009A0000B4D8DF8020069462846FFF7D0FCADF8E4
:1009B000004048218DF8031069460648FFF7C7FC40
:1009C00000F0C4F8012210212846FFF710FD38BDC1
:1009D000000801400010014000F0FCB810B50022F2
:1009E00010210548FFF703FD00F061F8002802D050
:1009F000FFF748FE012010BD0008014070B50C460D
:100A0000054600F054F808B1012070BD204600F002
:100A1000E1F8FD2C18D000244FF40076285D00F09A
:100A2000D9F8641CA4B2B442F8D3FF2000F0D2F885
:100A3000FF2000F0CFF8FF20FFF7CEFF00F01F00EF
:100A4000052801D0022070BD002070BD70B516468B
:100A50000C460546FFF716FEFFF7C0FF08B1FF2062
:100A600070BD45F0400000F0B5F8200E00F0B2F87F
:100A7000C4F3074000F0AEF8C4F3072000F0AAF872
:100A8000E0B200F0A7F8304600F0A4F80C2D02D137
:100A9000FF2000F09FF8FF24FF20FFF79DFF0106D5
:100AA000DED52100A4F10104E4B2F5D170BD10B58A
:100AB0000024FF20FFF790FFFF2804D0641C601C77
:100AC000F7D1012010BD002010BD000070B5064612
:100AD0001D4815460C460078062800D04C02012D12
:100AE00013D0012809D0012200213720FFF7AEFFE3
:100AF000012229461720FFF7A9FF012221461920CC
:100B0000FFF7A4FF04000AD01AE0012221461820B2
:100B1000FFF79CFF040013D1FE2130460DE0FC21BD
:100B20003046FFF76BFF6D1E06F5007615F0FF05EA
:100B300001D00028F3D0FD210020FFF75FFF04461D
:100B4000FFF7A0FD204670BD1800002010B586B04C
:100B500001210520FFF72AFD01210803FFF726FDEB
:100B6000E020ADF8140018208DF8170003208DF850
:100B7000160005A91548FFF7EAFB0020ADF80000B4
:100B80004FF48271ADF80210ADF804000221ADF807
:100B900006100121ADF808104902ADF80A103821FD
:100BA000ADF80C10ADF80E000720094CADF81000A0
:100BB0006946204600F05DF80121204600F044F827
:100BC000FF2000F007F806B010BD0000000801404B
:100BD000003001402DE9F041074600244FF4FA654A
:100BE000114E03E0641CA4B2AC420FD8022130467F
:100BF00000F034F80028F5D03946304600F037F8D8
:100C0000002406E0641CA4B2AC4202D90020BDE876
:100C1000F0810121304600F021F80028F2D0304662
:100C200000F023F8C0B2F2E7003001400146054869
:100C3000028822F03802028002880A4302800121E1
:100C400000F002B8003001400029018802D041F0D4
:100C5000400101E021F04001018070470246002080
:100C600012890A4200D00120704780897047818133
:100C7000704730B502884C8802F441530A88CD8809
:100C800022438C882C4322430C8922434C892243E3
:100C90008C892243CC8922431A430280828B22F41E
:100CA00000628283098A018230BD70470CB500233F
:100CB0002E4800930193016841F4803101604FF6A2
:100CC000FF71026802F400320192009A521C0092F5
:100CD000019A12B9009A8A42F3D10168890342D578
:100CE0000121019122490A6842F010020A600A6853
:100CF00022F003020A600A6842F002020A604168B8
:100D0000416041684160416841F480614160C16A6D
:100D1000184A1140C162C16A174A1143C162016891
:100D200041F08061016001680901FCD5416821F44E
:100D30007C114160416841F4E8114160016841F073
:100D40008071016001688901FCD5416821F00301CF
:100D50004160416841F0020141604168C1F3810195
:100D60000229FAD10CBD01930CBD00000010024015
:100D70000020024000F0FEFF140801000C488168CA
:100D8000491C81604168491C416081684FF47A7256
:100D9000B1FBF2F302FB1311012902D1C168491C16
:100DA000C1600178002901D1012101707047000064
:100DB000500000200B484FF47A710068B0FBF1F04E
:100DC000B0F1807F0DD220F07F414FF0E020491E2E
:100DD0004161054AF0211170002181610721016103
:100DE0007047FEE70400002023ED00E0124810B534
:100DF000016841F0010101604168104A1140416001
:100E000001680F4A11400160016821F480210160EE
:100E1000416821F4FE014160016821F0A0510160A8
:100E20004FF47F0181600021C162FFF73FFF054958
:100E30004FF00060086010BD001002400000FFF09D
:100E4000FFFFF6FE08ED00E010B50A4C0121204638
:100E500000F017F800280AD00121204600F00EF813
:100E60000549D1F8900118B10020C1F8900110BDDA
:100E70000120FAE70004004000002342C943018238
:100E8000704702460020138A92890B4202EA01024F
:100E900002D0002A00D001207047FEE702E008C817
:100EA000121F08C1002AFAD170477047002001E0E4
:100EB00001C1121F002AFBD17047000070B50F4C12
:100EC0008318A34201D9032070BDA2B101250023DC
:100ED0000BE004780E78A64204D0FF2C01D002204B
:100EE00070BD0025401C491C5B1C9342F1D3012DB1
:100EF00001D0012070BD002070BD0000000002087C
:100F00002DE9F0418846074615462649042628441F
:100F1000884202D90120BDE8F081EDB3E80700D096
:100F2000551C2A4641463846FFF7C8FF0400F2D058
:100F3000012080F31088FFF7EDF93520FFF762F903
:100F4000022C06D1F80AC002FFF762F9064604280F
:100F500021D14FF47A700100A0F1010080B2FAD1E2
:100F600000240EE008EB440118F81400497840EA28
:100F700001213846FFF788F90646042804D1BF1C32
:100F8000641CB4EB550FEDD3FFF776F9002080F326
:100F90001088042E03D000E001E00220BBE700200F
:100FA000B9E700000000020810B5044600202071D7
:100FB000401EE062204601F0AAFA08B1032010BDED
:100FC000B4F82E02A0F52A41553901D0022010BDF7
:100FD00094F86600B4F8671040EA01210848B0EBC5
:100FE000012F08D094F88210B4F8832041EA02213E
:100FF000B0EB012F01D1002010BD012010BD000079
:101000000046415400E0401C02780AB18A42FAD1FD
:10101000D0B2704770B5FFF77DF90C4C4020E0600E
:101020003420FFF7EFF80020094DA06007E005EB42
:101030008020FFF7EDF86070A068401CA060E168B8
:10104000884202D261780429F1D070BD18000020D6
:1010500000800008426A0068121D490A8078B1FBCE
:10106000F0F002CA21B1884204D3401A121DF8E7F9
:10107000002070471168084470474269891E921E1B
:101080008A4201D800207047826A807801FB0020E4
:1010900070472DE9F0410F00064606D001F02CF90B
:1010A000022809D20120BDE8F081F56815B1706908
:1010B000A84207D8012505E0411CF4D0716981429E
:1010C000F1D83D462C467069641CA04202D8022427
:1010D000022D0AD32146304601F00EF938B1411CE9
:1010E000E1D00128DFD0AC42EDD10020DBE76FF08A
:1010F00070422146304601F0E9FA30B957B1224634
:101100003946304601F0E2FA20B101280DD0012421
:101110002046C8E7F4603069411CF9D0401E3061B8
:10112000707940F001007071F2E74FF0FF34EFE7A3
:101130002DE9F35F88460D6800E06D1C28782F28A4
:10114000FBD05C28F9D0009800242646D0F81C90EB
:10115000A85D761C202815D32F2813D05C2811D029
:10116000FF2C2FD2012100F0DBFE07002AD0802FB8
:1011700004D201465FA0FFF745FF18BB29F81470A1
:10118000641CE5E7AA19C8F80020202801D204262B
:1011900016E0002614E009EB440030F8020C202889
:1011A0000DD02E280BD06CB1002129F81410009816
:1011B0000B222021806901F0A3F9002706E0641EBC
:1011C000002CE8D10620BDE8FC9F7F1C39F81700F1
:1011D0002028FAD02E28F8D01FB146F0030600E0F0
:1011E000641E2CB109EB440030F8020C2E28F7D114
:1011F0004FF0000AD0464FF0080B39F817507F1C0B
:1012000005B3202D03D02E2D04D1A74202D046F0E5
:101210000306F2E7DA4501D2A74219D1BBF10B0F61
:101220000ED0A74201D046F003060BD84FEA8860E3
:1012300027464FF0080A4FF00B0B4FEA1068DCE727
:1012400046F00306009880690178E5292ED02FE04A
:10125000802D0CD30021284600F062FE050003D04B
:101260002748284410F8805C46F0020625B129463C
:1012700024A0FFF7C7FE18B15F2546F003060EE075
:10128000A5F14100192802D848F0020807E0A5F1AD
:101290006100192803D8203D48F00108ADB200983C
:1012A000816901F80A500AF1010AA6E705210170D7
:1012B000BBF1080F03D14FEA88604FEA1068C8F30A
:1012C0008100032803D06FEA0801890701D146F0A5
:1012D0000206B10709D408F00301012901D146F043
:1012E0001006012801D146F0080600988069C672F0
:1012F000002068E7222A3A3C3E3F7C7F0000000045
:10130000B82900082B2C3B3D5B5D000070B50E46F4
:101310000546002100F087FA88B900242969286869
:1013200001F0F5F858B969690978E5290BD051B190
:1013300000240121284600F0A1F80028EED004285E
:1013400000D1072070BD641CB442F2D170BD000012
:101350002DE9F05F0446002100F065FA00287AD1FB
:10136000FF254FF6FF70AB4620842169206801F00D
:10137000CEF807007CD16669307848B1F17AE5286B
:1013800001F03F0169D00A0704D50F2965D105E0B6
:1013900004276DE00F2901D08DB34DE0E16979B3E9
:1013A000420606D596F80DB020F04000E2880546CA
:1013B0002284A84236D1727B5A4533D130788A468E
:1013C00020F04000401EB14600EB800101EBC0065A
:1013D0004FF000080127284810F8081001EB090019
:1013E000008877B100F0BCFD0746FF2E1AD23AF80C
:1013F0001600761C00F0B4FDB84213D105E016E0EB
:101400002FE0A0F57F41FF390CD108F10108B8F1B8
:101410000D0FE0D399F80000400606D52FB13AF839
:10142000160010B1FF25EDB21BE06D1EFBE7304644
:1014300001F022FA58451BD0A069C17AC9070CD126
:101440000B210022491E07D316F8012B10F8013B8F
:10145000D21AF7D001E00CE052B14FF6FF70FF2531
:1014600020840021204600F009F807003FF47DAFFA
:101470003846BDE8F09F0000382A00082DE9F04109
:10148000C78804467F1C38040E46000C2CD0206907
:1014900050B339075AD1401C2061E168206829B156
:1014A0008278521E12EA171F04D04FE00089B8421A
:1014B0001AD94BE000F020FF0546012819D9681C15
:1014C00030D020684169A9423AD86EB1E168FFF78F
:1014D000E0FD05000BD0012D0BD0681C22D0206848
:1014E00001F02FFAF0B906E00420BDE8F0810720F2
:1014F000FBE70220F9E720684FF40072303000214A
:1015000000F0FEFF29462068FFF7B7FD216800269E
:101510004FF00108C8620CE080F80480206801F0F8
:1015200010FA08B10120E0E72068C16A491C761C66
:10153000C16220688178B142EED8C16A891BC1625C
:10154000E56029462068FFF798FD2061E78007F0F5
:101550000F013022206802EB411108446061002035
:10156000C3E700002DE9F35FFF2504462E4604275C
:101570004FF6FF7A4FF0000B67E0206800F0C7FFDE
:10158000070066D16269107878B1D17AE52801F058
:101590003F0108D02E2806D0082908D00023DDF806
:1015A00004C0634505D0FF2540E0042751E0012336
:1015B000F5E70F2901D0B5BB3FE0410605D5567BC5
:1015C00020F04000E18805462184A8422CD1507BC0
:1015D000B04229D11078DFF8849000F03F00401E1F
:1015E00000EB800101EBC0010020E7690123D44634
:1015F00019F800809044B8F8008033B1FF2913D265
:1016000027F811804346491C01E0E0450CD1401CFD
:101610000D28EDD31078400603D5FF2904D227F812
:1016200011B06D1E01E00DE0FF25EDB20021204656
:10163000FFF724FF070008D00BE0104601F01CF96B
:10164000B04208D0A4F820A005E02169002994D177
:101650000FB1C4F810B03846BDE8FC9F382A000826
:101660002DE9FF5F04460C22D4E906763946684628
:1016700000F03EFF9DF80B00C00718D00020F87264
:101680000125E0612B4632466946384600F0F2FDFE
:101690002046FFF75DFE10B96D1C642DF2D3642D5A
:1016A0000BD004280AD19DF80B00F872E6619DF872
:1016B0000B0080070FD5002004E0072004B0BDE830
:1016C000F09F401C36F810100029FAD119300D2176
:1016D000B0FBF1F500E0012529462046FFF716FE94
:1016E00006006BD16D1E50D0E088411B204600F0F3
:1016F0009AF8060062D1A06901F0BEF84FF6FF7AB1
:1017000003902169206800F002FF060056D161694C
:10171000D4F81C90039848730F20C87200200873F7
:101720008876EEB2C876701E00EB800202EBC00332
:101730000022DFF88CB001F1010801E0504502D031
:1017400039F813005B1C1BF802C001F80C001BF8F1
:1017500002704FEA102C07F808C000B95046521C1E
:101760000D2AEBD3504502D039F8130008B946F0E2
:1017700040060E7021680120087100212046FFF705
:101780007DFE06001AD16D1EBBD12169206800F0D4
:10179000BEFE060012D120220021606900F0B0FEDA
:1017A000D4E905010B2200F0A3FEA0696169C07AAB
:1017B00000F01800087321680120087130467DE7A9
:1017C000382A00082DE9F041018C0446C688A1F5AD
:1017D0007F40FF3800D13146204600F024F8050054
:1017E0001ED1E5274FF001082169206800F08FFE27
:1017F000050012D120220021606900F081FE60699D
:101800000770216881F80480E088B04208D2002186
:101810002046FFF733FE0500E6D0042D00D1022557
:101820002846BDE8F08170B5C18083680D46044646
:10183000012B34D020684169994230D923B901780D
:10184000032904D1436A13B18078060110E00189AD
:10185000A94224D9406A11E000F04EFD0346401C25
:101860001BD0022B1BD320684069984217D9AD1BAF
:101870002068B5421946EFD2FFF7FFFBE36070B175
:1018800000EB1510206105F00F013022206802EBFB
:10189000411108446061002070BD012070BD02202C
:1018A00070BD10B530B9FEF75BFF002803D0FF20F4
:1018B000FFF792F8012010BD10B5144660B939B198
:1018C000012912D0022909D003290AD0042010BD11
:1018D000FFF7EDF80028FAD0012010BD4FF400709A
:1018E00000E008201080002010BDFEF702FF2060FD
:1018F000F9E770B514460D460BB160B901E004205C
:1019000070BDDAB221462846FEF7E8FF0028F7D07E
:10191000FF20FFF761F8012070BD0020704770B50F
:1019200014460D460BB148B901E0042070BDDAB28F
:1019300021462846FFF7CAF80028F7D0012070BDDD
:1019400010B5044600F080F9002806D1204601F0C9
:1019500020F8002801D10021216010BD17B581B009
:10196000144602980090684600F023FD002802DA31
:101970000B2004B010BD0B4B002253F8201001B116
:101980000A700199002900D00A7043F8201001D094
:10199000012C01D00020ECE7002202A901A800F0F0
:1019A000F1FAE6E7EC0C00202DE9F74F8CB00600C9
:1019B0000ED04FF0000902F01F0727F001020DA919
:1019C0006846C6F8009000F0DDFA040004D095E007
:1019D00009200FB0BDE8F08F4FF4007000F0BCFAA2
:1019E0005FEA00080AD009A8CDE9060868460D9903
:1019F00000F0E4FB059D040002D003E01120E8E7BD
:101A000005B9062417F01C0F4CD054B1042C03D197
:101A10006846FFF725FE0446059D47F0080754B1C8
:101A200052E0E87A10F0110F01D007244CE078075B
:101A300001D5082448E0380742D500F0B8FCA87367
:101A4000010AE973010C2974000E687485F80B9083
:101A500085F81C9085F81D9085F81E9085F81F90DC
:101A60002946009800F0C3FC82460021284600F079
:101A7000FBFE00990120BAF1000F08711ED00098FA
:101A80005146D0F82CB000F09DFE04001CD1009906
:101A9000AAF10100C8605946009800F038FD040022
:101AA0000AD011E084B9E87AC10601D504240BE01C
:101AB000B90701D5C007B8D1380701D547F02007CD
:101AC0000098C06AC6E90705404600F047FAACB97D
:101AD000B77186F807904F462946009800F087FCBA
:101AE0003061287FD5F81D1040EA0120C6E9027058
:101AF000B761776200983060C088B080204668E7A0
:101B00002DE9F84F894600219A4616460446196089
:101B100000F03FFF002812D1E07900280FD1A07912
:101B2000C0070BD0D4E90210401A04F128014FF08D
:101B3000010B0091864200D9064680E00720BDE8EF
:101B4000F88FA168C80562D120688278521E02EA27
:101B5000512212F0FF0510D129B1626A2AB1204644
:101B6000FFF778FA04E0206902E0616900F0C4FB45
:101B7000022819D3411C44D0606161692068FFF7D5
:101B80007CFA88B100EB0508770A21D02068EA19B1
:101B900081788A4200D94F1B40783B4642464946ED
:101BA000FFF7A7FE68BB02E00220E071C7E7A0795B
:101BB00040060BD5A169A1EB0800B84206D209EB9B
:101BC00040204FF40072009900F092FC7D022CE05E
:101BD000A269424519D0A07940060AD520680123A0
:101BE00000994078FFF79BFE58B9A07920F040009B
:101BF000A07120680123424640780099FFF779FEE2
:101C000018B184F807B0012099E7C4F8188020893A
:101C1000C0F30800C0F50075B54200D9354601197A
:101C200028312A46484600F063FCA068A9442844AD
:101C3000A060DAF800004119761BCAF80010002EE7
:101C40007FF47FAF00207AE770B5044600F0A1FE74
:101C500000280ED1A1798A060BD548060ED520683A
:101C6000012304F128014078A269FFF758FE08B16A
:101C7000012070BDA07920F04000A071E1692068CA
:101C800000F045FC0028F4D1256AE87A40F02000F5
:101C9000E872207B2877A089000A6877E068000C4A
:101CA000A877E068000EE8772846216900F0DCFD9F
:101CB00000F07DFBA875010AE975010C2976000E7C
:101CC00068760020A874E874A07920F02000A07144
:101CD0002168012008712068BDE8704000F0D9BD7E
:101CE000F1B596B0012216A9684600F04BF9040040
:101CF00053D14FF4007000F02FF9070009D012A85B
:101D0000CDE906076846169900F058FA040003D09A
:101D100040E0112017B0F0BD059E56B1F07AC00723
:101D200000D007243146009800F061FB054614B14D
:101D300030E00624F6E7F07AC0061BD5022D01D26A
:101D4000022427E02422694609A800F0D1FB0221E1
:101D500009A80B95FFF767FD04001BD1002109A816
:101D6000FFF700FC040003D0042C03D014B111E0F1
:101D700007240FE06846FFF725FD04000AD12DB1C6
:101D80002946009800F01EFD040003D1009800F0E1
:101D900080FD0446384600F0E1F82046BAE72DE918
:101DA000F84F894600219A4616460446196000F00D
:101DB000F0FD002806D1E079002803D1A079800742
:101DC00002D40720BDE8F88FA06804F12801821929
:101DD0004FF0010B0091824273D392E0A168C805D5
:101DE00073D122689078401E00EA512010F0FF0560
:101DF00018D129B1606A38B12046FFF72BF907E006
:101E0000206938B9002100E061691046FFF741F907
:101E1000002879D001282BD0411C4ED06061216967
:101E200001B92061A07940060BD520680123A26981
:101E300040780099FFF773FD78BBA07920F040004F
:101E4000A07161692068FFF718F988B100EB0508F7
:101E5000770A23D02068EA1981788A4200D94F1B7B
:101E600040783B4642464946FFF759FDA8B902E093
:101E70000220E071A6E7A169A1EB0800B8420AD2EE
:101E800009EB40214FF40072009800F031FBA0797B
:101E900020F04000A0717D0229E00EE0A1694145DB
:101EA00011D0D4E9020188420DD2206801234246B4
:101EB00040780099FFF71DFD28B184F807B0012094
:101EC00080E721E001E0C4F818802089C0F3080011
:101ED000C0F50075B54200D93546204428302A4661
:101EE000494600F005FBA07940F04000A071A068D1
:101EF000A9442844A060DAF800004119761BCAF80A
:101F00000010002E7FF46AAFD4E90201884200D9A4
:101F1000E060A07940F02000A071002052E70000AE
:101F2000802804D30B4A49B1FF2801D9002070470B
:101F300002EB4000A0F580700088704732F8113045
:101F4000834203D0491C89B28029F7D38031C8B2BB
:101F500070470000722A000800F094BA00F062B9DD
:101F60000021064B00E0491C33F81120002A04D060
:101F70008242F8D1024830F811007047722B0008F5
:101F8000522D00082DE9FF474FF000090746C0F821
:101F900000901646084600F00CFA051E03DA0B20E6
:101FA00004B0BDE8F087814850F825408CB13C6012
:101FB000207820B16078FFF7B0FCC1070BD084F81F
:101FC0000090E8B26070FFF76CFCC10708D00320F6
:101FD000E6E70C20E4E70EB1400704D40020DFE779
:101FE0001EB1400701D50A20DAE700252946204620
:101FF000FEF7DAFF012821D100206E4604EB001124
:1020000001F5F7710A792AB10A7AD1F8091042EA82
:10201000012100E0002146F82010401C0428EDD3E7
:10202000002756F8275025B129462046FEF7BCFF69
:1020300000E0022040B17F1C042FF2D3032801D01E
:10204000F0BB01E00120ABE7B4F83B00B0F5007F46
:102050005DD1B4F8461029B994F85400D4F855105D
:1020600040EA0121A16194F840C084F803C0BCF1AA
:10207000010F02D0BCF1020F49D194F83D600CFB76
:1020800001FCA670E6B1701E064240D1B4F84120B2
:10209000228110073BD1B4F8430028B994F85000CE
:1020A000D4F8513040EA0320E38F4BB103EB0C0727
:1020B00007EB1217B8422AD3C01BB0FBF6F000E0C2
:1020C00025E020B3012640F6F678404500D30226ED
:1020D0004FF6F678404500D30326801C2F44A762B4
:1020E0002B446061C4E90753032E12D07AB103EB8D
:1020F0000C026262022E17D000F0010200EB4000D9
:1021000002EB500000F2FF10B1EB502F0ED20D2069
:1021100046E7002AFBD194F85C20D4F85D308000BB
:1021200042EA03226262EDE74000EBE74FF0FF3046
:102130002061E06080206071032E30D1B4F860002F
:1021400001282CD1691C204600F0E1F938BB84F845
:102150000590B4F82E02A0F52A4155391FD194F804
:102160003000D4F8311040EA01201149884216D1DC
:1021700094F81402D4F8151240EA01200D4988425F
:102180000DD194F81802D4F8191240EA0120206108
:1021900094F81C02D4F81D1240EA0120E0600649C0
:1021A00026700888401C0880E08017E7EC0C0020AF
:1021B00052526141727241617400002073B504464D
:1021C000019908782F2801D05C2801D1491C019180
:1021D0000025A56001980078202805D2002120461E
:1021E000FFF721FB65617CBD01A92046FEF7A0FF3A
:1021F0000028F8D12046FFF7ABF8A169C97A28B1C9
:102200000428F0D14907EED405207CBD4907FCD451
:102210006169C87AC006F7D5206800F0E8F8A060C8
:10222000E2E7000010B5002821D0114B001F00226A
:10223000196803E0814203D80A4649680029F9D1A8
:1022400052B11368841A9C4204D10068184410608B
:10225000104602E0506000E0186039B102680B1AC5
:10226000934203D10B681A4402604968416010BD73
:10227000780000207CB516461C4605460B2200F06F
:1022800037F9052C14D91B4A0FE006F102064FF06E
:1022900000012346044663F35F044FEA5000E30362
:1022A00000D55440491C1029F3D330880028ECD1C4
:1022B00007216B4604F00F003030392800D9C01DCB
:1022C0005854491E2409F5D17E205854002200E0BC
:1022D000521C8A4202D2A85C2028F9D1082902D2D5
:1022E000585C491C00E02020A854521C082AF5D351
:1022F0007CBD0000211001002DE9F0410D4604468F
:10230000022909D36069A84206D92078012806D09D
:10231000022828D0032832D00120BDE8F081206AAD
:1023200005EB550600EB5621204600F0F0F868BB9F
:10233000C6F308002044761C90F83070206A00EB49
:102340005621204600F0E3F800BBC6F30800204405
:10235000E90790F8300047EA002001D00009DCE7E7
:10236000C0F30B00D9E7206A00EB1521204600F0EE
:10237000CEF858B9E8B204EB4000008ECDE7206AF1
:1023800000EBD511204600F0C2F810B14FF0FF303D
:10239000C3E740F2FF1000EA8500204490F83010B7
:1023A000D0F8310041EA002020F07040B5E700206D
:1023B000704710B503464FF0FF301C68002C13D057
:1023C000214600E0491C0A78202A0ED33A2AF9D186
:1023D00014F8012B303A0A2A06D28C4204D1032A7F
:1023E00002D2491C1046196010BD002010BD0246E3
:1023F000488B1278032A02D1898A40EA014070474B
:1024000086B0FEF7F3FCFEF7D5FC6846FEF7DAF877
:10241000FEF7BCF8FDF7F0FF0A20FDF7EBFEFEF734
:1024200047F84FF004084FF00209124D4FF0030A2D
:10243000114E124F124CFDF7F3FF2878012808D0F7
:102440007068386020603068FDF795FE206880472E
:10245000F1E785F8008000F071F810B185F800A070
:10246000E9E7C820FDF7C6FE85F8009000F0DCF92A
:10247000E1E7000000000020008000084800002084
:1024800044000020F0B50B30154D20F0070100246A
:10249000144A0FE003688B420BD38B4205D95E1AB6
:1024A00043184768C3E9006700E04368136002C04F
:1024B00004E0021D10680028ECD12046002802D15B
:1024C000286808B10020F0BD064A07481060074A96
:1024D000121A22F00702C0E9002401202860D7E781
:1024E0007C00002078000020FC0C0020F80E00206A
:1024F00003E011F8013B00F8013B521EF9D270478E
:10250000C9B201E000F8011B521EFBD2704770B542
:102510000446C06A0D46A8420ED0204600F011FACB
:1025200038B9607801232A4604F13001FFF7E1F958
:1025300008B1012070BDE562002070BD2DE9F041B9
:102540004E4DADF58A6D002401224DA14D486C61C0
:10255000FFF704FA06460520FDF74CFE01224AA1CA
:102560006846FFF721FAE87001224AA16846FFF7A2
:102570001BFAE87001224AA16846FFF715FAE870D5
:1025800030004FF0FF3605D06846FFF7D9F9012239
:1025900046A10FE00520FDF72DFE0398A8610B2250
:1025A00043A18AA8FFF700FA60B18AA8FFF7C8F92B
:1025B000012242A10020FFF7D1F930460DF58A6DC6
:1025C000BDE8F081FEF726FDAC804FF40047DFF850
:1025D000F0803C4C3E11A87840B10020A870002843
:1025E0003946404604D0FDF7FEFE03E00120F5E742
:1025F000FDF7FBFEA888314604EBC0202861324875
:10260000FDF7D9FD1D4B324614332F496846FFF7BD
:1026100077FA00BB6A69F2B1B24205D2A8882A49AA
:1026200004EBC020FEF76CFC144B27491C338AA82E
:102630006A69FFF7B4FB8AA8FFF706FB6A69B24232
:1026400005D1A888204904EBC020FEF759FCA888D2
:10265000401CA880BFE78AA8FFF772F96846FFF719
:102660006FF9012211A10020FFF778F9012213A1CF
:102670000020FFF773F90020A0E7000018000020F9
:10268000303A00008C000020303A2F4170702E62EA
:10269000696E0000303A2F546573742E747874009C
:1026A000303A2F546573742E62696E00303A2F00F1
:1026B000303A2F746573742E62696E00313A2F00C0
:1026C0000008014000800008EC0400202DE9F047DC
:1026D00016460D460446022902D36069A84202D874
:1026E0000220BDE8F087207806F0FF084FF00109CE
:1026F000012807D0022837D0032846D0022084F8CA
:102700000490EEE7206A05EB550700EB57212046C1
:10271000FFF7FDFE0028F2D1C7F308002044303057
:10272000E90703D0017868F31F1100E0314601701A
:1027300084F80490206A7F1C00EB57212046FFF7A5
:10274000E6FE0028DBD1C7F3080121443031EA0757
:1027500002D0C6F3071205E00A78C6F3032302F09D
:10276000F0021A430A70CAE7206A00EB15212046DE
:10277000FFF7CDFE0028C2D1E9B204EB4101320AD5
:1027800081F8308081F83120B9E7206A00EBD5115B
:102790002046FFF7BCFE0028B1D140F2FF1101EA4C
:1027A0008501214430314FF07043D1F8012003EA14
:1027B000022232430A70130A4B70130C8B70120EF4
:1027C000CA709CE72DE9F0410F460446022916D352
:1027D0006069B84213D900261FE039462046FFF74A
:1027E0008BFD05001CD0012D09D0681C09D00022EA
:1027F00039462046FFF76AFF060011D103E00226A2
:102800000EE001260CE02069411C05D0401C20612F
:10281000607940F0010060712F466069B842DCD8F1
:102820003046BDE8F081000010B5012206A107483E
:10283000FFF794F806A0FFF753FA0122BDE8104015
:1028400008A10020FFF78AB8303A00008C00002071
:10285000303A2F55706C6F6164436F6E6669672EF6
:1028600074787400303A2F0081760A0AC2760A0C16
:102870000275090E41757047014600200B2243087E
:1028800003EBC01011F8013B521E1844C0B2F6D140
:10289000704770B5044600F054F805004FD1207819
:1028A000032845D16079012842D1420204F1300069
:1028B00000210646FFF724FE552084F82E02AA20A8
:1028C00084F82F02522084F8300084F8310061220D
:1028D00084F83220412084F83300722184F81412E5
:1028E00084F8151284F8160284F81722206984F8F7
:1028F0001802010A84F81912010C84F81A12000E49
:1029000084F81B02E06884F81C02010A84F81D1296
:10291000010C84F81E12000E84F81F02E2690123E4
:10292000521CE26260783146FEF7F9FF00206071C8
:10293000002260781146FEF7BFFF00B1012528464E
:1029400070BD2DE9F0410446007900B3E66A04F158
:1029500030016078012332460F46FEF7E0FF10B1E8
:102960000120BDE8F08100202071206AA169301AA1
:1029700088420CD2E57808E0A0690123064460781B
:1029800032463946FEF7CBFF6D1E022DF4D20020F1
:10299000E7E710B538B1016829B10A781AB1CA88D9
:1029A0008088824201D0092010BD4878FEF7B5FF2B
:1029B000C007F9D0032010BD809A90418E418F80CE
:1029C0004545454949498E8F9092924F994F5555AB
:1029D00059999A9B9C9D9E9F41494F55A5A5A6A795
:1029E000A8A9AAABAC21AEAFB0B1B2B3B4B5B6B77B
:1029F000B8B9BABBBCBDBEBFC0C1C2C3C4C5C6C7DF
:102A0000C8C9CACBCCCDCECFD0D1D2D3D4D5D6D7CE
:102A1000D8D9DADBDCDDDEDFE0E1E2E3E4E5E6E7BE
:102A2000E8E9EAEBECEDEEEFF0F1F2F3F4F5F6F7AE
:102A3000F8F9FAFBFCFDFEFF01030507090E101271
:102A40001416181C1E000004000200018000400043
:102A50002000100008000400020000000080004078
:102A600000200010000800400020001000080004B2
:102A70000002C700FC00E900E200E400E000E5001D
:102A8000E700EA00EB00E800EF00EE00EC00C40015
:102A9000C500C900E600C600F400F600F200FB0025
:102AA000F900FF00D600DC00A200A300A500A720CB
:102AB0009201E100ED00F300FA00F100D100AA005C
:102AC000BA00BF001023AC00BD00BC00A100AB00E9
:102AD000BB00912592259325022524256125622599
:102AE000562555256325512557255D255C255B25F4
:102AF0001025142534252C251C2500253C255E2574
:102B00005F255A25542569256625602550256C25A5
:102B1000672568256425652559255825522553259F
:102B20006B256A2518250C25882584258C2590255C
:102B30008025B103DF009303C003A303C303B500E3
:102B4000C403A6039803A903B4031E22C603B50356
:102B500029226122B1006522642220232123F7006B
:102B60004822B0001922B7001A227F20B200A02507
:102B7000A0006100620063006400650066006700F9
:102B8000680069006A006B006C006D006E006F00E9
:102B90007000710072007300740075007600770099
:102BA000780079007A00A100A200A300A500AC0083
:102BB000AF00E000E100E200E300E400E500E60031
:102BC000E700E800E900EA00EB00EC00ED00EE00B1
:102BD000EF00F000F100F200F300F400F500F60061
:102BE000F800F900FA00FB00FC00FD00FE00FF0009
:102BF000010103010501070109010B010D010F018D
:102C0000110113011501170119011B011D011F01FC
:102C1000210123012501270129012B012D012F016C
:102C200031013301350137013A013C013E014001D8
:102C300042014401460148014B014D014F01510140
:102C400053015501570159015B015D015F016101AC
:102C500063016501670169016B016D016F0171011C
:102C60007301750177017A017C017E019201B10344
:102C7000B203B303B403B503B603B703B803B90390
:102C8000BA03BB03BC03BD03BE03BF03C003C10340
:102C9000C303C403C503C603C703C803C903CA03E8
:102CA0003004310432043304340435043604370468
:102CB000380439043A043B043C043D043E043F0418
:102CC00040044104420443044404450446044704C8
:102CD000480449044A044B044C044D044E044F0478
:102CE0005104520453045404550456045704580420
:102CF00059045A045B045C045E045F047021712172
:102D0000722173217421752176217721782179210F
:102D10007A217B217C217D217E217F2141FF42FF81
:102D200043FF44FF45FF46FF47FF48FF49FF4AFF77
:102D30004BFF4CFF4DFF4EFF4FFF50FF51FF52FF27
:102D400053FF54FF55FF56FF57FF58FF59FF5AFFD7
:102D50000000410042004300440045004600470097
:102D6000480049004A004B004C004D004E004F0007
:102D700050005100520053005400550056005700B7
:102D8000580059005A002100E0FFE1FFE5FFE2FF93
:102D9000E3FFC000C100C200C300C400C500C600FC
:102DA000C700C800C900CA00CB00CC00CD00CE00CF
:102DB000CF00D000D100D200D300D400D500D6007F
:102DC000D800D900DA00DB00DC00DD00DE0078018D
:102DD000000102010401060108010A010C010E01B3
:102DE000100112011401160118011A011C011E0123
:102DF000200122012401260128012A012C012E0193
:102E0000300132013401360139013B013D013F01FE
:102E100041014301450147014A014C014E01500166
:102E200052015401560158015A015C015E016001D2
:102E300062016401660168016A016C016E01700142
:102E400072017401760179017B017D019101910389
:102E500092039303940395039603970398039903AE
:102E60009A039B039C039D039E039F03A003A1035E
:102E7000A303A403A503A603A703A803A903AA0306
:102E80001004110412041304140415041604170486
:102E9000180419041A041B041C041D041E041F0436
:102EA00020042104220423042404250426042704E6
:102EB000280429042A042B042C042D042E042F0496
:102EC00001040204030404040504060407040804BE
:102ED00009040A040B040C040E040F046021612190
:102EE00062216321642165216621672168216921AE
:102EF0006A216B216C216D216E216F2121FF22FF40
:102F000023FF24FF25FF26FF27FF28FF29FF2AFF95
:102F10002BFF2CFF2DFF2EFF2FFF30FF31FF32FF45
:102F200033FF34FF35FF36FF37FF38FF39FF3AFFF5
:102F300000000000542F0008000000208000000066
:102F40009C0E0008D42F0008800000207816000096
:102F5000AC0E00080000000000A24A0400000000BF
:102F60000000000001020304060708090004000035
:102F70000000000000000000000000000000000051
:102F80000000000000000000000000000000000041
:102F90000000000000000000000000000000000031
:102FA0000000000000000000000000000000000021
:102FB00000000000020406080000000001020304F3
:102FC00001020304060708090000000000000000D9
:042FD00000000000FD
:04000005080001519D
:020000040800F2
:108000002074002065810008D1C80008EBBE00087C
:10801000CDC800080199000825ED00080000000007
:1080200000000000000000000000000091D80008DF
:108030008DB2000800000000A9D000082DDC000867
:1080400075EE00087F8100087F8100087F810008AD
:108050007F8100087F8100087F8100087F81000800
:108060007F8100087F8100087F8100087F810008F0
:108070007F8100087F8100087F8100087F810008E0
:108080007F8100087F8100087F81000889990008AE
:10809000059900087F810008259900087F81000864
:1080A0007F8100087F8100087F8100087F810008B0
:1080B0007F810008BDDD00087F8100087F81000806
:1080C0007F8100087F8100087F8100087F81000890
:1080D0007F810008EDE2000895E300086DE40008E8
:1080E0007F8100087F8100087F8100080000000078
:1080F0000000000000000000000000000000000080
:1081000000000000000000007F8100087F8100085F
:108110000DE1000805E200087F8100087F8100086A
:108120007F8100087F8100087F8100087F8100082F
:108130007F8100087F8100087F810008F59B00088F
:108140007F810008619B0008859B00087F810008F3
:10815000DFF80CD000F050FC00480047CD1E0108AD
:10816000207400200648804706480047FEE7FEE7E7
:10817000FEE7FEE7FEE7FEE7FEE7FEE7FEE7FEE7D7
:1081800001DD00085181000840EA01039B0703D08C
:1081900009E008C9121F08C0042AFAD203E011F846
:1081A000013B00F8013B521EF9D27047D2B201E008
:1081B00000F8012B491EFBD270470022F6E710B5EC
:1081C00013460A4604461946FFF7F0FF204610BD45
:1081D00030B505462A460B4612F8010B13F8014B41
:1081E00008B1A042F8D01CB1002802D06D1CF1E704
:1081F000284630BD421C10F8011B0029FBD1801A13
:10820000704730B504460020034600E05B1C9342F3
:1082100003D2E05CCD5C401BF8D030BDF0B480EA06
:108220000102D40F4200B2EB410F02D202460846CF
:1082300011464A0042D0C30DDDB2C1F3C752AD1A98
:10824000202D35DAC1F3160141F4000204B1524287
:10825000C5F1200602FA06F12A411044B3EBD05FC3
:1082600023D0C4B1012DA0EBC35009DCF0BC4FF00A
:10827000004202EAC352DBB200F5000000F019BB75
:10828000400000F1807000EBC350A0F1807040EA24
:10829000D170490009E0490841EAC071A0EBC35020
:1082A00000F50000400800EBC350F0BC00F0F8BA45
:1082B0006142012202EB4101001BF6E7F0BC70476E
:1082C00081F00041AAE780F00040A7E780EA0102C0
:1082D00010B502F00043400022D04A001FD0010E2A
:1082E00001EB1261C0F35600C2F3560240F40000E5
:1082F00042F40002A0FB022000047F39140400D0E5
:10830000401C50EA124001D44000491EC2B20C0683
:1083100004EBD010401C4008802A02D003E000206B
:1083200010BD20F00100002900DA0020184310BD24
:1083300030B480EA010202F0004530F0004221F042
:10834000004013D090B1C30DD40DC2F31601C0F399
:108350001600E41A41F4000140F400027D34914219
:1083600001D3641C00E04900002C02DA30BC00207C
:1083700070474FF400000023914201D3891A034350
:1083800040084FEA4101F7D151B1914202D14FF07B
:10839000004105E002D24FF0010101E06FF0010160
:1083A00003EBC450284430BC00F07ABA2DE9FE4FEC
:1083B000804681EA0300C00F0C46009021F0004186
:1083C00023F00045B8EB0200A94105D24046214602
:1083D00090461C460B46024623F00040104347D00F
:1083E000270DC7F30A00C3F30A510290401A019007
:1083F00040286BDAC3F3130040F4801B00989246C8
:1084000020B10023D2EB030A63EB0B0B0198594612
:10841000C0F14002504600F022FA06460D46504692
:108420005946019A00F02AFA10EB08006141002435
:1084300087EA115284EAE7731A4340D0009A62B384
:10844000019A012A4FEA075215DC001B61EB020179
:108450004FF0004202EA0752CDE90042001C41F50C
:10846000801132462B4600F061FA03B0BDE8F08F70
:1084700040462146F9E7001B61EB0201001C41F573
:10848000801300185B412018A2F5001747EB030189
:1084900040EAD570B6196D4111E06D084FEA360615
:1084A00045EAC0754FEA0752001B61EB0201001C50
:1084B00041F5801149084FEA300000195141324618
:1084C0002B4603B0BDE8F04F00F021BA009801221E
:1084D00040000023D0EB020263EBE07300982146DA
:1084E0004FEAE074B8EB000061EB0401E9E783F0C8
:1084F00000435BE781F0004158E72DE9FE4F81EA38
:10850000030404F0004421F0004100944FF0000BFC
:1085100023F0004350EA01045ED052EA03045BD02A
:10852000C3F30A54C1F30A552C44A4F2F334019462
:10853000A0FB0254C1F3130141F48011C3F31303F0
:1085400043F4801301FB024400FB034E840A970AA4
:1085500044EA815447EA8357A4FB076802958D0AD1
:1085600005FB07854FEA932C04FB0C542705029D5D
:108570004FEA065847EA1637B5EB08056EEB070CCD
:10858000870E920E47EA811742EA8312A7FB020187
:10859000B6EB0B0164EB00042B0D43EA0C335E18C1
:1085A00044EB1C50DA465146E7FB0201C5F31304C5
:1085B0004FEA0B3343EA14534FEA0432019C43EA77
:1085C0000603A4F10C040294009CCDE900B400F071
:1085D000ADF903B0BDE8F08F00200146F9E72DE9C1
:1085E000F04D81EA030404F0004B21F000451446ED
:1085F0004FF0000A23F0004150EA050220D054EA6F
:1086000001021DD0C5F30A570246C5F31303C1F397
:108610001300C1F30A5640F4801543F48013A7EB0E
:108620000608101BD64608F2FD3873EB050002D38E
:1086300008F1010801E092185B41B8F1000F03DA7C
:1086400000200146BDE8F08D00204FF48011064661
:1086500084460EE0171B73EB050705D3121B63EB73
:10866000050306434CEA010C49084FEA3000921812
:108670005B4150EA0107EDD152EA030012D082EAD1
:10868000040083EA0501084305D0101BAB4106D264
:108690000122002306E000224FF0004302E06FF0C9
:1086A000010253101AEB06004CEB085110EB0A00C4
:1086B00041EB0B01BDE8F04D00F029B9C10F80EA94
:1086C000E0700844CA079623002100F0F2B8962310
:1086D0000022114600F0EDB80EB540F23341029190
:1086E0000021CDE900110A460B4600F01FF903B046
:1086F00000BD20F00040C10DC0F3160040F40000A2
:108700007F2901DA00207047962903DCC1F1960128
:10871000C840704796398840704700F0004230F0FA
:1087200000400AD0C10D01F56071C0F3160042EAA5
:108730000151C208400711437047002001467047AD
:1087400030B5041E71F1000404DB4FF000444042D8
:1087500064EB0101141E73F1000405DB1C464FF0AD
:108760000043524263EB0403994208BF904230BD7C
:1087700001F0004330B421F0004150EA010206D07C
:108780000A0DA2F56072C1F31301002A02DC30BCAD
:1087900000207047440F44EAC104C100E01830BC17
:1087A00000EBC25000F07CB8002801DBC0F10040B3
:1087B000002901DBC1F1004181427047002801DB43
:1087C000C0F10040002901DBC1F10041884270473F
:1087D00030B50B46014600202022012409E021FA91
:1087E00002F59D4205D303FA02F5491B04FA02F58E
:1087F0002844151EA2F10102F1DC30BD2DE9F05F25
:108800000546002092469B468846064681464024FF
:108810001BE0284641464746224600F0FFF85346F3
:108820005A46C01A914110D311461846224600F00C
:1088300016F82D1A67EB01084F4622460120002149
:1088400000F00DF817EB00094E41201EA4F10104C1
:10885000DFDC484631462A464346BDE8F09F202AE1
:1088600004DB203A00FA02F1002070479140C2F187
:10887000200320FA03F3194390407047202A06DBB7
:10888000CB17203A41FA02F043EAE07306E041FADE
:1088900002F3D040C2F120029140084319467047CC
:1088A0000029A8BF7047401C490008BF20F0010004
:1088B000704710B4B0FA80FC00FA0CF050EA0104E2
:1088C00004BF10BC704749B1CCF1200421FA04F474
:1088D00011FA0CF118BF012121430843A3EB0C014D
:1088E000CB1D4FEA00614FEA102042BF002010BCB0
:1088F000704700EBC35010440029A4BF10BC704760
:10890000401C490008BF20F0010010BC704710B5A2
:10891000141E73F1000408DA401C41F100019218A2
:108920005B411A4301D120F0010010BD2DE9F04D4B
:1089300092469B4611B1B1FA81F202E0B0FA80F2A0
:1089400020329046FFF78BFF04460F4640EA0A00AC
:1089500041EA0B0153465A46084313D0114653EAE5
:10896000010019D0C8F14002504600F057F8054602
:108970000E46504659464246FFF771FF084305D060
:10898000012004E020463946BDE8F08D0020054373
:1089900046EAE0762C4337430A986305E40AA0EBE5
:1089A00008000022FD0A44EA47540A3002D500209C
:1089B0000146E9E7010510196941DDE9084500199B
:1089C0006941BDE8F04DA2E7C1F30A52C1F31301BA
:1089D00040F2FF3341F480119A4202DA002001464E
:1089E000704740F233439A42A2F2334202DC5242D1
:1089F00000F014B8FFF733BF064C074D06E0E068FF
:108A000040F0010394E8070098471034AC42F6D3D5
:108A1000FFF7A2FB1456010834560108202A04DB94
:108A2000203A21FA02F00021704721FA02F3D040E7
:108A3000C2F12002914008431946704770B58C1866
:108A400010F8015B15F0070301D110F8013B2A1162
:108A500006D110F8012B03E010F8016B01F8016B4F
:108A60005B1EF9D12B0705D40023521E0DD401F84B
:108A7000013BFAE710F8013BCB1A921C03E013F814
:108A8000015B01F8015B521EF9D5A142D8D3002049
:108A900070BD21B1826842F00102826003E0826809
:108AA00022F001028260704721B1826842F4807234
:108AB000826003E0826822F480728260704701461F
:108AC00000208A6802F004020AB1012000E00020C0
:108AD0007047014600208A6802F008020AB10120AE
:108AE00000E000207047000030B50246002000235F
:108AF00050680F4C20400D790C6844EA052420434F
:108B0000506090680B4C2040D1E902542C434D79C1
:108B100044EA450420439060D06A20F470000C7C45
:108B2000641EE4B2234340EA0350D06230BD00002B
:108B3000FFFEF0FFFDF7F1FFF0B504460D46002003
:108B40000021092D11DDE068A5F10A0606EB4607B4
:108B5000072606FA07F18843A5F10A0606EB460642
:108B600003FA06F10843E0600CE0206905EB4507D5
:108B7000072606FA07F1884305EB450603FA06F1D6
:108B800008432061072A0FDA606B561E06EB860742
:108B90001F2606FA07F18843561E06EB860605FADD
:108BA00006F10843606322E00D2A0FDA206BD61F1E
:108BB00006EB86071F2606FA07F18843D61F06EB49
:108BC000860605FA06F10843206310E0E06AA2F188
:108BD0000D0606EB86071F2606FA07F18843A2F169
:108BE0000D0606EB860605FA06F10843E062F0BDC5
:108BF000816841F008018160704721B1826842F4C8
:108C0000A002826003E0826822F4A00282607047C2
:108C1000816841F00401816070470000F8B50546A5
:108C20000E46002490208DF8000001208DF80100F0
:108C30008DF802608DF803500949086003F06AFA64
:108C400000BF08E01DF8040003F09EFA0A2000F0BF
:108C500029F8601CC4B2042CF4DB03F07BFAF8BDE5
:108C60009881214208B50121082004F0AFFBC02003
:108C7000ADF8000003208DF8020010208DF80300ED
:108C80006946054802F084FD012004490860044952
:108C9000C1F8980108BD0000000C01409C812142F0
:108CA0000080214200BF411E89B2081EFBD17047DF
:108CB00000B591B00121084604F058FB012140F2B3
:108CC000112004F083FB4FF4004004F043FB3920F3
:108CD000ADF8400000208DF8430010A9374802F09D
:108CE00057FD00200B900E904FF460200D90012056
:108CF0008DF8310004208DF83C0001208DF8300003
:108D00000BA92F48FFF7F0FE052301220A212C486A
:108D1000FFF712FF052302220D212948FFF70CFF60
:108D2000052303220E212648FFF706FF0523042210
:108D30000F212348FFF700FF21484C300090801599
:108D40000690002004901F4801904FF48060079027
:108D5000802005900020029004200390202008909D
:108D600000200A904FF4805009906946164802F09E
:108D70000FFA0121144802F0FFF901211048FFF712
:108D800093FE01210E48FFF784FE0D48FFF730FFE8
:108D900000BF0B48FFF79DFE0028FAD10848FFF7F7
:108DA00037FF00BF0648FFF78AFE0028FAD10121ED
:108DB0000348FFF722FF11B000BD00000010014082
:108DC0000024014060000020080002402DE9F0412D
:108DD00004460F460C2009F059FB054638882880C8
:108DE00078686860206830B9012020726560AD60E5
:108DF0002560BDE8F081266800E0B668B06861686B
:108E00008842FAD1B5602068A86000BFF1E7000091
:108E100070B502F02FF90E4909780E4A52F8210078
:108E200080470B4909780C4A52F8210080470446D4
:108E30000748007800EB4000084901EBC00050F8FB
:108E400024501DB12046A8470149087070BD00009C
:108E500088230020300700205007002070060020E3
:108E6000014601F00F000A0902EB820200EB42000A
:108E7000C0B2704710B5012004F0B8FA002004F029
:108E8000B5FA10BD10B5A2B0002441F204000C499F
:108E9000A1F80500202048800A48007C401C0949B0
:108EA000087409A006F046F801AA02A9044802F0D5
:108EB0008DF90021094805F03FF822B010BD0000EF
:108EC0007E1D0020041F002073656E6420436861CE
:108ED00072676520646174610A0D00009C050020C2
:108EE00010B5114890F86600642804D1062002F0FD
:108EF00033FA002010BD0C4A906E926ED1688847FC
:108F000020B91C2002F028FA0020F3E7064A906EF0
:108F1000926E5169884720B9212002F01DFA002085
:108F2000E8E70120E6E70000A007002010B5A2B0A6
:108F3000002441F209000A49A1F8050012204880E6
:108F40000848007C401C0749087407A005F0F2FFA0
:108F500001AA02A9024802F039F922B010BD0000AE
:108F60007E1D0020041F002053656E64204368614D
:108F70007267696E6744617461200A0D0000000029
:108F800000B5A1B00020009041F203000E49A1F805
:108F900005000E4801780C48817204200A49488077
:108FA0000B48007C401C0A4908740AA005F0C2FF67
:108FB0006A4601A9044802F009F900210A4804F0B0
:108FC000BBFF21B000BD00007E1D00200C02002070
:108FD000041F002073656E642073746174652064DF
:108FE000617461200A0D00009405002010B5242052
:108FF00002F082F90021034804F09EFF002002F0F5
:1090000033F810BD9823002010B5A2B0002441F21F
:1090100021001549A1F805001448007DC8711348C6
:10902000808A010A1048017210484069010C0E48FC
:1090300041720E484069000E0B4988720420488036
:109040000B48007C401C0A4908740AA005F072FF16
:1090500001AA02A9044802F0B9F804210248C01D7F
:1090600008F016F922B010BD7E1D0020381900202E
:10907000041F00200A0D7368656E676A6979696E5E
:10908000676461200A0D000010B5A2B000244FF4FF
:1090900081500F49A1F805005520C871AA210C483C
:1090A000017202200A4948800A48007C401C094994
:1090B000087409A005F03EFF01AA02A9044802F0C5
:1090C00085F802210248C01D08F0E2F822B010BD68
:1090D0007E1D0020041F00204F54412041434B209F
:1090E0000A0D000010B5A2B0002441F208001E498C
:1090F000A1F805001D481EA1096801601EA10968AC
:109100004160194819490968C0F8071017494968AA
:10911000C0F80B101548017A1348C1731348008931
:10912000010A1148017411488068010C0E4841740D
:109130000E488068000E0C4988740C48017B0A4870
:10914000C1740D20084948800D48007C401C0C4922
:1091500008740CA005F0EEFE01AA02A9024802F074
:1091600035F822B010BD00007E1D00203621002001
:109170005332303100000000574C494E4700000088
:10918000041F002073656E6420626D732076657223
:1091900073696F6E0A0D0000F0B503460C46FF259B
:1091A000FF261512D6B209E013F8010B80EA05017B
:1091B0000648405C80EA06050548465C201EA4F18E
:1091C0000107BCB2F0D146EA0520F0BD705101089C
:1091D0007052010870B502460C46FF25FF2309E0D6
:1091E00012F8010B80EA05010648405C80EA03059D
:1091F0000548435C201EA4F10106B4B2F0D143EA55
:10920000052070BD705101087052010810B502218F
:1092100001A004F02CFA10BD4154000010B50A2141
:1092200001A004F024FA10BD41542B53544154457D
:109230003D3F000070B504460E462546288845F699
:10924000A521884202D1284609F0A0F970BD00008E
:1092500030B589B00446202101A8FEF7AEFF2021D9
:1092600001A8FEF7AAFF224606A101A805F072FE9A
:1092700001A8FEF7BFFF0546294601A804F0F7F94B
:1092800009B030BD41542B4E414D453D2573000082
:1092900010B5092101A004F0EAF910BD41542B4E8C
:1092A000414D453D3F00000010B50D2101A004F0E7
:1092B000DEF910BD41542B554152545F4346473DA2
:1092C0003F00000010B50B2101A004F0D0F910BD43
:1092D00041542B564552494F4E3D3F0010B525484D
:1092E0000078012845D124480078062837D2DFE8E5
:1092F00000F003170D36202A072220A12148FEF78F
:1093000080FF10B902201C49087028E00A221EA123
:109310001C48FEF776FF10B90120174908701EE0BF
:109320001C491848FEF754FF10B104201249087078
:1093300015E00B2218A11348FEF763FF10B90520B2
:109340000D4908700BE00F480B494860154800882C
:109350000881144801880B48FFF76CFF00BF00BF6D
:109360000020044908700F49088080210548FEF755
:1093700024FF10BD12020020041F002041542B4F77
:109380004B0D0A00281A002041542B4F4B0D0A3078
:1093900033303300A814002041542B4F4B0D0A30BA
:1093A000310D0A001002002010B516480078072879
:1093B00024D2DFE800F0040A07230D1F220000F08A
:1093C00077FA1CE000F078FA19E000F031FA16E0C4
:1093D00000F05CFA0C4890F8760018B900200949B2
:1093E000887006E0084890F87600012801D1054908
:1093F000887004E000F00AF801E000E000BF00BF60
:1094000010BD0000041F00209814002010B559481A
:1094100090F8A800012808D15748007C0A2803DBEF
:109420000020544981F8A80010BD4FF47A705349C8
:1094300008805148007C14280EDD4E4890F87600D4
:1094400018B900204C49887006E04A4890F8760028
:10945000012801D1484988704748807807287AD286
:10946000DFE800F004070E666782830000F0B0F9C1
:109470007DE000F06DF900203E4981F8A80076E01B
:109480003E4801883E4804F057FD01284FD13D4831
:109490000088401C3B49088008460088092801DDF7
:1094A000002008800021364804F046FD3548008839
:1094B00010B900F021F93AE032480088012802D1C1
:1094C000FFF7E0FC33E02F480088022802D1FFF7C5
:1094D00057FD2CE02B480088032828D02948008815
:1094E000042802D100F050F821E026480088052821
:1094F00002D1FFF7F7FD1AE022480088062802D1C2
:10950000FFF714FD13E01F480088072802D106F07A
:10951000DDFA0CE01B480088082802D106F070FA3A
:1095200005E018480088092801D106F097FA1EE0E6
:109530001DE01148417C407C401C0F4A50741429A6
:1095400011DD0020114608700A4890F8760018B91D
:109550000020887007E009E0064890F876000128AE
:1095600001D10549887002E001E000E000BF00BFC2
:1095700000BF59E798140020041F00208005002038
:109580007C0500207805002010B5A2B000200190D5
:10959000002441F207004B49A1F805004A48808B9E
:1095A0004949C98B484342F2107190FBF1F084B2F3
:1095B0004548007F4349C8714348808B01124148A8
:1095C00001724148817F3F4841723F48C08B011280
:1095D0003C488172C4723C4890F8291039480173A4
:1095E000394890F8281037484173202181735F2152
:1095F000C1733548C17E33480174334890F8261052
:10960000304841743048C08C01122E4881742E4875
:10961000C17E2C48C1742C48417A2A4801752A48D9
:10962000B0F809000112274841752748C17A25483A
:1096300081752548B0F80B0001122248C1752248F7
:109640004178204801762048B0F8010001121D48F9
:1096500041761D4841791B4881761B48B0F80500CA
:1096600001121848C1761848C17916480177164882
:10967000817C144841771448408A010A1148817757
:10968000114890F82A100F48C1770F4890F82B1016
:109690000C4880F820100DA005F04CFC1A20094958
:1096A000488001AA02A9074801F090FD0C48007CFF
:1096B000401C0B49087400210A4804F03DFC22B00C
:1096C00010BD00007E1D0020780B002073656E64C5
:1096D000204443444320646174610A0D000000008B
:1096E000041F0020B405002070B504460D4629462D
:1096F000204603F0AFFF70BD00B5A1B00020009080
:109700000AA005F017FC3A200E4948806A4601A9D4
:109710000C4801F05BFD0C48007C401C0A490874B1
:1097200000210A4804F008FC21B000BD73656E6496
:10973000206865617274626561742064617461207F
:109740000A0D00007E1D0020041F00208C05002053
:1097500000B591B00020009040F6B831134804F0F5
:10976000EBFB01281FD141F201001149A1F80500CE
:1097700010A005F0DFFB0E48C01D1349CA6E026041
:10978000096F416011490A6882604968C160102010
:10979000074948806A4601A9054801F017FD0021E4
:1097A000024804F0C9FB11B000BD0000880500208C
:1097B0007E1D002073656E64204C6F67696E2064A7
:1097C0006174610D0A0000009814002080500108A7
:1097D00000B591B00020009041F288310C4804F0AF
:1097E000ABFB012811D100030A49A1F805000020B4
:1097F000488009A005F09EFB6A4601A9054801F0D2
:10980000E5FC0021024804F097FB11B000BD000008
:10981000840500207E1D002053656E64205265671C
:109820006973746572656420646174610A0D000077
:1098300010B54FF47A71124804F07EFB01281ED156
:109840001048007818B901200E49087013E00D483F
:109850000078012806D10C48FFF7FAFC02200949DC
:10986000087008E007480078022804D1FFF710FDCF
:109870000020044908700021014804F05DFB10BD80
:10988000700500206C050020A814002010B540F6DB
:10989000B831064804F050FB012805D1FFF7BEFCA3
:1098A0000021024804F048FB10BD000074050020B0
:1098B00010B5FFF7ABFC10BD10B54FF47A710E4830
:1098C00004F03AFB012815D10C48007828B9FFF7BD
:1098D000F9FC01200949087008E0084800780128CF
:1098E00004D1FFF7E1FC0020044908700021024880
:1098F00004F022FB10BD0000680500206705002071
:1099000000BFFEE700B585B06A460021044800F0BC
:1099100072FE6946002006F07FFF05B000BD000022
:109920000064004010B54FF40071154800F01EFCB3
:1099300001280DD11349124800F0DCFB012802D1A7
:10994000002007F047F84FF400710D4800F0A6F929
:109950004FF480610A4800F009FC01280ED1094942
:10996000891C074800F0C6FB012802D1002007F03F
:1099700057F84FF48061024800F090F910BD0000E4
:10998000006400400200F01010B50021194800F0FA
:109990006BFF0446022C08D0012C00D100E000200F
:1099A00002460021084606F073FF0121114800F02D
:1099B0005BFF0446022C08D0012C00D100E00020FF
:1099C00002460121002006F063FF0221094800F051
:1099D0004BFF0446022C08D0012C00D100E00020EF
:1099E00002460221002006F053FF0121014800F049
:1099F00055F910BD0064004000B585B003F049FF83
:109A00000121092003F0E2FC0121480603F0BEFC1D
:109A10000121880603F0BAFC00214A4800F09AFDB3
:109A20004FF40050ADF8100003208DF812001820FC
:109A30008DF8130004A9444801F0AAFE4FF48050A9
:109A4000ADF8100048208DF8130004A93E4801F03D
:109A50009FFE00208DF80A0001208DF80B000020E9
:109A60008DF80C008DF80D008DF80E0001208DF89A
:109A70000F0000208DF8060001208DF80700082057
:109A80008DF8080001208DF809000620ADF80400CB
:109A900001A92C4800F003FC2C49002000F015FB24
:109AA00001221021274800F0F1FB41208DF8000031
:109AB00001208DF8010000208DF8020001208DF8B2
:109AC0000300684602F00CFF012211461D4800F019
:109AD000DDFB012251021B4800F0D8FB012291025C
:109AE000184800F0D3FB0122D103164800F0CEFB4A
:109AF0000121144800F02EFD3F208DF800000120C8
:109B00008DF8010000208DF8020001208DF803007F
:109B1000684602F0E5FE42208DF8000001208DF835
:109B2000010000208DF8020001208DF80300684636
:109B300002F0D6FE03F0AFFE05A005F0FBF9002011
:109B400005B000BD00680040000C01400806002080
:109B500063616E2032206F70656E210A0000000084
:109B600000B585B06A460121054800F044FD9DF826
:109B7000090018B96946012006F04EFE05B000BD87
:109B80000068004010B54FF40071184800F0EEFA7C
:109B9000012810D11649154800F0ACFA012805D16A
:109BA00006F018FF1249114800F05CF84FF40071FC
:109BB0000E4800F073F84FF480610C4800F0D6FABC
:109BC000012812D10A49891C084800F093FA01289B
:109BD00006D106F025FF0649891C044800F042F82A
:109BE0004FF48061014800F059F810BD0068004052
:109BF0000200F01010B50021194800F035FE0446AF
:109C0000022C08D0012C00D100E0002002460021E7
:109C1000012006F03DFE0121114800F025FE04461A
:109C2000022C08D0012C00D100E0002002460121C6
:109C3000084606F02DFE0221094800F015FE0446F4
:109C4000022C08D0012C00D100E0002002460221A5
:109C5000012006F01DFE0121014800F01FF810BD93
:109C60000068004000220C4B994202D1002383611E
:109C700011E0C1F3130201F000730BB1C2600AE0FE
:109C800001F080630BB1026105E001F000630BB1EC
:109C9000826000E0426070477000F030B1F5007FF4
:109CA0003AD00FDC202928D006DC01291CD0042959
:109CB0001DD0082940D11DE0402921D0B1F5807F79
:109CC0003AD126E0B1F5004F31D006DCB1F5806F16
:109CD00025D0B1F5006F2FD124E0B1F5803F12D02F
:109CE000B1F5003F28D111E0154A826025E0082235
:109CF000C26022E01022C2601FE0082202611CE064
:109D00001022026119E00822426016E0102242602F
:109D100013E00422426010E0042242600DE00422BD
:109D200042600AE0002282610422426005E00022D3
:109D300082610422426000E000BF00BF7047000063
:109D40000101010010B504460B48844209D10121EC
:109D5000480603F02BFB00214FF0007003F026FBB8
:109D600008E00121880603F021FB00214FF080600C
:109D700003F01CFB10BD0000006400402DE9F04121
:109D800004460D4617461E46ECB1002020722060A6
:109D90006060B5F5006F03D304202072656002E0B7
:109DA00000202072256006B127B90020A072022091
:109DB000607208E000206072A6723246394604F1F3
:109DC0000B00FEF7E1F9BDE8F0812DE9F041044612
:109DD0000D4617461E46ECB10020207220606060E0
:109DE000B5F5006F03D304202072656002E0002007
:109DF0002072256006B127B90020A072022060728F
:109E000008E000206072A6723246394604F10B0069
:109E1000FEF7BAF9BDE8F08110B50021837A01227E
:109E200002FA03F13D4A126842F001023B4B1A600C
:109E30003A4A1C3212688A43384B1C331A60027B40
:109E4000CAB9364A0C3212688A43344B0C331A6052
:109E50004288C38842EA0343304A4032847A42F857
:109E600034300288838842EA03432C4A4032847AA1
:109E700002EBC4025360027B012A19D1274A0C323B
:109E800012680A43254B0C331A604288038842EA61
:109E90000343224A4032847A42F83430C2888388AD
:109EA00042EA03431D4A4032847A02EBC402536003
:109EB000C27A3AB9194A121D12688A43174B1B1D00
:109EC0001A6006E0154A121D12680A43134B1B1D47
:109ED0001A60028932B9114A143212688A430F4B50
:109EE00014331A600289012A06D10C4A143212680E
:109EF0000A430A4B14331A60427B012A06D1074AEF
:109F00001C3212680A43054B1C331A60034A12685C
:109F100022F00102014B1A6010BD000000660040F3
:109F20002DE9FF4706460F46B94600244FF00108C9
:109F3000404600F0D9FB8DF80A8001208DF80B0017
:109F40008DF80C00ADF808008DF80D0000253EE0FE
:109F5000204604EBD0714910A4EB4101491C0129B2
:109F600002D0022920D10FE056F83500042101EB80
:109F7000C000000CADF8000036F8350001EBC00061
:109F800080B2ADF802000FE056F83500042101EB75
:109F9000C000000CADF8040036F8350001EBC0003D
:109FA00080B2ADF8060000BF00BF641C204604EB81
:109FB000D0714910A4EB410141B96846FFF72CFF6D
:109FC0009DF80A00401CC0B28DF80A006D1C4D457A
:109FD000BEDB204604EBD0714910A4EB410111B166
:109FE0006846FFF719FFBDE8FF872DE9FF470646E2
:109FF0000F46B94600244FF00108404600F074FBBC
:10A000008DF80A8001208DF80B0000208DF80C00DF
:10A010000120ADF808008DF80D00002547E020462E
:10A02000E11704EB91718910A4EB8101491C01290E
:10A0300006D002290DD0032914D0042924D11AE016
:10A0400056F835004FF6FF7101EA4010ADF80000F8
:10A050001AE056F835004FF6FF7101EA4010ADF8EE
:10A06000020011E056F835004FF6FF7101EA40108A
:10A07000ADF8040008E056F835004FF6FF7101EA2C
:10A080004010ADF8060000BF00BF641CE11704EBF0
:10A0900091718910A4EB810141B96846FFF7BCFEBC
:10A0A0009DF80A00401CC0B28DF80A006D1C4D4599
:10A0B000B5DBE11704EB91718910A4EB810111B1BB
:10A0C0006846FFF7A9FEBDE8FF8770B504460D4658
:10A0D0000C2624B931462846FFF787FF08E0012CFB
:10A0E00004D131462846FFF71BFF01E0002070BD78
:10A0F0000120FCE710B50246002001F4700343B1D3
:10A100009369C1F3130423400BB101202DE000201B
:10A110002BE001F0807343B15368C1F31304234073
:10A120000BB1012021E000201FE001F0006343B1EA
:10A130009368C1F3130423400BB1012015E0002004
:10A1400013E001F0007343B1D368C1F3130423405B
:10A150000BB1012009E0002007E01369C1F31304EB
:10A1600023400BB1012000E0002010BD70B5044673
:10A170000D46002660692840002871D0B5F5807F23
:10A180005CD010DC082D35D006DC012D20D0022D4E
:10A1900024D0042D72D127E0102D31D0202D35D0C0
:10A1A000402D6BD138E0B5F5004F60D009DCB5F536
:10A1B000007F49D0B5F5806F4CD0B5F5006F5DD10B
:10A1C0004FE0B5F5803F2DD0B5F5003F56D12FE0DB
:10A1D000A0682D4900F03EFF064651E0E0680321EB
:10A1E00000F038FF06464BE0E068082100F032FF3F
:10A1F000064645E0E068102100F02CFF06463FE0EF
:10A200002069032100F026FF064639E02069082175
:10A2100000F020FF064633E02069102100F01AFF0D
:10A2200006462DE06068082100F014FF064627E08E
:10A230006068102100F00EFF064621E0A0690121B0
:10A2400000F008FF06461BE0A069022100F002FFB3
:10A25000064615E0A069042100F0FCFE06460FE06A
:10A260000FE0A069702100F0F5FE064608E0606886
:10A27000042100F0EFFE064602E0FFE7002600BFE3
:10A2800000E00026304670BD010101001AB14369AB
:10A290000B43436102E043698B434361704730B530
:10A2A000024600200023146824F00204146014689D
:10A2B00044F00104146000E05B1C546804F00104E5
:10A2C0001CB94FF6FF74A342F6D1546804F00104A0
:10A2D0000CB900206CE08C79012C04D1146844F096
:10A2E0008004146003E0146824F080041460CC79C6
:10A2F000012C04D1146844F04004146003E0146895
:10A3000024F0400414600C7A012C04D1146844F049
:10A310002004146003E0146824F0200414604C7AD4
:10A32000012C04D1146844F01004146003E0146894
:10A3300024F0100414608C7A012C04D1146844F0C9
:10A340000804146003E0146824F008041460CC7A54
:10A35000012C04D1146844F00404146003E0146870
:10A3600024F0040414608C78A407CD7844EA0564D2
:10A370000D7944EA05444D7944EA05540D886D1E73
:10A380002C43D461146824F001041460002300E01D
:10A390005B1C546804F001041CB14FF6FF74A34227
:10A3A000F6D1546804F001040CB1002000E0012053
:10A3B00030BD2DE9F04107460C461546264616B13C
:10A3C00000212846B047BDE8F08170B506460C462E
:10A3D0001546E9B2E0B207F01DFB70BD00B589B0CB
:10A3E0000121052002F0F2FF0121480602F0CEFF14
:10A3F0000021524800F0AEF84FF48050ADF8200034
:10A4000003208DF8220018208DF8230008A94C485D
:10A4100001F0BEF94FF40060ADF8200048208DF83F
:10A42000230008A9464801F0B3F900208DF81A006E
:10A4300001208DF81B0000208DF81C008DF81D00F8
:10A440008DF81E008DF81F008DF816008DF817008E
:10A450000C208DF8180001208DF819000920ADF8A6
:10A46000140005A93548FFF71AFF00208DF80E00EB
:10A470008DF80F0001208DF810000020ADF80400C9
:10A48000ADF80600ADF80800ADF80A00ADF80C0014
:10A4900001208DF8110001A8FFF7BEFC0122022166
:10A4A0002648FFF7F3FE14208DF8000001208DF8F8
:10A4B000010000208DF8020001208DF8030068469D
:10A4C00002F00EFA012211461C48FFF7DFFE0122BE
:10A4D00051021A48FFF7DAFE012291021748FFF7EE
:10A4E000D5FE0122D1031548FFF7D0FE0121134804
:10A4F00000F030F813208DF8000001208DF80100E5
:10A5000000208DF8020001208DF80300684602F05B
:10A51000E7F916208DF8000001208DF801000020D9
:10A520008DF8020001208DF80300684602F0D8F98A
:10A5300004A004F0FFFC002009B000BD006400404E
:10A540000008014063616E2031206F70656E210A42
:10A550000000000010B502460B4600204FF6FF71C8
:10A56000BBB9146824F0020444F00104146000E054
:10A57000491E546804F00304012C01D00029F7D1CE
:10A58000546804F00304012C01D0002032E00120C3
:10A5900030E0012B13D1146824F00304146000E0B0
:10A5A000491E546804F003040CB10029F8D1546822
:10A5B00004F003040CB100201CE001201AE0022B7F
:10A5C00017D1146824F0010444F00204146000E080
:10A5D000491E546804F00304022C01D00029F7D16D
:10A5E000546804F00304022C01D0002002E0012092
:10A5F00000E0002010BD10B500F5D87303EB011387
:10A600001B6803F004031372137A53B900F5D8736F
:10A6100003EB01131B6840F2FF7404EA5353136009
:10A6200009E000F5D87303EB01131B686FF0604479
:10A6300004EAD303536000F5D87303EB01131B68DE
:10A6400003F00203537200F5D87303EB01135B6848
:10A6500003F00F03937200F5D87303EB01135B68EB
:10A660001B0AD37400F5D87303EB01139B68D372F4
:10A6700000F5D87303EB01139B681C0A147300F5F3
:10A68000D87303EB01139B681C0C547300F5D8734B
:10A6900003EB01139B681B0E937300F5D87303EB58
:10A6A0000113DB68D37300F5D87303EB0113DB6888
:10A6B0001C0A147400F5D87303EB0113DB681C0C3F
:10A6C000547400F5D87303EB0113DB681B0E93740D
:10A6D00021B9C36843F02003C36003E0036943F07A
:10A6E0002003036110BD00000B49096841F001011E
:10A6F000094A11601146096843F60E729143064AF1
:10A7000011601146096841EA00211160114609688B
:10A7100021F00101116070470066004010B502464B
:10A720000020504B9A420CD10B68B3F5457F00D105
:10A7300020E00B68B3F57A7F01D101201AE00220F6
:10A7400018E0936803F08063B3F1806F01D10020BB
:10A7500010E0936803F00063B3F1006F01D10120B2
:10A7600008E0936803F08053B3F1805F01D10220C9
:10A7700000E00420042874D002F5C07303EB00133A
:10A780001B6803F0010402F5C07303EB00131C60A7
:10A790000B7A7BB94B7A0C8843EA445302F5C074B8
:10A7A00004EB00142468234302F5C07404EB001486
:10A7B000236010E00B7A4C6843EAC4034C7A2343CD
:10A7C00002F5C07404EB00142468234302F5C0743E
:10A7D00004EB001423608B7A03F00F038B7202F5F5
:10A7E000C07303EB00135B6823F00F0402F5C07322
:10A7F00003EB00135C6002F5C07303EB00135B68AE
:10A800008C7A234302F5C07404EB001463608B7BE5
:10A810001C064B7B44EA03440B7B44EA0323CC7ABB
:10A82000234302F5C07404EB0014A3608B7C1C0668
:10A830004B7C44EA03440B7C44EA0323CC7B234354
:10A8400002F5C07404EB0014E36002F5C07303EB7F
:10A8500000131B6843F0010402F5C07303EB0013FF
:10A860001C6010BD0068004010B50246002321B1F5
:10A87000012907D002290FD109E090681D4C00EA98
:10A8800004030BE090681C4C00EA040306E09068A7
:10A890001A4C00EA040301E0002300BF00BF184C7B
:10A8A000181BA34216D007DC83B16FF080601844F8
:10A8B00070B1022818D111E0B0F5007F10D0114C12
:10A8C000204448B1B0F5003F0ED10BE002230DE06B
:10A8D00000230BE0002309E0002307E0012305E04B
:10A8E000012303E0012301E0002300BF00BFD8B231
:10A8F00010BD000003000004000300080000031066
:10A90000000100080001FFF770B51D4885888488A4
:10A910001C480068E8B11C4800683C21B0FBF1F01D
:10A920001949086008460068C000184908600846D0
:10A930000068FDF7CCFE06461549FDF7F9FC154900
:10A94000086000200F4908600F4908600F4908603F
:10A9500014E0114800683C280AD20B4800682044E3
:10A96000094908600C480068401C0B49086005E074
:10A9700000200949086001200249086070BD0000FC
:10A98000600000209800002090000020940000202B
:10A9900000401C46380B00209C00002030B50346C8
:10A9A0000C46002118785D7800EB0520184DA5F8BD
:10A9B0001B009878DD7800EB052001B2B1F57A6FC5
:10A9C00002DDA1F57A6001E0C1F57A6001B2104DB7
:10A9D000A5F81D100A2906DB2846B0F81D000D4D0C
:10A9E000A5F8070003E000200A4DA5F80700187934
:10A9F0005D7900EB0520064DA5F81F002846B0F84C
:10AA00001F00A5F81F00987985F82100012030BDAE
:10AA1000C00B00203A0C002010B503461C780748F4
:10AA200080F827405C7880F828409C7880F829409E
:10AA3000DC7880F82A40012010BD0000C00B002007
:10AA400070B505460C461646032C00DD032422464D
:10AA500029460248FDF798FB012070BDC00B00207D
:10AA600030B503460C46002118785D7840EA052091
:10AA7000144D68829878DD7840EA0520114DA8824F
:10AA800018795D7940EA052001B2B1F57A6F02DDEF
:10AA9000A1F57A6001E0C1F57A6001B2094DE98261
:10AAA0009879DD7940EA052001B2B1F57A6F02DDCF
:10AAB000A1F57A6001E0C1F57A6001B2014D298308
:10AAC000012030BDC00B002010B50346082900DD71
:10AAD000082118780A4CE070587820719C78084852
:10AAE0004471DC7884711C79C4715879044C2072EB
:10AAF0009C7903484472DC798472012010BD000007
:10AB0000C00B002010B503461878024CA076012037
:10AB100010BD0000C00B002010B503461879074C8B
:10AB200084F834005C79054880F835409C7980F8D9
:10AB30003640DC7980F83740012010BDC00B002082
:10AB400010B503461C78074880F823405C7880F8ED
:10AB500024409C7880F82540DC7880F8264001204D
:10AB600010BD0000C00B002030B503460C46154652
:10AB7000082C00DD08241878FEF772F91449C87211
:10AB80005878FEF76DF9124908739878FEF768F95E
:10AB90000F494873D878FEF763F90D49887318791F
:10ABA000FEF75EF90A49C8735879FEF759F9084962
:10ABB00008749879FEF754F90549487405480B3133
:10ABC0000A6802608A88828089798171012030BD9B
:10ABD000C00B0020B50B002010B5044605A004F002
:10ABE000A9F900F0B9F900F0ABF901F001FF01207B
:10ABF00010BD000054310D0A0000000010B50446DD
:10AC000002A004F097F9022010BD00005431300D6D
:10AC10000A00000010B5044602A004F08BF90620DB
:10AC200010BD00005431310D0A00000010B504467B
:10AC300002A004F07FF9062010BD00005431320D4F
:10AC40000A00000010B5044603A004F073F900F0F8
:10AC500083F9012010BD00005431330D0A000000BB
:10AC600010B5044602A004F065F9002010BD0000F4
:10AC70005431340D0A00000010B5044609A004F058
:10AC800059F901F0B1FE00BF01200849C870084819
:10AC900001F091FD00F048F900BF064801F08BFD7E
:10ACA000072010BD5431350D0A0000006806002051
:10ACB000F4090020080A002010B5044607A004F09B
:10ACC00039F900F03DF901F093FE002005490870C4
:10ACD000054908700549087010BD00005431360D53
:10ACE0000A000000AD000020AC000020080B00208E
:10ACF00010B5044603A004F01DF901F079FE02200E
:10AD000010BD000054320D0A0000000010B50446CA
:10AD100002A004F00FF9032010BD000054330D0A07
:10AD20000000000010B5044602A004F003F904205E
:10AD300010BD000054340D0A0000000010B5044698
:10AD400002A004F0F7F8052010BD000054350D0AEC
:10AD50000000000010B5044602A004F0EBF8062045
:10AD600010BD000054360D0A0000000010B5044666
:10AD700004A004F0DFF800F0EFF800F0D5F80020B0
:10AD800010BD000054370D0A0000000010B5044645
:10AD900002A004F0CFF8022010BD000054380D0AC4
:10ADA0000000000010B5044602A004F0C3F8022021
:10ADB00010BD000054390D0A0000000010B5252018
:10ADC00000F09AFA0021034803F0B6F8012000F0E1
:10ADD0004BF910BD9C23002010B52248406A00F0BA
:10ADE000004018B120A004F0A5F834E01D48406AE6
:10ADF00000F0804018B120A004F09CF82BE0194826
:10AE0000406A00F0005018B120A004F093F822E04E
:10AE10001448406A00F0805018B121A004F08AF86C
:10AE200019E01048406A00F0006018B11FA004F05B
:10AE300081F810E00B48406A00F0806018B11FA054
:10AE400004F078F807E00748406A00F0007010B19D
:10AE50001DA004F06FF80348406A40F0807001497B
:10AE6000486210BD00100240B5CDB9A6BAC4B8B44E
:10AE7000CEBB0D0A00000000B4B0BFDABFB4C3C53A
:10AE8000B9B7B8B4CEBB0D0A00000000B6C0C1A26D
:10AE9000BFB4C3C5B9B7B8B4CEBB0D0A000000003B
:10AEA000C8EDBCFEB8B4CEBB0D0A0000C9CFB5E7F3
:10AEB0002FB5F4B5E7B8B4CEBB0D0A00D2FDBDC5C1
:10AEC000B8B4CEBB0D0A0000424F52B8B4CEBB0D91
:10AED0000A00000010B50A4801F042FC012000F011
:10AEE000D6F9084801F067FC4FF4FA7000F0CFF98A
:10AEF000044801F035FC04A004F01CF810BD00006B
:10AF0000A80A0020BC0A0020434C4F53455F313251
:10AF100056506F7765725265616C790D0A000000BA
:10AF200010B5FFF7D7FF10BD10B50020024988709B
:10AF3000024801F015FC10BD68060020CC09002075
:10AF400010B500200249C870024801F009FC10BD8C
:10AF500068060020F409002010B50020024948705E
:10AF6000024801F028FC10BD68060020A40900205A
:10AF700010B519480078052803D01748007807282D
:10AF800001D1012010BD062000F0CCF948B91248CB
:10AF90000078052807D1114890F8380000F020000B
:10AFA00008B10220EEE7282000F0BCF978B926208D
:10AFB00000F0B8F958B91C2000F0B4F938B92120D4
:10AFC00000F0B0F918B904480078062801D1032030
:10AFD000D8E70020D6E7000088230020C00B00201F
:10AFE0000120704710B51848007920B1012807D01A
:10AFF00002280DD108E01121144800F057FB07E0AA
:10B00000124800F085FB03E0112000F091FB00BF27
:10B0100000BF32210E4802F08FFF012805D104F055
:10B02000C9FE00210A4802F087FFFA2108480830CB
:10B0300002F082FF012806D105F0DAF90021044868
:10B04000083002F079FF10BD4423002065FF00089E
:10B050006C2300200246002002EA01030BB101200C
:10B0600000E0002070470000012201490A547047A7
:10B07000A02300200120704710B5044908698047CB
:10B08000022801D1012010BD0020FCE76C00002047
:10B0900070B51349134800F0A1FA0446124911484B
:10B0A000083000F09BFA054602F0AEFA28B1012CF8
:10B0B00003D1012000F050F90FE002F0A5FA28B109
:10B0C000022C03D1022000F047F906E0032D04D141
:10B0D000052000F041F9002070BD0120FCE70000D0
:10B0E000440B0020B4230020DD0B002010B5002409
:10B0F0000E48007800B917E00C480078012805DBFD
:10B100000A480078042801DC01240DE00748007893
:10B11000052803D005480078072801D1022403E060
:10B1200000F0DAF800B10324204610BD8823002087
:10B1300010B541F288310F4802F0FEFE012807D118
:10B14000252000F009F9012002F0D6FC002010BDF6
:10B1500041F288310748001F02F0EEFE012807D1B6
:10B16000242000F0F9F8002002F0C6FC0020EEE7F1
:10B170000120ECE79C23002021B1026842F001028B
:10B18000026004E002684FF6FE731A4002607047E6
:10B1900010B50022026847F6F0739A430C6A8B6878
:10B1A00023430C6923434C6923438C692343CC69B3
:10B1B00023434C6A23438C6A23431A430260CB68BF
:10B1C00043600B6883604B68C36010BD2DE9F04796
:10B1D00006460C4692460025A946A84606B114B973
:10B1E0000020BDE8F087708819301FFA80F8A5228A
:10B1F0002846691CCDB222545A222846691CCDB279
:10B2000022542846691CCDB204F800804FEA182267
:10B210002846691CCDB2225420222846691CCDB292
:10B220002254601910221849FCF7AEFF05F11000F6
:10B23000C5B272792846691CCDB22254B6F8050011
:10B24000020A2846691CCDB222547088022807DB06
:10B2500072886019F11DFCF797FFB0782844C5B2D9
:10B2600029462046FDF7B6FF07462846691CCDB2A1
:10B2700027543A0A2846691CCDB222542946204652
:10B28000FEF732FA0120ACE798140020704710B5A1
:10B29000044606E0142003F003FE00F0E7FF601E02
:10B2A00084B2002CF6DC10BD10B510210648FCF766
:10B2B00084FF0648002101600171002004490860F4
:10B2C0000449086010BD0000C42300207C08002051
:10B2D0007408002078080020002106E00548405C42
:10B2E00008B101207047481CC1B21029F6DB0020CC
:10B2F000F8E70000C423002070B50546284600F09A
:10B300005DFB0446284600F04FFB06460448005DFE
:10B310000021B140084302490855012070BD0000DA
:10B32000C42300202DE9F0410446204600F046FBEE
:10B330000546204600F038FB06460648405D0121E0
:10B34000B14000EA010717B10120BDE8F0810020FB
:10B35000FBE70000C423002070B506463046FFF727
:10B36000E1FF10B9304604F077FA304600F026FBD2
:10B370000446304600F018FB05460448005D0121F4
:10B38000A940084301490855012070BDC42300208D
:10B3900070B5002418E00E48005D98B100250FE05C
:10B3A0000B48005D0121A940084038B105EBC400FD
:10B3B000C6B2314607A003F0BDFD00BF681CC5B290
:10B3C000082DEDDB601CC4B2102CE4DB012070BD45
:10B3D000C4230020457272436F6465206973202581
:10B3E000640D0A000149C860704700000020024057
:10B3F00030B5044604250F4800F0AAF80546042D90
:10B4000016D10D48006940F002000B49086108465A
:10B410004461006940F040000861064800F098F877
:10B4200005460548006941F6FD710840024908617A
:10B43000284630BDFFFF0F000020024004200B49CA
:10B44000C96801F0010109B101200EE00749C9688E
:10B4500001F0040109B1022007E00449C96801F0C4
:10B46000100109B1032000E00420704700200240D1
:10B470000348006940F080000149086170470000FE
:10B480000020024070B504460D4604264FF6FF70BA
:10B4900000F05EF80646042E12D10A48006940F01A
:10B4A00001000849086125804FF6FF7000F050F850
:10B4B00006460448006941F6FE71084001490861EA
:10B4C000304670BD0020024078B506460C46042583
:10B4D000002000904FF6FF7000F03AF80546042D6A
:10B4E00026D11448006940F00100124908613480F7
:10B4F0004FF6FF7000F02CF80546042D11D1B01C5A
:10B500000090200C009908804FF6FF7000F020F8A2
:10B5100005460848006941F6FE7108400549086182
:10B5200006E00448006941F6FE71084001490861DF
:10B53000284678BD0020024002480349486003487D
:10B54000486070472301674500200240AB89EFCD7A
:10B5500000B502460423FFF771FF034603E0FFF73F
:10B560006DFF0346521E012B01D1002AF7D102B90B
:10B570000523184600BD0000042900DD704702784D
:10B580000B4B03F83120427803EBC1035A708278E9
:10B59000074B03EBC1039A70C278054B03EBC10361
:10B5A000DA70034B03EBC10342685A6000BFE5E762
:10B5B000A423002000B501210548FFF7DDFF02218B
:10B5C0000448FFF7D9FF03210348FFF7D5FF00BD6B
:10B5D0005C080020640800206C08002070B5044658
:10B5E0000E463046616888470546E078A84203D099
:10B5F00000206070E5700EE0A078A84202D1002023
:10B60000607008E06078401C607060782178884243
:10B6100001DBE078A070A07870BD00002DE9F0415A
:10B62000074620480088401E86B2002500241E4898
:10B6300000EBC60041683846FDF7B6F807D31A4854
:10B6400000EBC50041683846FDF7B8F803D240F674
:10B65000FF70BDE8F0811EE0A81900EBD071C1F3C6
:10B660004F04114800EBC40041683846FDF7A6F8C6
:10B6700002D2601E86B20EE00B4800EBC4004168A7
:10B680003846FDF791F802D2601C85B203E0064807
:10B6900030F93400DDE7B542DEDD034830F935002E
:10B6A000D7E700006A000020044B010870B504468B
:10B6B0000D466421124802F03FFC012808D1A04742
:10B6C00000201049C872486000210D4802F034FC87
:10B6D0000C48C07A112811D10A48407CA8420DD1EB
:10B6E000084840686FF30F000749884206D10020E0
:10B6F0000449C872486001200449087170BD000007
:10B700005C230020500C00200000EC1C442300208F
:10B7100010B504460220A047022003490871002109
:10B72000024802F009FC10BD4423002060230020E1
:10B7300010B504461148C07A132812D10F48407C36
:10B74000A0420ED10D4840686FF30F000C498842AB
:10B7500007D100200949C87248600A4908710A499E
:10B7600088633221094802F0E7FB012804D1002058
:10B77000044908710449886310BD0000500C002082
:10B780000000EC1C44230020C00B0020602300209C
:10B790002DE9F04102460025002600200023002468
:10B7A000002791F803C00CF00F0591F803C00CF0CE
:10B7B000100CBCF1000F03D091F802C04CEA050553
:10B7C00091F800C0BCF1000F31D0146800202BE0CC
:10B7D0004FF0010C0CFA00F3B1F800C00CEA0306BC
:10B7E0009E4220D183004FF00F0C0CFA03F7BC43AC
:10B7F00005FA03FC4CEA040491F803C0BCF1280FDD
:10B8000006D14FF0010C0CFA00FCC2F814C00AE09B
:10B8100091F803C0BCF1480F05D14FF0010C0CFAB0
:10B8200000FCC2F810C0401C0828D1D31460B1F845
:10B8300000C0BCF1FF0F34DD546800202EE000F1A1
:10B84000080C4FF0010808FA0CF3B1F800C00CEA3C
:10B8500003069E4221D183004FF00F0C0CFA03F730
:10B86000BC4305FA03FC4CEA040491F803C0BCF1A4
:10B87000280F05D100F1080C08FA0CF8C2F8148062
:10B8800091F803C0BCF1480F07D100F1080C4FF04C
:10B89000010808FA0CF8C2F81080401C0828CED322
:10B8A0005460BDE8F0810000F0B50A460023002492
:10B8B0000021002500F00046B6F1004F02D11D4ED8
:10B8C000F16901E01B4E7168C0F3034583B200F4D7
:10B8D0004016B6F5401F08D121F07061154E76680C
:10B8E00026F07066134F7E6012E000F48016B6F505
:10B8F000801F06D1032606FA05F4A14341F07061CA
:10B9000006E0460D360103FA06F6B14341F07061D8
:10B9100022B1460D360103FA06F6314300F0004627
:10B92000B6F1004F02D1034EF16101E0014E7160AA
:10B93000F0BD0000000001400246002093680B406B
:10B940000BB1012000E000207047416170470161A8
:10B9500070470146087870472DE9F0470D48448844
:10B960000D4A0121204603F001FA0B480068FCF75C
:10B97000D4FE07463A460B4608480949FCF72FFE15
:10B980000546FCF7F5FE8146FFF748FE054948727B
:10B99000BDE8F08760000020B80000209A999999CE
:10B9A00099991340380B002001460A46C81701EB4D
:10B9B0005070C010A1EBC000C0B2704701460A46EB
:10B9C000C81701EB5070C0F3C70070470246002152
:10B9D00012E001EB410000EBC1000E4B03EB001045
:10B9E0000078904206D101EB410000EBC10003EB6F
:10B9F00000107047481CC1B2022909D201EB410076
:10BA000000EBC100034B03EB00100078FF28E0D1EE
:10BA10000020EEE7B41200202DE9F0478246BAF18B
:10BA2000010F34D1EB21822006F012FA644908801C
:10BA300008460088B0F5004F0CDB08460088B0F5DA
:10BA4000803F07DA084600884FF6FF71081A5C4904
:10BA5000088008E05A4800884FF6FF71884202DBF0
:10BA600000205749088056480088FCF735FE80467C
:10BA7000544A554BFCF741FD06460022534BFCF758
:10BA8000AEFD0446FCF774FE5149086094E0BAF13B
:10BA9000020F59D1E321B22006F0DAF948490880B3
:10BAA00008460088B0F5004F0ADB012049490880AC
:10BAB000434800884FF6FF71081A4149088002E0A8
:10BAC0000020444908803E480088FCF705FE804677
:10BAD0003C4A3D4BFCF711FD064600223B4BFCF770
:10BAE0007EFD0446FCF744FE3949086008460068BC
:10BAF000FCF713FE06464FF03332374BFCF7FDFCE4
:10BB00000446364A364BFCF76AFD8046FCF730FEA9
:10BB10002F4908602F48008801284DD14FF4FA6161
:10BB2000304802F009FA012806D12FA003F002FAEA
:10BB300000212C4802F000FA254801680020FCF79B
:10BB4000BFFB2349086037E0BAF1030F34D1E3218A
:10BB5000B42006F07DF91A49088008460088B0F53F
:10BB6000004F0CDB08460088B0F5803F07DA084636
:10BB700000884FF6FF71081A1149088008E0104844
:10BB800000884FF6FF71884202DB00200C490880D4
:10BB90000B480088FCF7A0FD06460A4A1B4BFCF741
:10BBA000ACFC04460022094BFCF719FD8046FCF76B
:10BBB000DFFD0749086000BF05480068BDE8F08761
:10BBC000CA000020FCA9F1D24D622040E0FFEF4006
:10BBD000CC000020D0000020F308CA40F6285C8F7B
:10BBE000C2F51340E40000204E6567617469766514
:10BBF00020766F6C746167652073616D706C652071
:10BC00006661756C74210D0A000000004D621040E1
:10BC10000146087908B1012070470020FCE7014681
:10BC2000087870470146C878032801D10120704781
:10BC3000C878042801D10020F9E70020F7E7014681
:10BC40008878012800D17047887808B90020FAE781
:10BC50000020F8E70148407A70470000380B0020C8
:10BC600010B503494868FCF744FD80B210BD0000E0
:10BC7000380B0020F8B504460020009057480078A3
:10BC800030B101282ED0022848D0032875D16CE0AD
:10BC900053492046FCF788FD01D2012700E0002728
:10BCA0002046FCF73AFD05464E4A4F4BFCF748FD4F
:10BCB00001D2012000E00020074017B101200090D0
:10BCC0000FE04FF081412046FCF778FD07D247494D
:10BCD0002046FCF769FD02D20220009001E000201E
:10BCE000009071E03E492046FCF75EFD01D201273D
:10BCF00000E000272046FCF710FD0546394A3A4B84
:10BD0000FCF71EFD01D2012000E00020074017B122
:10BD10000120009001E00020009055E04FF07F519D
:10BD20002046FCF741FD01D2012500E00025304905
:10BD30002046FCF743FD01D2012000E00020054031
:10BD400015B1032000900FE04FF081412046FCF731
:10BD500035FD07D227492046FCF726FD02D20220F6
:10BD6000009001E0002000902EE04FF07F5120462F
:10BD7000FCF71AFD02D2012701E022E0002720464D
:10BD8000FCF7CBFC0546174A174BFCF7D9FC01D250
:10BD9000012000E00020074017B1032000900FE0D1
:10BDA0004FF081412046FCF709FD07D21249204699
:10BDB000FCF7FAFC02D20220009001E00020009083
:10BDC00002E00020009000BF00BF69460B48FFF76B
:10BDD00005FC0249087008460078F8BD080B0020F1
:10BDE000333373407B14AE47E17A843F0000C04098
:10BDF0000AD7233C0000B0400000E040AC23002004
:10BE00002DE9FC471A48046801681A48FCF758FAFB
:10BE10000646174908681849FCF758FA074631469C
:10BE2000FCF786FA05461549FCF7F8F90446204662
:10BE3000FCF773FC07460022114BFCF75BFB054641
:10BE40000E462046FCF769FC074600220C4BFCF727
:10BE500054FB81462A463346FCF7C1FBCDE900017D
:10BE6000FCF786FC0446074804602046BDE8FC87D2
:10BE7000380B00200000A0403333A3408FC2F53DB3
:10BE8000000024406C0000200148007A7047000048
:10BE9000380B002001464878012800D170474878C7
:10BEA00008B90020FAE70020F8E700000148007810
:10BEB00070470000AD000020014601F00F01092984
:10BEC00003DD01F13700C0B2704701F13000C0B2AC
:10BED000FAE701460911092903DD01F13700C0B273
:10BEE000704701F13000C0B2FAE700BFFEE770B55D
:10BEF0000446002500BF00259120005D06281ED2C3
:10BF0000DFE800F0031E4C4D5C7094F854000328E9
:10BF100015DB04F1700008F0EFFB80B904F1940127
:10BF200004F1700008F008FC40B101219120015596
:10BF3000002084F890000021AC200155012567E025
:10BF400094F8993094221159207804F19A02A66845
:10BF5000B04784F8980094F89000401C84F8900052
:10BF600094F89800FF280ED002219120015500215D
:10BF7000AC200155012594F8540081280DD10320EF
:10BF800084F8540009E094F8901094F84400814239
:10BF900003DB042191200155012539E038E094F8B4
:10BFA000901094F84400814203DB04219120015554
:10BFB00002E0012191200155012529E00021912075
:10BFC0000155D4F8A80020B10121D4E929029047F5
:10BFD00006E0206D20B10121226DD4F8A400904725
:10BFE000012515E0002191200155D4F8A80028B1C1
:10BFF0000220D4E9292104F053FE07E0206D28B186
:10C000000220D4F8A420216D04F04AFE012500BFCF
:10C0100000BF012D04D19120005D04287FF46BAF97
:10C0200025B122780421012004F03AFE70BD10B53C
:10C0300004469120005D022811D194F8901094F8E4
:10C040004400814203DB04219120015502E00321D9
:10C050009120015522780421012004F021FE10BD19
:10C0600070B504460D469120005D022803D0912052
:10C07000005D03280DD194F89800A84209D105214C
:10C080009120015594F85400032802DB2046FFF765
:10C090002EFF70BD70B50024002515E001201B495E
:10C0A00008600520FCF7FEFD6006040E1848D0F875
:10C0B0001C0108B144F00104002014490860052067
:10C0C000FCF7F0FD681CC5B2082DE7DB00200F4926
:10C0D00008600520FCF7E6FD00200D49C1F89C0131
:10C0E0000520FCF7DFFD0120084908600520FCF76A
:10C0F000D9FD00200649C1F898010520FCF7D2FDC2
:10C1000001200249091D0860204670BD9881214226
:10C110000080214210B501200C4908600520FCF781
:10C12000C1FD01200A49C1F898010520FCF7BAFDBC
:10C130000020064908600520FCF7B4FD00200449F2
:10C14000C1F898010520FCF7ADFD10BD9C8121428E
:10C150000080214210B50020094908600520FCF745
:10C16000A1FD01200749C1F898010520FCF79AFDBF
:10C170000120034908600520FCF794FD10BD000074
:10C180009C8121420080214270B50446002018495C
:10C19000086000251CE004F0800020B10120144953
:10C1A000091D086003E000201149091D08600120F5
:10C1B0000F4908600520FCF775FD00200D49C1F806
:10C1C00098010520FCF76EFD6006040E681CC5B2E0
:10C1D000082DE0DB01200649091D08600549C1F86A
:10C1E00098010520FCF75EFD00200149086070BD44
:10C1F000988121420080214201460A88002000BF28
:10C20000034BB3F83530934200DA03207047000047
:10C21000A00700202DE9F04704462568002600BF4E
:10C220001048B0F839008046FCF751FA0746294615
:10C23000FCF7BAFA01D2012611E000BF0948C08F0D
:10C24000A0F164094846FCF739FA80462946FCF714
:10C2500037F807460449FCF7B1FA00D80226304601
:10C26000BDE8F087A00700200000C8427F200349F6
:10C27000086000200249087070470000002C004050
:10C28000E90100200EB542F20F70ADF8000026481B
:10C29000019069462548FCF799FD40F6C310ADF8BA
:10C2A00000002148019069462048FCF78FFD41F6C7
:10C2B0004B50ADF800001E48019069461B48FCF742
:10C2C00085FD42F22730ADF800001748019069461D
:10C2D0001648FCF77BFD40F2E730ADF8000015484A
:10C2E000019069461148FCF771FD41F64B50ADF8DD
:10C2F00000000D48019069460C48FCF767FD40F6C8
:10C30000C310ADF800000A48019069460748FCF7E1
:10C310005DFD42F20F70ADF80000034801906946E0
:10C320000248FCF753FD0EBDC1CD000814340020B7
:10C3300065CF000825D0000810B5002414E004EBF8
:10C34000440101EBC4010F4A02EB0110B021FBF7DD
:10C3500034FFFF2004EB440101EBC401094A02EB66
:10C3600001110870601CC4B2022CE8D301F01AFC61
:10C370000549012004F0AEFC0449022004F0AAFCA7
:10C3800010BD0000B4120020CBA30008B3A3000826
:10C3900010B548210E48FBF710FF28210D48FBF788
:10C3A0000CFF0D4801F024FA044624B11422214662
:10C3B0000848FBF7E9FE0848203001F019FA044666
:10C3C0002CB11422214603481430FBF7DDFE10BDCA
:10C3D000E40E0020BC0E00203450010810B51A48AD
:10C3E00000F050F9194800F04DF9194800F04AF9E9
:10C3F000184800F047F9184800F044F9174800F0D1
:10C4000041F9174800F03EF9164800F03BF916488C
:10C4100000F038F9154800F035F9154800F032F908
:10C42000144800F02FF9144800F02CF9134800F0DC
:10C4300029F9134800F026F9124800F023F91248B0
:10C4400000F020F910BD0000A4090020B809002068
:10C45000CC090020E0090020F4090020080A00208F
:10C460001C0A0020300A0020440A0020580A00203C
:10C470006C0A0020800A0020940A0020A80A0020EC
:10C48000BC0A0020D00A0020E40A00202DE9F04177
:10C4900080460D46164600244046FFF797FA0446AC
:10C4A0000CB105B116B90020BDE8F081287818B1AB
:10C4B00094F85400012801D00020F5E795F82000F9
:10C4C00000F0010018B1A86A08B90020ECE795F85F
:10C4D000251084F8451094F8450010B9322184F8ED
:10C4E000451094F8451001EB4101C80005F0BCFD72
:10C4F000C4F88C00D4F88C0048B194F84530182268
:10C5000004F17000D4F88C1008F008F901E0002064
:10C51000CAE795F8200000F00100D8B994F845105A
:10C52000080105F0A1FDC4F88800D4F8880048B1DE
:10C5300094F84530102204F15800D4F8881008F01F
:10C54000EDF807E0D4F88C0004F01AFF0020C4F8DE
:10C550008C00A9E7296A216404F1200720213846CC
:10C56000FBF72BFE1F2229463846FBF70DFEE86A33
:10C57000F862A86AB86295F8240087F82400286B4E
:10C580003863084830610848F0600848B0600848DF
:10C5900070600848306008487061022084F85400D8
:10C5A000012081E78D230108B92101083922010802
:10C5B00053220108DD220108D520010838B50546BF
:10C5C00001213C2000F002FF0121084600F0FEFEA0
:10C5D00001211348FFF768F9AC681CB911A002F0FB
:10C5E000A9FC38BD2088ADF8000010208DF80300AC
:10C5F00002208DF8020069466068FFF7C9F8207ACA
:10C60000012804D121886068FFF7A1F905E0207AAC
:10C6100018B921886068FFF798F900BFE1E70000CA
:10C62000000230004F5053206973204E554C4C0D82
:10C630000A00000010B5054800F092F8044800F028
:10C640008FF804A002F076FC10BD0000A80A0020BC
:10C65000BC0A0020414320C8ABB5CD0010B5054849
:10C6600000F0A9F8044800F0A6F804A002F062FC6B
:10C6700010BD0000A80A0020BC0A0020414320C8C9
:10C68000ABB8DF0070B505462C68206800B970BDF6
:10C6900020462168884700BFF9E7000038B5054605
:10C6A00001213C2000F092FEAC681CB910A002F001
:10C6B00041FC38BD2088ADF8000010208DF8030043
:10C6C00002208DF8020069466068FFF761F8207A61
:10C6D000012804D121886068FFF739F905E0207A44
:10C6E00018B921886068FFF730F900BFE1E7000062
:10C6F0004F5053206973204E554C4C0D0A000000DA
:10C7000038B505460121042000F060FEAC6804B98C
:10C7100038BD2088ADF8000010208DF803000320FC
:10C720008DF8020069466068FFF732F8207A012828
:10C7300004D121886068FFF70AF905E0207A18B96A
:10C7400021886068FFF701F900BFE1E710B50446F2
:10C7500021886068FFF7F9F800202072012010BDE1
:10C7600070B5044620684568686808B9002070BD47
:10C7700022689068696888470120F8E710B5044688
:10C7800021886068FFF7D8F810BD70B504462068AE
:10C790004568A86808B9032070BD22689068A96838
:10C7A0008847F9E710B5044621886068FFF7CFF89D
:10C7B0000120207210BD70B50446206845682868C5
:10C7C00008B9002070BD2268906829688847012058
:10C7D000F8E738B505460121102000F0F7FDAC68F8
:10C7E00004B938BD2088ADF8000048208DF803005A
:10C7F00003208DF8020069466068FEF7C9FF00BF9C
:10C80000EFE7000010B50748C488074A0221204618
:10C8100002F0ACFA054904480068FBF757FD0449EB
:10C82000486010BD60000020B400002000003041CE
:10C83000380B002070B50446002000BF14F8016BCF
:10C840008E4204D1012A00D108E0551EEAB203B994
:10C8500004E0451CA8B25D1EABB2EFE700BF70BD9F
:10C8600010B51548C07E012803D164201349086023
:10C8700003E04FF47A7011490860104801681048CD
:10C8800001F05AFB012816D10E4801780068401CBF
:10C890000C4A106001F0010020B100BF0A48FFF708
:10C8A0005FFF04E000BF0848FFF785FF00BF0021DD
:10C8B000034801F041FB10BD780B00200800002068
:10C8C0000000002004000020300A002000BFFEE726
:10C8D000704710B54FF4A06000F03AF810BD0000AA
:10C8E00070B5002100230F22C47804B3154C2468CE
:10C8F00004F4E064C4F5E064210AC1F10403CA4011
:10C90000447804FA03F184781440214309010E4C61
:10C910000678A155047804F01F050124AC40057881
:10C920006D11AD0005F1E025C5F8004109E004787E
:10C9300004F01F050124AC40044D0678761145F83B
:10C94000264070BD0CED00E000E400E080E100E076
:10C9500002490143024A1160704700000000FA05D5
:10C960000CED00E0024A0A400243024B1A60704795
:10C9700080FFFF1F08ED00E00648006800F4E0605B
:10C9800005490843001D03490860BFF34F8F00BFEE
:10C99000FEE700000CED00E00000FA0510B50A48C3
:10C9A000FFF709FF0120FEF772FC0848FFF703FFBD
:10C9B0004FF4FA70FEF76BFC0448FFF7D1FE04A0B9
:10C9C00002F0B8FA10BD0000A80A0020BC0A00203E
:10C9D0004F50454E5F313256506F776572526561E8
:10C9E0006C790D0A0000000010B5FFF7D7FF10BDED
:10C9F00010B50120024988700248FFF7DCFE10BD27
:10CA000068060020CC090020014908627047000038
:10CA100000000E4210B5044604F10B03184607F05F
:10CA2000C7FE1868C0F309300A2190FBF1F081B20B
:10CA30000F4881871868C0F309300A2190FBF1F094
:10CA40000B4981F866005868800C81B20848C1879C
:10CA50005868800C0649A1F8460018791968890DB4
:10CA600060F38D210248A0F84810012010BD00009D
:10CA7000A007002070B5054605F10B04204607F01D
:10CA800097FE6268C2F3C262D0B2074A926E116A20
:10CA900088472268C2F30262D0B2034A926E916A5A
:10CAA0008847012070BD0000A007002010B5044693
:10CAB00004F10B03184607F07BFE988881B2074803
:10CAC000A0F860105868010C0448A0F862101868BB
:10CAD000000C024981F84F00012010BDA007002082
:10CAE00010B5044604F10B03184607F061FE988860
:10CAF000010A0E4880F864105868010E0B4880F84F
:10CB000065109888010A094880F850105868010E8D
:10CB1000064880F852105868010C044880F85110FB
:10CB2000197980F85310012010BD0000A0070020E3
:10CB300070B50546FCF75AFA05F10B04204607F0DC
:10CB400037FE6068C0F3892000EB80004FF6FF716C
:10CB500001EA40000549A1F841006068000D81B27A
:10CB60000248A0F84310012070BD0000A00700207B
:10CB700010B5044604F10B03184607F019FE0449EA
:10CB80001868886202485968C162012010BD00001F
:10CB9000D022002010B5044604F10B03184607F01C
:10CBA00007FE044918680863024859684163012078
:10CBB00010BD0000D022002010B5044604F10B0384
:10CBC000184607F0F5FD044918688863024859685B
:10CBD000C163012010BD0000D022002070B50546C1
:10CBE00005F10B04204607F0E3FD2068C0F3404048
:10CBF000C1B21F4880F845106068000C0A2190FB04
:10CC0000F1F01B49A1F833006068000C0A2190FB89
:10CC1000F1F080B240F480511548A0F84A10A08885
:10CC2000C0F38D0012490880217811484171208895
:10CC3000010A0F4880F83B106068010C0C48A0F80E
:10CC400039102268C2F30042D0B2094A926E91684C
:10CC500088472068C0F30040C1B2054880F85A10E8
:10CC60002068800C81B202480181012070BD000063
:10CC7000A007002010B5044604F10B03184607F086
:10CC800097FD9888C0F38D0081B20C48A0F837104A
:10CC90009888C0F38D0081B20848C1801868000AE6
:10CCA00006494880000C08715868000DA0F57A60AC
:10CCB00081B20248A0F83510012010BDA007002065
:10CCC00010B5044604F10B03184607F071FD044942
:10CCD00018680865024859684165012010BD0000C8
:10CCE000D02200202DE9F0412A48058801272A4852
:10CCF0002A494860002008702B463A4620212648E1
:10CD0000FFF798FD044625494C700846416824A069
:10CD100002F010F9AC4202D10120BDE8F081781C8C
:10CD2000C7B231E01C48005D202802D1601C84B2EB
:10CD30002AE026461848011918480278083040F8B9
:10CD400022102B463A4620211348FFF773FD044674
:10CD5000A01BC1B2114802781830815418380378EA
:10CD6000083050F823200838017811A002F0E2F8CA
:10CD70000A480078401C09490870084600780428D1
:10CD800000DB03E0781CC7B2AC42CBD100BF01206E
:10CD9000C3E700001E020020EE1B0020E81E00205A
:10CDA000696E6F757420636D643A25730A00000024
:10CDB000256420706172616D3A25730A00000000DD
:10CDC0007CB5002000900190009001904FF44570D8
:10CDD0005E49086048600020087248720820887226
:10CDE0006C4600F001FC012801D0012200E0002285
:10CDF000D4E9000162F31961C4E9000100F0F4FB19
:10CE0000012801D0012200E00022D4E9001062F3E1
:10CE10009B60C4E9001000F0EFFB012801D0012065
:10CE200000E00020D4E9001260F31D72C4E9001292
:10CE300000F0E2FB012801D0012100E00021D4E94B
:10CE4000002061F39F70C4E900204148C07808B910
:10CE5000012200E00022D4E9000162F31141C4E99B
:10CE600000013B48807808B9012100E00021D4E9A5
:10CE7000002061F39340C4E90020FEF737F9D4E9BC
:10CE8000001260F38B21C4E90012FEF771F8D4E9B7
:10CE9000001260F31552C4E900122E48B0F81B10BE
:10CEA000D4E9000261F35D50C4E900022948B0F8FA
:10CEB0001D20D4E9001062F31431C4E90010FEF71C
:10CEC000DBF80246D4E9001062F3DF71C4E9001018
:10CED000214908682149FBF7F9F90646FBF709FCE7
:10CEE000054642F210718D4201D90A4600E02A46F9
:10CEF000D4E9000162F30C01C4E900012420FEF72B
:10CF000011FAD4E9002160F39E72C4E900211048AF
:10CF10000179D4E9000261F34F32C4E9000200BF95
:10CF20000F48FFF732FCD4E9001260F3D752C4E98E
:10CF30000012204607F043FC04480B3000990160C2
:10CF4000019941600B3804F003F87CBD30230020C8
:10CF500068060020C00B00206C00002000007A440E
:10CF6000E40A00201CB50020009001900090019080
:10CF70004FF47A70284908604860002008724872AF
:10CF8000082088726C462820FEF7CCF958B9262074
:10CF9000FEF7C8F938B91C20FEF7C4F918B92120EA
:10CFA000FEF7C0F908B1012200E00022D4E9000137
:10CFB00062F38E31C4E9000118480078042805DBCB
:10CFC00016480078052801DC012200E00022D4E99F
:10CFD000000162F3CF31C4E900011149486880477C
:10CFE0000246D4E9001062F31F60C4E90010142265
:10CFF000D4E9000162F31741C4E90001204607F0BB
:10D00000DEFB05480B3000990160019941600B3847
:10D0100003F09EFF1CBD0000302300208823002069
:10D020006C0000201CB50020009001900090019041
:10D0300040F23F400E490860486000200872487284
:10D04000082088726C460122D4E9001062F30701BF
:10D05000C4E90010204607F0B2FB05480B300099E8
:10D060000160019941600B3803F072FF1CBD0000A4
:10D070003023002070B5054605F10B04204607F06B
:10D0800097FB2268C2F30362D0B2064A926E91699E
:10D0900088476268920FD0B2024A926E116988473F
:10D0A000012070BDA00700207047000070B544A0AB
:10D0B00001F040FF4D4A906E926ED16988474C490D
:10D0C00051F8204021464BA001F034FF474890F82A
:10D0D00066204E4800784E4B53F820104DA001F0CA
:10D0E00029FF424890F8450008B151A000E054A043
:10D0F000014657A001F01EFF3C48B0F84320B0F8AD
:10D10000411056A001F016FF5C48B0F81D20B0F8A1
:10D110001B105BA001F00EFF6149C868FBF7FDFA28
:10D12000044622460B465FA001F004FF624988686E
:10D13000804704466049486880470546224629469C
:10D140005EA001F0F7FE00BF6248FFF71EFB08B1CA
:10D1500061A000E062A0044600F056FA08B15EA0AB
:10D1600000E05FA00546224629465FA001F0E2FEEE
:10D170006448C07808B164A000E064A00246614839
:10D18000807808B162A000E062A0014662A001F0D0
:10D19000D1FE49490868FBF7C0FA044622460B460F
:10D1A00063A001F0C7FE114A906E926ED16A884763
:10D1B0000446214662A001F0BDFEFEF7E9F870BD0D
:10D1C0000D0AA1AAA1AAA1AAA1AAA1AAA1AAA1AA3B
:10D1D000A1AAA1AAA1AAA1AAA1AAA1AAA1AAA1AAF7
:10D1E000A1AAA1AAA1AAA1AA0D0A0000A007002035
:10D1F0002C0800200D0A56435520576F726B696E3C
:10D2000067204D6F64652025730D0A008823002078
:10D210000C0800204368617267696E67205374616F
:10D22000676520257309534F432025640D0A0000CC
:10D23000436F6E7374616E74566F6C7461676500D2
:10D24000436F6E7374616E7443757272656E7400B1
:10D250004D6F64652025730D0A00000044656D6103
:10D260006E6420766F6C7461676520256420637539
:10D270007272656E742025640D0A0000C00B0020D8
:10D280004F757470757420766F6C746167652025B6
:10D29000642063757272656E742025640D0A000047
:10D2A000380B002053616D706C20766F6C74616771
:10D2B00065202566200D0A006C00002054656D7005
:10D2C000312025642047554E5F54454D502025643C
:10D2D0000D0A0000440A00204F70656E0000000037
:10D2E000436C6F736500000044435F52656C617965
:10D2F0002025732041435F52656C61792025730DB1
:10D300000A00000068060020434300004343320047
:10D31000434331004350000043502D434331202507
:10D32000732043432D4343322025730D0A00000030
:10D33000434320522069732025660D0A0000000037
:10D340004F424320636F6E6E6563742025640D0A3F
:10D350000000000001460020034A506820F44040CD
:10D3600008435060704700000010024029B1064A8F
:10D3700052690243044B5A6104E0034A52698243F2
:10D38000014B5A61704700000010024029B1064A63
:10D39000D2690243044BDA6104E0034AD269824352
:10D3A000014BDA61704700000010024029B1064AC3
:10D3B00012690243044B1A6104E0034A1269824372
:10D3C000014B1A61704700000010024029B1064A63
:10D3D00092690243044B9A6104E0034A92698243D2
:10D3E000014B9A617047000000100240014908603B
:10D3F00070470000400442422DE9F0410021002224
:10D40000002500230026002400278C46DFF86081D9
:10D41000D8F8048008F00C0121B1042907D00829AC
:10D4200059D109E0DFF84C81C0F8008058E0DFF8FE
:10D430004481C0F8008053E0DFF83481D8F80480DC
:10D4400008F47012DFF82881D8F8048008F48035D9
:10D45000920C0D2A01D0921C00E0062235B9DFF8AB
:10D46000188102FB08F8C0F8008033E0DFF8008183
:10D47000D8F82C8008F48036DFF8F480D8F82C80B7
:10D4800008F00F0808F1010446B9DFF8E880B8FB9E
:10D49000F4F808FB02F8C0F800801BE0DFF8D08049
:10D4A000D8F82C80C8F3031808F10107DFF8C08012
:10D4B000D8F82C80C8F3032808F1020CDFF8B480F8
:10D4C000B8FBF7F808FB0CF8B8FBF4F808FB02F817
:10D4D000C0F8008004E0DFF89C80C0F8008000BF46
:10D4E00000BFDFF88C80D8F8048008F0F00109094B
:10D4F000DFF8888018F80130D0F8008028FA03F8A7
:10D50000C0F80480DFF86880D8F8048008F4E0618F
:10D51000090ADFF8688018F80130D0F8048028FA8A
:10D5200003F8C0F80880DFF84880D8F8048008F4D1
:10D530006051C90ADFF8448018F80130D0F804803F
:10D5400028FA03F8C0F80C80DFF82480D8F80480AB
:10D5500008F44041890BDFF8288018F80130D0F832
:10D560000C80B8FBF3F8C0F81080BDE8F081000033
:10D570000010024000127A0000093D00ED05002075
:10D58000FD05002010B501460022002300204A11AD
:10D59000012A02D1094C236806E0022A02D1074C75
:10D5A000236A01E0054C636A01F01F0201249440E4
:10D5B0001C400CB1012000E0002010BD0010024012
:10D5C0000149086070470000800442420149086038
:10D5D000704700003C0442420249096A0143014A83
:10D5E000116270470010024010B50248FFF7CDF8F5
:10D5F00010BD0000440A002010B50248FFF7C5F82E
:10D6000010BD0000580A002010B50248FFF7BDF811
:10D6100010BD0000580A002010B50D48008F00F41E
:10D62000804058B90A4890F8380000F0200028B926
:10D63000074890F8380000F0400030B12720FDF78F
:10D640008BFE00200249886310BD0120FCE700002A
:10D65000C00B002070B505460E46002400BF03E055
:10D66000285D00F087FE641CB442F9DB70BD70B524
:10D6700005460E46002400BF03E0285D00F07AFE58
:10D68000641CB442F9DB0D2000F074FE0A2000F0A7
:10D6900071FE002403E0285D00F028FD641CB44204
:10D6A000F9DB70BD0348008840F010000149088094
:10D6B0007047000004280040034800884FF6EF71CF
:10D6C00008400149088070470428004000210348B1
:10D6D0000188001F008841EA004070471C28004074
:10D6E00010B501214FF0C050FFF750FE4FF400700D
:10D6F000FFF772FF0120FFF769FF0120FFF784F9B0
:10D70000FBF7B8FB0120FFF75BFF00BF6120FFF7CD
:10D7100039FF0028FAD04FF40070FFF75DFF0120B9
:10D72000FFF754FF00F024F800F018F849F63F40E6
:10D7300000F004F800F012F810BD000000B5024639
:10D74000FFF7B0FFC2F3034003490880091D0A80B8
:10D75000FFF7B2FF00BD00000828004000BF0348EB
:10D76000008800F020000028F9D07047042800400D
:10D77000074800884FF6F77108400549088000BF48
:10D780000348008800F008000028F9D07047000026
:10D790000428004010B5012013490860FEF7BAFCC8
:10D7A0009020FEF7F1FC0020FEF7EEFCFEF7D2FC25
:10D7B000FEF7B0FC9120FEF7E7FCFEF76BFC0B498F
:10D7C0000880FEF767FC09494880FEF7C3FC07485C
:10D7D00040880649098840EA012000B203490880D0
:10D7E0000846008880B210BD98812142C400002004
:10D7F00070B505461DB1686808B1A86808B9002071
:10D8000070BD00240EE004EB440000EBC4001B4993
:10D8100001EB001000782978884201D10020EFE761
:10D82000601CC4B2022CEED3002422E004EB4400BE
:10D8300000EBC400114901EB00100078FF2816D15D
:10D8400004EB440101EBC4010C4A02EB011020225D
:10D850002946FAF799FC012004EB440101EBC401CD
:10D86000064A02EB011181F854000548C8E7601C24
:10D87000C4B2022CDAD30020C2E70000B4120020A8
:10D880004401002000200149088070471E0200204A
:10D89000704772B6704762B67047000070B5FEF709
:10D8A000AFFA0646FEF7E6F904460025012C01D141
:10D8B000012506E0022C01D0032C01D1022500E055
:10D8C000002512480078854205D0002010490860E4
:10D8D0000E48057019E00F480078854203D10020FA
:10D8E0000B49086011E00A480068401C08490860BC
:10D8F00008460068022808D30448007805490870E3
:10D900000548047000200249086070BDAC0000208A
:10D91000C0000020AD000020AE00002070B504461D
:10D920000D46FFF7D3FE0646206818B9266020682A
:10D93000284460606068B04201D8012070BD0020BA
:10D94000FCE70146002008604860012070470000A5
:10D9500010B50A48B0F8410020B90920FDF7FCFCD9
:10D96000002010BD0548B0F8430020B90A20FDF79B
:10D97000F3FC0020F5E70120F3E70000A0070020FA
:10D9800010B500F001F810BD0CB50020019000901A
:10D990004048006840F480303E49086000BF3D4880
:10D9A000006800F4003000900198401C019000983D
:10D9B00020B94FF6FF7101988842F0D135480068D0
:10D9C00000F4003010B10120009001E00020009030
:10D9D000009801285CD13048006840F010002E49C2
:10D9E00008600846006820F00300086008460068E8
:10D9F00040F0020008602748406826494860084611
:10DA0000406848600846406840F4806048600846C6
:10DA1000C06A224908401F49C8620846C06A2049B6
:10DA200008431C49C8620846006840F080600860EE
:10DA300000BF1848006800F000600028F9D01548C1
:10DA4000406820F47C10134948600846406840F460
:10DA5000E81048600846006840F08070086000BF29
:10DA60000C48006800F000700028F9D009484068B0
:10DA700020F00300074948600846406840F0020073
:10DA8000486000BF0348406800F00C000828F9D146
:10DA90000CBD0000001002400020024000F0FEFF1C
:10DAA000140801000146024801710120704700007E
:10DAB00070070020014602480170012070470000F5
:10DAC000700700200146032903D0042901D000205B
:10DAD00070470248C1700120FAE70000700700207B
:10DAE0000146012902D009B1002070470148817028
:10DAF0000120FAE770070020002201490A5470470C
:10DB0000A02300200146012902D009B1002070475E
:10DB1000014841700120FAE77007002010B5FFF7B7
:10DB2000E1F808B9002010BD0020154908801DE06B
:10DB3000134A128802EB4202124B03EB8202516835
:10DB4000114A5068FAF744FB58B10D48008800EBC1
:10DB500040000C4901EB8000846804B1A04701201B
:10DB6000E1E707480088401C054908800448008810
:10DB70001328DDD305A001F0DDF90020D3E7000074
:10DB8000280200208C500108E81E0020416E2075FC
:10DB90006E7265636F676E697A656420434D4420D9
:10DBA000210A000010B50948006820B9084803F0B0
:10DBB00009F9064908600548006803F096F920B99C
:10DBC0000A210248006803F083F910BD58010020C3
:10DBD0002D4A010810B5FBF783F920B908A001F020
:10DBE000A9F9002010BDFDF7A3FA08B90020F9E754
:10DBF000FDF74EFA08B90020F4E70120F2E7000033
:10DC0000424D5320546865204368617267696E67AE
:10DC10002050686173652053746F70732041626E89
:10DC20006F726D616C6C790A0D0000000F4800681E
:10DC3000401C0E4908600E480068401C0C490860F2
:10DC40000A4800684FF47A71B0FBF1F201FB120050
:10DC5000012804D107480068401C064908600648AE
:10DC6000007810B90120044908707047F4010020C1
:10DC7000EC010020F8010020F001002030B516482A
:10DC800000684FF47A72B0FBF2F1B1F1807F01D3FA
:10DC900001201DE021F07F40401E4FF0E022506146
:10DCA00050170F22002807DA13071D0E0B4B00F048
:10DCB0000F04241F1D5503E013071C0E084B1C54B2
:10DCC00000BF00204FF0E02290610720106100208B
:10DCD00008B100BFFEE730BD0C00002018ED00E0E9
:10DCE00000E400E010B5FEF7C1FA4FF417720249E4
:10DCF000024802F019FD10BD9814002000F0010840
:10DD000010B51648006840F0010014490860084644
:10DD100040681349084011494860084600681149A5
:10DD200008400E4908600846006820F4802008601A
:10DD30000846406820F4FE0048600846006820F06D
:10DD4000A05008604FF47F0088600020C862FFF791
:10DD500017FE4FF000600449086010BD001002403B
:10DD60000000FFF0FFFFF6FE08ED00E02DE9F047B0
:10DD70000D4804880D4A0021204600F0F7FF0B48AB
:10DD80000068FAF7CAFC07463A460B4608480949B4
:10DD9000FAF725FC0546FAF7EBFC8146FDF73EFC59
:10DDA00005490872BDE8F08760000020B00000203F
:10DDB0009A99999999991340380B002010B501212F
:10DDC000054800F04AF828B100F0D6F801210248D1
:10DDD00000F034F810BD0000000400407FB5054697
:10DDE0000C4601210220FFF7D1FAADF80850ADF83A
:10DDF00004400020ADF80A00ADF8060001A90E4865
:10DE000000F048F8012211460B4800F037F81D20B9
:10DE10008DF8000001208DF8010003208DF802002C
:10DE200001208DF803006846FEF75AFD01210248E3
:10DE300000F007F87FBD000000040040CA430282E2
:10DE4000704721B1028842F00102028004E002889A
:10DE50004FF6FE731A400280704730B5024600202C
:10DE600000230024158A05EA0103958905EA0104C7
:10DE700013B10CB1012000E0002030BD1AB183893C
:10DE80000B43838102E083898B43838170478185C3
:10DE900070470000002202881D4B98420ED01D4B97
:10DEA00098420BD0B0F1804F08D01B4B984205D060
:10DEB0001A4B984202D01A4B984204D14FF68F73F6
:10DEC0001A404B881A43174B984207D0164B98427A
:10DED00004D04FF6FF431A40CB881A4302808B8848
:10DEE00083850B8803850A4B98420BD0094B9842D7
:10DEF00008D00E4B984205D00D4B984202D00D4BE6
:10DF0000984201D10B7A0386012383827047000077
:10DF1000002C014000340140000400400008004093
:10DF2000000C004000100040001400400040014080
:10DF300000440140004801400246002321B90D4839
:10DF400000681060012070470A4803681068984212
:10DF500005D81068181A884209D30120F3E7106821
:10DF6000C0F1FF301844884201D30120EBE70020C4
:10DF7000E9E70000F401002010B5084800680188B6
:10DF80000748FFF784FF0549096848688047034848
:10DF9000006880680149086010BD0000143400204A
:10DFA000000400404F48007801280AD14E48C0685C
:10DFB000401C4D49C8600120087000204949087084
:10DFC00000E070474848C0680521B0FBF1F201FB52
:10DFD000120030B94448C06818B101204249487065
:10DFE00000E0EEE74048C0680A21B0FBF1F201FB17
:10DFF000120028B93C48C06810B101203A49887025
:10E000003948C0681421B0FBF1F201FB120028B9B5
:10E010003548C06810B101203349C8703248C06823
:10E020003221B0FBF1F201FB120028B92E48C06882
:10E0300010B101202C4908712B48C0686421B0FB45
:10E04000F1F201FB120028B92748C06810B1012085
:10E05000254948712448C0684FF4FA71B0FBF1F2C9
:10E0600001FB120028B92048C06810B101201E49E8
:10E0700088711D48C0684FF47A71B0FBF1F201FB62
:10E08000120028B91848C06810B101201649C8719B
:10E090001548C06840F2DC51B0FBF1F201FB120000
:10E0A00028B91148C06810B101200F4908720E4804
:10E0B000C0684FF4FA61B0FBF1F201FB120028B91D
:10E0C0000948C06810B10120074948720648C06875
:10E0D00041F27071884202D300200349C86000BF3A
:10E0E0006FE70000F00100208814002010B50446FE
:10E0F0002146054800F01FFB00BF0348008800F0E0
:10E1000080000028F9D010BD004C004010B540F24E
:10E110002551394800F04FFAF8B1374800F006FBB6
:10E12000C4B236480088C82808DA34480188008814
:10E13000401C324A10803248445402E000202F49EB
:10E1400008800A2C04D1FFF7E9FCFFF79BFB10BD08
:10E1500040F22551284800F006FA40F224412648B2
:10E1600000F029FA48B1FFF78DFB234800F0DEFAF2
:10E1700040F22441204800F0F6F940F227711E4891
:10E1800000F019FA20B140F227711B4800F0EBF9BA
:10E1900040F22661184800F00EFA20B140F22661E4
:10E1A000154800F0E0F90821134800F0F7F90128BC
:10E1B00006D10821104800F0CDF90F4800F0B6FA5A
:10E1C00004210D4800F0EAF9012806D104210A488B
:10E1D00000F0C0F9084800F0A9FA0221064800F052
:10E1E000DDF9012806D10221034800F0B3F9024805
:10E1F00000F09CFA00BFAAE7004C00401E0200207D
:10E20000EE1B002010B540F22551334800F0D3F941
:10E21000E8B1314800F08AFAC4B230480088C82812
:10E2200008DA2E4801880088401C2C4A10802C48AF
:10E23000445402E000202949088000202949088030
:10E240002949087040F22551234800F08CF940F22A
:10E250002441214800F0AFF950B11F4800F066FAA0
:10E2600001202149087040F224411B4800F07BF94D
:10E2700040F22661184800F09EF920B140F2266174
:10E28000154800F070F90821134800F087F90128BB
:10E2900006D10821104800F05DF90F4800F046FA59
:10E2A00004210D4800F07AF9012806D104210A481A
:10E2B00000F050F9084800F039FA0221064800F051
:10E2C0006DF9012806D10221034800F043F9024804
:10E2D00000F02CFA10BD0000005000402402002085
:10E2E000B61C0020200200202202002010B540F2BF
:10E2F00025511D4800F05FF910B31B4800F016FAD5
:10E30000C4B21A48008800F40040C8B91748008811
:10E3100000F4804060B10A2C03D00020134908802B
:10E3200020E01248008840F400401049088019E0BD
:10E330000D2C06D10D48008840F480400B49088020
:10E3400010E00A480088C0F30D0009490C54074842
:10E350000088401C0549088008460088C72801DD60
:10E360000020088010BD0000003801400E0200208F
:10E370006019002010B504462146054800F0DBF97D
:10E3800000BF0348008800F080000028F9D010BDCD
:10E390000044004010B540F22551304800F00BF920
:10E3A000C0B12E4800F0C2F9C4B22D480088FE2842
:10E3B00008DA2B4801880088401C294A1080294827
:10E3C000445402E000202649088040F225512348A9
:10E3D00000F0C9F840F22441204800F0ECF850B1B8
:10E3E0001E4800F0A3F901201F49087040F22441A3
:10E3F0001A4800F0B8F840F22661184800F0DBF83F
:10E4000020B140F22661154800F0ADF8082113480C
:10E4100000F0C4F8012806D10821104800F09AF84D
:10E420000E4800F083F904210C4800F0B7F80128E9
:10E4300006D10421094800F08DF8084800F076F96B
:10E440000221064800F0AAF8012806D1022103485B
:10E4500000F080F8014800F069F910BD0044004068
:10E4600010020020281A00201202002010B540F2ED
:10E470002551334800F09FF8E8B1314800F056F9D3
:10E48000C4B230480088C82808DA2E4801880088BD
:10E49000401C2C4A10802C48445402E0002029499A
:10E4A00008800020294908802949087040F2255138
:10E4B000234800F058F840F22441214800F07BF84E
:10E4C00050B11F4800F032F901202149087040F294
:10E4D00024411B4800F047F840F22661184800F03C
:10E4E0006AF820B140F22661154800F03CF8082196
:10E4F000134800F053F8012806D10821104800F015
:10E5000029F80F4800F012F904210D4800F046F8F0
:10E51000012806D104210A4800F01CF8084800F040
:10E5200005F90221064800F039F8012806D1022138
:10E53000034800F00FF8024800F0F8F810BD0000A2
:10E540000048004018020020261B00201402002072
:10E550001602002001F40072B2F5007F00D100BF66
:10E56000CA430280704710B50022002340F66A14A7
:10E57000A14200D100BF0A1201249440A3B2DC439F
:10E58000048010BD21B1828942F40052828104E0EE
:10E5900082894DF6FF731A4082817047024600203F
:10E5A000B1F5007F00D100BF13880B400BB10120F3
:10E5B00000E00020704770B50246002400230025CB
:10E5C000002040F66A16B14200D100BFC1F34215E7
:10E5D00001F01F03012606FA03F3012D02D19689EB
:10E5E000334006E0022D02D1168A334001E0968ABC
:10E5F00033400C12012606FA04F41688344013B195
:10E600000CB1012000E0002070BDF0B503460024ED
:10E6100000260025002040F66A17B94200D100BF4D
:10E620001846C1F3421401F01F06012707FA06F548
:10E63000012C01D10C3004E0022C01D1103000E09B
:10E6400014301AB107682F43076002E00768AF4330
:10E650000760F0BD2DE9F04786B005460E46002460
:10E66000A24600BFA1460027B08900B100BF2F46D7
:10E670002C8A4CF6FF700440F08804432C82AC894D
:10E680004EF6F3100440B08831890843718908437D
:10E690000443AC81AC8A4FF6FF400440B089044388
:10E6A000AC8201A8FEF7A8FE1F48874202D1DDF820
:10E6B00010A001E0DDF80CA0A88900F4004040B1F2
:10E6C0000AEBCA0000EB0A1031684900B0FBF1F810
:10E6D00007E00AEBCA0000EB0A1031688900B0FBC2
:10E6E000F1F86420B8FBF0F004012009642101FB7B
:10E6F0001089A88900F4004040B1322000EBC90025
:10E70000B0FBF1F000F00700044308E0322000EB1A
:10E7100009106421B0FBF1F000F00F0004432C81DC
:10E7200006B0BDE8F0870000003801400146888847
:10E73000C0F308007047C1F30802828070470000F0
:10E740002DE9F74F84B00C4617460026FDF78EFDE5
:10E750000498002856D12079D34908706079487010
:10E76000A0790006E17940EA0140217A40EA0120DF
:10E77000617A0843CC494860A07AE17A40EA0120F6
:10E78000C9490881E07B0006A17B40EA0140617B2A
:10E7900040EA0120217B0843C349C860207C617C9A
:10E7A00040EA0120C0490882701E88610020C861CB
:10E7B00048624FF6FF7008840020BC490870BA48D0
:10E7C000008AB949C968B84A1289CDE90021029086
:10E7D000B548436842780178B5A000F0ABFBB24879
:10E7E000008AB149C968B04A1289CDE90021029076
:10E7F000AD48436842780178BC4800F09BFBFAF7CB
:10E8000043FC4EE104980128FBD1A848007810B1E0
:10E8100007B0BDE8F08FE0780006A17840EA01403B
:10E82000617840EA0120217808439F494861FAF75E
:10E83000EBFBFDF71BFD9C483A464169ACA000F09C
:10E8400079FB9948806998494969884272D096480D
:10E850004069954988610846C169A7F10D000844DF
:10E860009149C8610846C369808BC0F30A02084613
:10E87000C069C10AA4A000F05DFBFCF75DFE8A48F8
:10E88000008C8949C969B0EBD12F14D08648C06982
:10E89000C0F3CF20844908840846C069A6490844CB
:10E8A0004FEAD0284FEAC8284146A4A000F042FB16
:10E8B0004046FCF79DFD04F1040AA7F10D00C117C5
:10E8C00000EB9171C1F3870BC11700EB91718910B7
:10E8D000A0EB810169B1A0A000F02CFBA7F1090118
:10E8E00008190322FF21F9F761FC0BF1010000F088
:10E8F000FF0B6D48406A904900EB01086A48C06907
:10E9000069494862002540E0002614E05AF82510C5
:10E910004046FCF7D9FD042800D10DE0701CC6B2BA
:10E92000032E08DB414692A000F004FB01205F4962
:10E9300008706DE7B3E0E9E700BFD8F80090012D5B
:10E9400003DBABF10100A84206DC5AF825204B4658
:10E95000414690A000F0EEFA5AF8250048450DD047
:10E9600094A000F0E7FA5AF825204B46414689A0CA
:10E9700000F0E0FA01204D49087049E708F1040869
:10E98000032E00DB03E0681CC5B25D45BCDB00BFA5
:10E99000FDF76CFCA7F10D0081B28F480288201DA5
:10E9A000FAF7FAFB8C4908803F4801898A480288B7
:10E9B0008AA000F0BFFAFDF759FC3B4840693A498C
:10E9C000C968884269D138480089834909888842E2
:10E9D00003D08BA000F0AEFA1AE700263248C168D7
:10E9E00091A000F0A7FA9948FCF702FD0FE09849C2
:10E9F0009648FCF769FD042800D109E0701CC6B2F6
:10EA0000032E04DB914993A000F094FA00E0EEE7B6
:10EA100000BF8E48D0F800904B468D4A01465DA05D
:10EA200000F088FA8A48814503D001201F49087008
:10EA3000EEE6002612E01C4841688448001DFCF701
:10EA400043FD042800D10AE0701CC6B2032E05DB8A
:10EA50007E49091D88A000F06DFA00E0EBE700BFD9
:10EA60007A48001DD0F800900F484B467749091DA1
:10EA700042688BA000F05EFA0B484068484503D01E
:10EA800001200A490870C3E6FDF7F0FBFAF7BCFA6B
:10EA90008CA000F04FFAFDF76FFFFCF7E9FCFDF7E3
:10EAA000E5FB00BFB4E60000381900206605002031
:10EAB0000D0A3636365570642D2D747970653A25F9
:10EAC00064202C7665723A25642C54627974653A18
:10EAD00025642C204372633A25642C5061673A25E3
:10EAE000642C506C656E3A25640D0A00745301085D
:10EAF0000A0D43757272204261673A25642C206CBE
:10EB0000656E2025640A0D0057726974652D616475
:10EB100064723A20736563746F722025642C2C6FC5
:10EB20006666736574202564202C7265636C656E5F
:10EB3000202530640D0A000000600208343443755B
:10EB400072722045726173652D2D616464723A2082
:10EB50002530780D0A0000000A0D6C6173742D2DAC
:10EB60002D2D2D626167212121212121210A0D00F6
:10EB70002132322121212121212121215772697441
:10EB8000652D4661696C2D616464723A2025307888
:10EB90000D0A000061646472202530782C2C5772B5
:10EBA000697465202530782C2C72656164202530CD
:10EBB000780D0A000A0D207265616476616C20216F
:10EBC0003D20557064646174615B695D2921212178
:10EBD00021210A0D00000000640500203132325569
:10EBE0007064486561642E46696C654372633D25B7
:10EBF00030782C544372633D2530780D0A000000B4
:10EC0000557064486561642E46696C654372632083
:10EC1000213D2054437263202121212072657475A7
:10EC2000726E210D0A0000002121217570642D698A
:10EC30006E666F21212057726974652D746F747030
:10EC40006167202564200D0A0000000000580208BA
:10EC50004433221155706444617461466C616721CC
:10EC60002057726974652D4661696C2D6164647208
:10EC70003A202530780D0A002121217570642D6914
:10EC80006E666F21212057726974652D4661696C2B
:10EC90002D616464723A202530780D0A000000006E
:10ECA0003161646472202530782C2C577269746548
:10ECB000202530782C2C72656164202530780D0A6F
:10ECC0000000000032327570642D616C6C20777228
:10ECD000697465204F4F4B4B2121726573746172CB
:10ECE0007421212121212121212121210D0A00002E
:10ECF00070B5C2B005460C46002641F20D00084929
:10ED0000A1F80500224629460548C01DF9F73CFA3E
:10ED10000348448001AA02A9FCF758FA42B070BD2A
:10ED20007E1D002000BFFEE710B5064A906E926E71
:10ED3000516A884720B92620FCF70EFB002010BD41
:10ED40000120FCE7A00700202DE9F04104460E4613
:10ED50001546601BF9F7B2FC80463146F9F7E8FA30
:10ED60000746F9F7C6FC80B2BDE8F0812DE9FC4703
:10ED700081460C46924604EB44003B4911F82000C2
:10ED8000002843D004EB440001EB8000408888B3A6
:10ED900004EB440001EB80004088142190FBF1F06B
:10EDA00004EB4401304A02EB8101488004EB44014A
:10EDB00002EB81014888F9F78FFC07464FF0663275
:10EDC0002A4BF9F79AFB05460022294BF9F707FC75
:10EDD000CDE90001F9F7CCFC04EB4401224A02EB37
:10EDE0008101886004EB4400114601EB80008068DB
:10EDF000CAF80000002004EB44011B4A02EB810129
:10EE0000488004EB440102F821002BE004EB4400AD
:10EE1000154901EB80000079401C04EB4401124AC3
:10EE200002EB8101087104EB4400114601EB800004
:10EE30004088484404EB440102EB8101488004EB24
:10EE40004400114601EB8000007914280AD101200A
:10EE500004EB440102F82100002004EB440102EB22
:10EE600081010871BDE8FC87480B002066660A40F6
:10EE70000000B04000200849086008480078401CA5
:10EE800006490870084600781E2803DC7F200249E6
:10EE90000839086070470000082C0040E901002094
:10EEA00044E032213EE000BF00BF00BF00BF00BF12
:10EEB00000BF00BF00BF00BF00BF00BF00BF00BF5A
:10EEC00000BF00BF00BF00BF00BF00BF00BF00BF4A
:10EED00000BF00BF00BF00BF00BF00BF00BF00BF3A
:10EEE00000BF00BF00BF00BF00BF00BF00BF00BF2A
:10EEF00000BF00BF00BF00BF00BF00BF00BF00BF1A
:10EF000000BF00BF00BF00BF00BF00BF00BF00BF09
:10EF100000BF00BF00BF00BF00BF00BF00BF00BFF9
:10EF20004A1ED1B20029BEDC421ED0B20028B8DC95
:10EF3000704700000FB4054B10B503A9044A0298AE
:10EF400000F0EEF810BC5DF814FB0000FD120108A3
:10EF5000080200200FB4084B10B504A902AA0398B8
:10EF600000F0DEF8044602A9002000F070FC204604
:10EF700010BC5DF814FB00004FF8000802E008C860
:10EF8000121F08C1002AFAD170477047002001E023
:10EF900001C1121F002AFBD1704700002DE9FF5F5D
:10EFA00082B00021DDE90430020DDDF840B00343FA
:10EFB00018D044F61050A2F2FF32424315141198B3
:10EFC00001281FD0A5EB0B00401C5FEA000A4FF0A0
:10EFD00000064E4FDFF83891B046504615D5CAF1BD
:10EFE000000413E0119801244AA3012801D16FEA1B
:10EFF0000B010298119AC0E90031C0E9024206B043
:10F00000BDE8F09FCBF10000DFE704460021404A55
:10F01000491842EB0450CDE9001012E0E00707D098
:10F0200032463B4640464946F9F767FA80468946EC
:10F0300032463B4610461946F9F75FFA06460F4638
:10F040006410002CEAD1DDE90401DDE90023BAF106
:10F05000000F06DAF9F751FA42464B46F9F74DFA36
:10F0600005E0F9F7BCFA42464B46F9F7B8FA044610
:10F070000E460022284BF9F763FB03D84FF0FF3010
:10F08000014607E00022254B20463146F9F78EF96C
:10F09000F9F79AFC102409E0002C0ADB0A2200236D
:10F0A000F9F7ACFB039B30321A55641E50EA01029B
:10F0B000F2D1641C039AC4F111031444119A012A79
:10F0C00003D0012208430DD10AE0084304D00020F8
:10F0D0004FF0110B119072E7A3EB0B056D1E0DE0C5
:10F0E0005B4504DD4FF0000205F1010504E003DAA1
:10F0F0004FF00002A5F10105002AECD00298119909
:10F10000C0E90231C0E9004579E700000000144081
:10F110000000F03F300000000000F0430000E03F3E
:10F120002DE9FF4F95B09B468946064600250FE224
:10F13000252877D100242746F84A0121059400E0CC
:10F14000044316F8013F203B01FA03F01042F7D1C7
:10F1500030782A2811D06FF02F033078A0F13002D8
:10F16000092A16D8059A44F0020402EB820203EB46
:10F1700042021044761C0590EFE759F8042B0592E3
:10F18000002A03DA504244F40054059044F002048B
:10F19000761C30782E2816D116F8010F44F004049E
:10F1A0002A280DD06FF02F023078A0F13003092B00
:10F1B00009D807EB870302EB4303C718761CF3E774
:10F1C00059F8047B761C30786C280FD006DC4C286C
:10F1D00017D068280DD06A2814D104E0742810D004
:10F1E0007A280FD10DE044F400140AE044F48014AE
:10F1F00001E044F440147278824202D104F5801494
:10F20000761C761C307866280BD013DC582877D013
:10F2100009DC002875D04528F6D04628F4D04728C8
:10F220001AD19DE118E0632835D0642879D065288B
:10F2300012D195E1702873D008DC6728F1D06928D5
:10F240006FD06E280DD06F2806D1B5E073282CD072
:10F25000752875D0782874D05A46179990476D1C38
:10F2600075E1C4F30250022809D003280DD0D9F863
:10F27000001004280DD00D6009F1040967E1D9F8E8
:10F280000010EA17C1E90052F6E7D9F800100D8026
:10F29000F2E70D70F0E719F8041B8DF8001000205C
:10F2A0008DF80100EA46012003E059F804AB4FF065
:10F2B000FF3061074FF0000102D40DE008F10101B9
:10F2C0008846B9420FDA8045F8DB1AF808100029A1
:10F2D000F4D108E008F1010188468142FADB1AF80E
:10F2E00008100029F6D105985B46A0EB08072146D7
:10F2F0003846179A00F094FA284400EB080507E016
:10F300004DE029E10DE01AF8010B5A461799904794
:10F31000B8F10108F7D25B4621463846179A13E147
:10F3200042E00A220092C4F302524FF0000A022A7D
:10F3300008D059F804CB032A4FEAEC710AD00DE04B
:10F3400029E02AE009F1070121F00702F2E802C1F1
:10F35000914609E00FFA8CFC4FEAEC71042A03D1C4
:10F360004FFA8CFC4FEAEC71002907DA0A460021BB
:10F37000DCF1000C61EB02012D2202E0220504D534
:10F380002B228DF80420012203E0E20701D0202285
:10F39000F7E7904659E00A2102E010220DE0102123
:10F3A0004FF0000A00910BE010224FF0000A44F0E9
:10F3B00004040827009203E008224FF0000A00929C
:10F3C000C4F30252022A05D059F804CB0021032AC3
:10F3D00008D009E009F1070121F00702F2E802C1B3
:10F3E000914605E01FFA8CFC042A01D10CF0FF0CB9
:10F3F0004FF00008220728D5702806D0009B83F024
:10F40000100353EA0A0305D00EE040228DF80420D1
:10F41000012208E05CEA010206D030228DF80420C7
:10F420008DF8050002229046009B83F0080353EA02
:10F430000A030AD15CEA010201D1620705D5302234
:10F440008DF804204FF001087F1E582804D034A006
:10F4500003900EA802900DE036A0F9E753466046EF
:10F46000009AF9F7CBF984460398825C0298401E13
:10F47000029002705CEA0100F0D1029806A9081A15
:10F4800000F1200A600702D524F4803400E001274F
:10F49000574502DDA7EB0A0000E0002000EB0A015F
:10F4A000009005984144401A0590E00306D45B465D
:10F4B0002146179A059800F0B3F90544002706E0A5
:10F4C00001A85A46C05D179990476D1C7F1C47459F
:10F4D000F6DBE0030CD55B462146179A059800F051
:10F4E0009FF9054404E030205A46179990476D1C57
:10F4F0000099481E00900029F5DC08E00298029966
:10F500005A460078491C0291179990476D1CBAF130
:10F510000001AAF1010AF1DC65E1000009280100FF
:10F520003031323334353637383961626364656679
:10F53000000000003031323334353637383941423B
:10F54000434445460000000000F058F90544761C8D
:10F55000307800287FF4ECAD19B02846BDE8F08F74
:10F56000620700D4062709F1070222F0070CFCE825
:10F570000223E14603F000485FEA080C02D00FF2D4
:10F58000702C0DE05FEA045C02D50FF2682C07E0F6
:10F590005FEAC47C02D00FF2602C01E0AFF2700C85
:10F5A0004FF0FF3823F00043CDF850C065280CD051
:10F5B00006DC452809D046281DD047283DD13DE02E
:10F5C000662818D067287ED138E00021112F01DB92
:10F5D000112000E0781CCDE9000106A90EA8FFF774
:10F5E000DDFCDDE90F010E9A03910021009207F185
:10F5F000010A04914DE04FF000400097CDE9011061
:10F6000006A90EA8FFF7CAFCDDE90F0203920E9BC4
:10F6100011990022DDF80CA00093049211B9791C15
:10F6200000EB010AB7EB0A0004D4C0F1FF3007F188
:10F63000010A0490AAEB0700019044E0012F00DAD0
:10F6400001270021112F01DD112000E03846CDE90E
:10F65000000106A90EA8FFF7A1FCDDE90F010E9A33
:10F660000391002104910092BA4621070CD403991A
:10F67000514500DA8A46BAF1010F05DD009AAAF178
:10F680000101515C302908D0B84202DA10F1040FB0
:10F6900006DA0121CDE9011015E0AAF10101E9E73F
:10F6A000002805DC049901440491AAEB000102E062
:10F6B000411C514500DD8A460499401A401C0190C6
:10F6C0004FF000400290200704D40198504501DB20
:10F6D000CDF8048000208DF84F0002980DF14F07FF
:10F6E000B0F1004F25D02B200E9002984FF0020869
:10F6F00000280CDA404202902D200E9007E00A21EB
:10F700000298F9F765F83031029007F8011DB8F159
:10F710000001A8F10108F2DC02980028EFD1791E5F
:10F720000E980870307800F0200040F0450007F88F
:10F73000020D12A8C01B00F107081498007800B150
:10F74000012000EB0A01019801EBE07105984144AA
:10F75000401A401E0590E00306D45B462146179AE6
:10F76000059800F05DF805441498007818B15A46E1
:10F77000179990476D1CE00324D55B462146179AE4
:10F78000059800F04DF805441CE00498002807DBBC
:10F79000DDE90301884203DD0098405C179901E030
:10F7A000179930205A469047049805F10105401CEE
:10F7B00004900198401E019004D12E205A461799BA
:10F7C00090476D1CBAF10001AAF1010ADDDC05E0E9
:10F7D00017F8010B5A46179990476D1CB8F10001B4
:10F7E000A8F10108F4DC5B462146179A0598ABE6C0
:10F7F0002D0000002B000000200000002DE9F0414A
:10F80000044600251E461746880404D405E0394600
:10F810002020B0476D1C641EF9D52846BDE8F08154
:10F820002DE9F041044600251E469046C80301D547
:10F83000302700E02027880404D505E041463846FB
:10F84000B0476D1C641EF9D52846BDE8F0810A68F2
:10F85000531C0B601070704710B5044602F0E4FAB8
:10F8600000B110BD074808490968445406480068BB
:10F87000401C052190FBF1F201FB120002490860D7
:10F8800000BFEEE77C0800207808002010B58CB09F
:10F8900001F01AFA26E09DF80C3004AA07A8069990
:10F8A000FAF793FA00208DF82F00012025490870FF
:10F8B0000B98009007A80FC800F0E6F901280FD1B7
:10F8C000142207A92048F8F75FFC1E480021CDE963
:10F8D00001101D48006900901B480FC800F070F926
:10F8E000FCF7C4FC1948406840B1184803AB04AAAF
:10F8F00006A944680020A0470128CCD011E09DF85B
:10F900000C3004AA07A80699FAF75FFA00208DF8D0
:10F910002F000B98009007A80FC800F029F9FCF7FA
:10F92000A5FC0A48C06940B1084803AB04AA06A96F
:10F93000C4690120A0470128E1D001F09DF80CB076
:10F9400010BD0000E80100207414002024140020E1
:10F9500010B520211A48F8F730FC30211948F8F783
:10F960002CFC01F0ABF9FCF7E7FCFCF711FD154AA4
:10F9700015490020FCF78AFD10B114A0FFF7DAFA50
:10F98000104A183217490120FCF780FD10B116A06B
:10F99000FFF7D0FA0B48C06830B10A4800231A4676
:10F9A0001946C4681846A0470648406A30B1054861
:10F9B00000231A461946446A0120A04710BD0000E2
:10F9C0005414002024140020B001002063616E3123
:10F9D00020D0ADD2E9B3F5CABCBBAFB3C9B9A60D4F
:10F9E0000A0000007C01002063616E3220D0ADD29D
:10F9F000E9B3F5CABCBBAFB3C9B9A60D0A00000094
:10FA000010B5A2B0002441F20B000D49A1F8050089
:10FA100000BF01E0601C84B2282CFBDB50200849A9
:10FA200048800848007C401C0649087406A0FFF77F
:10FA300081FA01AA02A90248FBF7C8FB22B010BD57
:10FA40007E1D0020041F002053656E642063656CDA
:10FA50006C2074656D70200A0D00000010B5A2B016
:10FA6000002441F20C001049A1F8050000BF06E097
:10FA70000E48015D0C48C01D0155601C84B2082C65
:10FA8000F6DB0820084948800948007C401C0849EA
:10FA9000087408A0FFF74EFA01AA02A90248FBF772
:10FAA00095FB22B010BD00007E1D0020CD2100205E
:10FAB000041F002073656E6420626D735F73746150
:10FAC00074655F696E666F0A0D00000010B5A2B024
:10FAD000002441F20A001149A1F8050000BF09E025
:10FAE00004EB44010E48084481780C48C01D0155C0
:10FAF000601C84B2282CF3DB282008494880094880
:10FB0000007C401C0749087407A0FFF713FA01AAFC
:10FB100002A90248FBF75AFB22B010BD7E1D00204F
:10FB200055210020041F002053656E642063656C1E
:10FB30006C2074656D70200A0D00000070B50546DC
:10FB4000002400BF0FE0094951F8341028688842AA
:10FB500007D1064800EBC4004168284688470020CA
:10FB60002860601C44B20C2CEDD370BD0806002048
:10FB70000FB410B5142202A90D48F8F705FB0C4884
:10FB80000468142201460B48F8F7FEFA80210A485F
:10FB9000FBF7DDFE09480168054888471421044841
:10FBA000F8F70BFB00200249086010BC5DF814FB5D
:10FBB000A80E00206C0E002000100140040600205A
:10FBC0000FB470B5DDE9095429484078142810DADB
:10FBD0002749497801EB81022549091D01EB820083
:10FBE000142204A9F8F7D0FA21484078401C204993
:10FBF000487005986FF30F001E49884218D19DF890
:10FC00001B00102803D09DF81B00132804D19DF879
:10FC10001E001949087007E09DF81B00112803D148
:10FC20009DF81C00144908700A201449086015E06A
:10FC300005986FF30F00124988420FD19DF81B0001
:10FC40000D490978884206D114200C49086000202B
:10FC50000949087002E0322008490860002109487B
:10FC6000FEF76AF90020207070BC5DF814FB0000FC
:10FC7000A00C00200000EC1C08010020F000002077
:10FC80000000EB1CEC0000200FB410B5142202A9F8
:10FC90003848F8F779FA37484068374908603548F6
:10FCA000808880B24FF25641884204D04FF0FF3036
:10FCB00010BC5DF814FB2F4840686FF30F002F490C
:10FCC000884207D114222B492D48F8F75DFA4FF0EE
:10FCD000FF30EDE7274840686FF30F00294988425D
:10FCE00007D1142223492648F8F74EFA4FF0FF3087
:10FCF000DEE721480068244988422CD01E4800686D
:10FD00002249884227D01C4800682149884222D0D5
:10FD1000194800681F4988421DD0174800681E49CD
:10FD2000884218D0144800681C49884213D01248F1
:10FD300000681B4988420ED00F4800681949884264
:10FD400009D00D4800681849884204D00A48006864
:10FD5000164988420BD1142206491548F8F714FABF
:10FD600004498A7A002348680B3100F0F1FB002037
:10FD70009EE70000940E0020040100200000EC1C0F
:10FD8000500C00200000EB1C56F4261856F4011805
:10FD900056F4071856F4081856F40A1056F41218B8
:10FDA00056F41D1856F41F0856F41A1056F41A1873
:10FDB0008C0C002070B5002015490860154848607B
:10FDC000042008720020487205208872FF22082152
:10FDD0000F480B30F8F7EAF90F48B0F84140B0F897
:10FDE0004300C0F57A6085B20949CC72210A0848FF
:10FDF00001734573290A8173074890F8450008B1DB
:10FE0000022100E001210248C17301F079F870BDC0
:10FE1000640C0020F4561018A007002070B50446AA
:10FE2000012C25D100204B4908604B484860042034
:10FE300008720020487208208872FF220821454875
:10FE40000B30F8F7B3F910204249C8720D21414830
:10FE500001730021417302218173FF21C1730021CD
:10FE60000174062141740021817401F049F870E0A9
:10FE7000022C6ED1002037490860384848600420C1
:10FE800008720020487208208872FF220821314839
:10FE90000B30F8F78BF901202E49C872304890F8E2
:10FEA00033102C4801732E48B0F83300010A29485A
:10FEB00041732B48B0F83500C0F57A60C1B22548CF
:10FEC00081732748B0F83500C0F57A60010A2148EF
:10FED000C173234890F837101E4801742048B0F8C9
:10FEE0003700010A1B4841741D4890F83910194821
:10FEF000817401F005F80320FBF7C9F902201549C8
:10FF0000C8721748B0F83900010A12480173144842
:10FF100090F83B000A30C1B20E4841731048808F00
:10FF200000EB80004FF6FF7101EA40050948857338
:10FF3000290AC1730A4890F83E100648017408481F
:10FF4000C08F010A034841740021817400F0D8FF7A
:10FF500000BF70BD640C0020F456EC1CF456EB1C82
:10FF6000A007002010B50446012C25D100204549EA
:10FF70000860454848600420087200204872082044
:10FF80008872FF2208213F480B30F8F70FF9102044
:10FF90003C49C87209213B48017300214173022189
:10FFA0008173FF21C173002101741121417400216B
:10FFB000817400F0A5FF64E0022C62D10020314979
:10FFC0000860324848600420087200204872082007
:10FFD0008872FF2208212B480B30F8F7E7F8012040
:10FFE0002849C8722A4890F84610264801732848C4
:10FFF000B0F84600010A234841732548B0F848008C
:020000040801F1
:10000000C0F57A60C1B21F4881732148B0F848003A
:10001000C0F57A60010A1B48C1731D4890F84A1068
:10002000184801741A48B0F84A00010A154841748A
:10003000174890F866101348817400F061FF0320A0
:10004000FBF725F9124890F86600C0F1640081B210
:100050000F48A0F84D1002200A49C8720C4890F8C9
:100060004D10084801730A48B0F84D00010A0548D0
:10007000417300218173C17301744174817400F074
:100080003FFF10BD640C0020F456EC1CF456EB1C32
:10009000A007002010B5044600200C4908600C4859
:1000A0004860042008720020487202208872FF22F3
:1000B000082106480B30F8F779F80449CC72210A78
:1000C0000248017300F01CFF10BD0000640C00200A
:1000D000F456271810B586B00446142101A8F8F785
:1000E0006CF8012C25D100209249086092484860A4
:1000F000042008720020487208208872FF2208211C
:100100008C480B30F8F752F810208A49C872312118
:10011000884801730021417307218173FF21C17356
:1001200000210174022141740021817400F0E8FE75
:10013000FEE0022CFCD100207E4908607F48486028
:10014000042008720020487208208872FF220821CB
:1001500078480B30F8F72AF801207649C87200BFBA
:1001600077488078087300BF7548C078487300BF2F
:1001700073480079887300BF71484079C87300BF25
:100180006F488079C1B26B48017400BF6C48C08869
:10019000010A6848417400BF6948007AC1B26548E5
:1001A000817400F0ADFE0320FBF771F80220614975
:1001B000C87200BF62480089010A5E480173604846
:1001C000817A5C4841735E48C17A5A4881735C48C1
:1001D000017B5848C1735A48417B5648017400213D
:1001E0004174817400F08CFE0320FBF750F803206B
:1001F0005049C87201214F48017302214173504890
:10020000817C4C4881734E48C17C4A48C1734C483C
:10021000017D484801744A48417D46484174484838
:10022000817D4448817400F06BFE0320FBF72FF8BA
:100230000020444981F88701084690F88701012889
:1002400006D112223E491A3101A8F7F79DFF04E0BA
:10025000FF22112101A8F7F7A9FF04203549C87230
:100260003748C17D334801733548017E31484173B9
:10027000002181739DF80410C1739DF8051001746D
:100280009DF8061041749DF80710817400F038FE47
:100290000320FAF7FCFF05202649C8729DF80810D4
:1002A000244801739DF8091041739DF80A10817369
:1002B0009DF80B10C1739DF80C1001749DF80D1082
:1002C00041749DF80E10817400F01AFE0320FAF7B5
:1002D000DEFF06201749C8729DF80F1015480173FC
:1002E0009DF8101041739DF8111081739DF8121044
:1002F000C1739DF8131001749DF8141041741021FE
:10030000817400F0FDFD0320FAF7C1FF07200949C1
:10031000C8720A21074801730B21417307218173B9
:10032000E021C173FF2101744174817400F0E8FD84
:1003300006B010BD640C0020F456EC1CF456EB1C07
:10034000A00700209814002010B5044600200A4998
:1003500008600A48486004200872002048720120A2
:100360008872FF22082104480B30F7F71FFF02486C
:10037000C47200F0C5FD10BD640C0020F4560910D5
:1003800010B504460020154908601548486004204F
:1003900008720020487207208872FF2208210F4847
:1003A0000B30F7F703FF4B200E4908804A200E4917
:1003B00008800E4890F866000849C8724C2107482A
:1003C000017304214173B02181730421C17364213D
:1003D00001746521417400F093FD10BD640C002090
:1003E000F4561C18180100201A010020A007002054
:1003F0002DE9F04781460024002500260027A0466D
:10040000002029490860294848600420087200201B
:10041000487207208872FF22082123480B30F7F723
:10042000C5FE234890F89701012806D105244B25E5
:1004300004264A274FF0030805E005244B2504262F
:100440004A274FF0030800BF1A4890F84F0016499A
:10045000C87200BF174890F850000A30C1B2124865
:10046000017300BF134890F851000F49487300BF53
:10047000104890F852000A30C1B20B48817300BF97
:100480000C4890F853000849C873002106480174CD
:1004900000BF084890F85A000007010E0248417456
:1004A00000F02EFDBDE8F087640C0020F456131810
:1004B00098140020A00700202DE9F04107460024F1
:1004C0000025002600201E4908601E4848600420C0
:1004D00008720020487204208872FF220821184800
:1004E0000B30F7F763FE184890F86600642802D1D5
:1004F00044F0010400E000BF144800781E2802D137
:1005000044F0100400E000BF2620FAF70BFF10B102
:1005100044F0400400E000BF0C480078182802D1E5
:1005200045F4806500E000BF00BF0548C472057354
:10053000290A4173867300F0E3FCBDE8F0810000F6
:10054000640C0020F4561910A00700200C020020B3
:100550002DE9F04105460E46174698460024FAF765
:100560002DFC5649681A8D424CD015DC5449A5EB38
:1005700001008D4273D008DC5248284400286CD01A
:1005800051490844002869D14AE050490844E8B17B
:10059000B0F5C02FF7D127E0B0F5202F4ED0B0F541
:1005A000901F5DD0B0F5A81F68D0B0F5F01FEAD15C
:1005B000424639463046FAF743FA04462CB14448DD
:1005C000806B40F480404249886374E0424639467B
:1005D0003046FAF779FA04462CB13D48806B40F07A
:1005E00001003B49886366E0424639463046FAF7E7
:1005F000BBFA04462CB13648806B40F00200344907
:10060000886358E0424639463046FAF729FA0446EC
:100610002CB12F48806B40F004002D4988634AE0DC
:10062000424639463046FAF76DFA04462CB128485E
:10063000806B40F00800264988633CE0424639461A
:100640003046FAF7ABF904462CB12148806B40F0F4
:1006500010001F4988632EE001E01DE02AE000BF82
:10066000424639463046FAF76BFA04462CB1184830
:10067000806B40F02000164988631CE042463946F2
:100680003046FAF749FA04462CB11148806B40F025
:1006900040000F4988630EE0424639463046FAF77B
:1006A000BBF904462CB10A48806B40F08000084931
:1006B000886300E000BF00BFBDE8F08156F4081871
:1006C00056F41A10AA0BE0F7000015F8000019F80C
:1006D000C00B0020F0B5034698180F4FB84201D95F
:1006E0000320F0BD0AB90020FBE7012600240BE03F
:1006F0001D780878A84204D0FF2D01D00220F0E731
:1007000000265B1C491C641C9442F1D3012E01D1CC
:100710000020E6E70120E4E700000208014600208F
:10072000C80AC002704700002DE9F84F06460F4680
:1007300014464FF0040B30192A49884202D901208F
:10074000BDE8F88F0CB90020FAE704F0010000B111
:10075000641C224639463046FFF7BCFF8046B8F19C
:10076000000F01D10020EBE7012080F3108800BFCB
:10077000FAF7E2FE3520FAF735FE3046FFF7CEFFF6
:100780000090FAF735FE83464FF47A7A00BFBAF14B
:100790000000AAF101011FFA81FAF8D1002511E049
:1007A00017F815906800401C385C49EA0029494652
:1007B0003046FAF767FE8346BBF1040F00D004E031
:1007C000B61C6D1CB5EB540FEAD300BFFAF750FE10
:1007D000002080F3108800BFBBF1040F00D1AFE709
:1007E0000220ADE70000020810B504463CB9002124
:1007F0000748F9F7AFFE0648F9F7A4FA06E000212A
:100800000448F9F7A7FE0348F9F79CFA012010BD48
:10081000006400400068004070B505460C46022D9B
:1008200000DB70BD05EB85000D4901EB8000006920
:1008300088B1A37A207A042801D1606800E020689A
:10084000014605EB8500064A02EB800004F10B022D
:1008500006692846B047284600F0DCF900BFE0E70B
:10086000BC0E002070B505460E460DB9064900E0E5
:10087000064908463146F9F751FF0446042C00D1D9
:10088000FF24204670BD0000006400400068004066
:1008900070B504460D461646022C00DB70BD04EB15
:1008A000C400144901EB8000C0680121A940084040
:1008B000F0B104EBC4000F4901EB8000C0680121D6
:1008C000A940884304EBC4010A4A02EB8101C860D5
:1008D000204600F09FF904EB8400074951F82000FE
:1008E00030B104EB840051F820202946204690477F
:1008F00000BFD3E7E40E0020BC0E002070B5044614
:100900000D4614B9F9F76AFD01E0F9F775F8012011
:1009100070BD000010B50446832C00D010BD0A48FD
:10092000007C01280ED00948C06A18B10748C16A86
:10093000012088470120044908740021024814302E
:10094000FDF7FAFA00BFE9E7541400202414002050
:100950002DE9F04105460E4626BB2F4600240FE048
:10096000124800EB04100068B84207D10F4901EBB0
:10097000041101F10C000021FDF7DEFA601C84B2C5
:10098000022CEDD300BF0A48807F00280BDD084809
:10099000007C022807D10021054881771830FDF737
:1009A000CBFA00E000BFBDE8F08100005C01002050
:1009B0005414002010B50446002004EBC401044A7E
:1009C00002EB810188602046FFF70EFF10BD00009A
:1009D000E40E002010B50446022C00DB10BD04EB31
:1009E00084000D4901EB8000806890B104EBC400E5
:1009F0000A4B03EB8000C06808B1012000E0002032
:100A0000014604EB8400044B03EB8000826820461F
:100A1000904700BFE2E70000BC0E0020E40E00207B
:100A200010B50446022C00DB10BDFCF732FF04EBCE
:100A300084000F4901EB8000C06838B104EB8400EA
:100A40000A4602EB8000C16820468847FCF723FF76
:100A500004EBC400074901EB8000C06830B10020FE
:100A600004EBC401034A02EB8101C86000BFDBE76D
:100A7000BC0E0020E40E00207CB500200090019008
:100A800000246CE0374800EB0410007801284CD1BA
:100A9000344800EB04108089062807D2314800EB67
:100AA00004108089304931F8105001E02E48458902
:100AB0002C4901EB0411081D2946FDF73DFA0028D9
:100AC0004BD0FCF7E6FE274800EB04108089401C61
:100AD000244901EB0411888104EB4400234901EB14
:100AE000C000C06848B104EB440001EBC000002323
:100AF0001A461946C6682046B0470220194901EB3C
:100B00000411087001208DF80000FCF7C4FE15499F
:100B100001EB041101F108000021FDF70DFA01209D
:100B2000104901EB0411887317E00E4800EB041024
:100B30000078022811D10B4901EB041101F10800E2
:100B40006721FDF7F9F940B10020064901EB0411D6
:100B50008881044901EB04110870601CC4B2022CA6
:100B600090DB7CBD54140020745001082414002034
:100B70002DE9F04104460D4616461F46022C02DBC5
:100B80000020BDE8F081012004EBC401204A02EB03
:100B900081018860002004EBC40102EB81014871EF
:100BA00004EBC400114601EB8000077104EBC400A4
:100BB00001EB8000C67004EBC40021F82050002037
:100BC00004EBC40102EB8101C86004EBC40002EB3A
:100BD00080012046FFF792FE38B1022004EBC401E9
:100BE0000B4A02EB8101886006E0002004EBC4019F
:100BF000074A02EB8101886004EBC400044901EB61
:100C000080008068022801D10120BAE70020B8E7FF
:100C1000E40E0020022800DB704700BFFCE7000064
:100C20002DE9F04104460E4617469846022C07DA95
:100C300004EBC400194901EB80008068022802D04F
:100C40000020BDE8F08104EBC401144A02EB8101ED
:100C500001F1100043463A463146F9F78FF804EBAC
:100C6000C4000E4A02EB800000F110012046FFF79D
:100C7000F9FD0546FF2D0ED004EBC400074901EB3A
:100C80008000C1680120A840014304EBC400034A6E
:100C900002EB8000C1602846D3E70000E40E00208C
:100CA000FEB504460D461646009401950296694627
:100CB000014803F05EFDFEBDAC11002010B500F050
:100CC000A9F800F047F810BD10B500F055F800F095
:100CD000ABF810BD10B502460B4612B94FF0FF300D
:100CE00010BD002114E01A4850F8310090420ED196
:100CF000174800EBC1004360154800EBC100406895
:100D000018B90020124C44F831000020E8E7491CD3
:100D10001429E8D313B94FF0FF30E1E7002111E0C7
:100D20000B4850F8310020B1094800EBC100406881
:100D300038B9074840F8312000EBC100436000207B
:100D4000CEE7491C1429EBD34FF0FF30C8E7000071
:100D50002C0F002010B54FF426710648F7F72DFA36
:100D600028230C220349A03101F5F07003F0D6FCD2
:100D7000002010BD2C0F00203EB518E069460F483A
:100D800003F0DAFC00240FE00D4850F8340000991D
:100D9000884208D10A4800EBC400456815B19DE8B7
:100DA0000700A84702E0641C142CEDD300BF0348E1
:100DB00003F0A2FC0028E1D000203EBDAC110020D1
:100DC0002C0F002010B502460AB9002010BD0021EA
:100DD00019E001EB41000E4B03EB8000806880B905
:100DE00001EB410003EB80008260002001EB410336
:100DF000074C44F8230001EB4100234603EB80003D
:100E0000E4E7481C81B21429E3D30020DEE70000A8
:100E1000C411002010B5F0210248F7F7CEF90020E8
:100E200010BD0000C4110020F8B50027002168465D
:100E3000FDF782F80098B84203D0781C00998142EF
:100E400001D10020F8BD009F00243BE004EB4400EA
:100E50001E4901EB8000866804EB440051F82050E5
:100E60007DB376B304EB4401184A02EB8101081DFF
:100E70002946FDF761F8012823D104EB440013490A
:100E800001EB80008068A8B104EB440001EB800016
:100E900040680099081AB0FBF5F004EB44010B4AD6
:100EA00002EB8101496800FB051004EB440102EBF1
:100EB000810148602EB104EB4401044A02EB810039
:100EC000B047641C142CC1D30020BBE7C411002020
:100ED00070B504460E46254605B970BD2E6000214A
:100EE000281DFDF729F800BFF7E701460A460AB9B1
:100EF00000207047106808B10120FAE70020F8E7E9
:100F00007CB50446002611480068E0B10021207A33
:100F1000042801D1606800E02068CDE90001607A12
:100F200008B9A07A00E000200346207A042801D105
:100F3000606800E020680146044804F10B0205687F
:100F40000020A8477CBD0020FCE7000024140020FE
:100F50007CB50446002612488069F0B10021207A51
:100F6000042801D1606800E02068CDE90001607AC2
:100F700008B9A07A00E000200346207A042801D1B5
:100F8000606800E020680146054804F10B028569AD
:100F90000120A84708B100207CBD0020FCE700002C
:100FA0002414002010B50C48008850B901200A49CB
:100FB000088000BF0948FBF7D3FB09A0FDF7BAFF83
:100FC00009E000200449088000BF0448FBF7F3FB58
:100FD00009A0FDF7AFFF10BD50050020080A002052
:100FE000B9D8B1D54143BDBBC1F7CEC2B6C8BCCCA0
:100FF000B5E7C6F70D0A0000BFAAC6F44143BDBB62
:10100000C1F7CEC2B6C8BCCCB5E7C6F70D0A000022
:1010100010B50A48008840B9012008490880F9F74E
:101020007FFF07A0FDF786FF07E000200349088047
:10103000FBF7DAFC07A0FDF77DFF10BD4805002097
:10104000B9D8B1D5BDBBC1F7BCCCB5E7C6F70D0A61
:1010500000000000BFAAC6F4BDBBC1F7BCCCB5E719
:10106000C6F70D0A000000007047000010B50F48D9
:10107000008868B901200D49088000BF00200C4994
:1010800088700C48FBF76CFB0BA0FDF753FF0CE0DE
:1010900000200649088000BF0120054988700548E6
:1010A000FBF789FB07A0FDF745FF10BD4C050020AD
:1010B00068060020CC090020B9D8B1D5434331439C
:1010C000500D0A00BFAAC6F443433143500D0A0035
:1010D00010B50F48008868B901200D49088000BF8D
:1010E00000200C49C8700C48FBF73AFB0BA0FDF739
:1010F00021FF0CE000200649088000BF01200549BF
:10110000C8700548FBF757FB08A0FDF713FF10BD9B
:101110004E05002068060020F4090020B9D8B1D59A
:101120004343325F43430D0A00000000BFAAC6F4E8
:101130004343325F43430D0A00000000FBF71CFCF1
:1011400010B50F48008868B901200D49088000BF1C
:1011500000200C4948700C48FBF72DFB0BA0FDF755
:10116000E9FE0CE000200649088000BF0120054987
:1011700048700548FBF7F4FA09A0FDF7DBFE10BD47
:101180004605002068060020A4090020B9D8B1D582
:10119000D6B1C1F7BCCCB5E7C6F70D0A0000000018
:1011A000BFAAC6F4D6B1C1F7BCCCB5E7C6F70D0AE5
:1011B00000000000704770477047000010B50C48F1
:1011C000008850B901200A49088000BF0948FBF790
:1011D000C7FA09A0FDF7AEFE09E000200449088027
:1011E00000BF0448FBF7E7FA07A0FDF7A3FE10BD18
:1011F0004A050020E0090020B9D8B1D5C9FDD1B910
:10120000C4A3BFE90D0A0000BFAAC6F4C9FDD1B945
:10121000C4A3BFE90D0A0000704770477047000083
:1012200010B51048008870B901200E49088000BF31
:101230000D48FBF795FA00BF0C48FBF791FA0CA09C
:10124000FDF778FE0DE000200649088000BF064843
:10125000FBF7B1FA00BF0548FBF7ADFA08A0FDF7B0
:1012600069FE10BD44050020E0090020B8090020F7
:10127000B9D8B1D5B8DFD1B9C4A3BFE90D0A000010
:10128000BFAAC6F4B8DFD1B9C4A3BFE90D0A0000F4
:101290002DE9F04705460E460D20FCF727FF0A20F2
:1012A000FCF724FF2C46002710E02078FAF711FE07
:1012B00080462078FAF700FE81464046FCF716FF8C
:1012C0004846FCF713FF641C781C87B2B742ECDB7E
:1012D0000D20FCF70BFF0A20FCF708FFBDE8F087A4
:1012E0000022002107E042F6E06200E0521E002AE0
:1012F000FCD14B1C99B28142F5DB704770B50446B6
:101300000D46E1B21948FDF716FA00BF17480088EC
:1013100000F080000028F9D0154890F8A8000128B6
:1013200022D11448807802281AD1134800789628D0
:1013300008DA114802780078401C0F4B18700F48EB
:10134000845411E00C4801780C48FDF7D1FC0948A1
:10135000007C401C0749087400200749087003E01E
:101360000020034981F8A800204670BD004C0040D1
:1013700098140020041F00203A050020D5210020E9
:1013800010B5002821D0114B0022001F196803E07E
:10139000814203D80A4649680029F9D152B113683D
:1013A000841A9C4204D1006818441060104602E080
:1013B000506000E0186039B102680B1A934203D103
:1013C0000B681A4402604968416010BD0C0B002094
:1013D00010B50D4A906E926ED16A884704468CB95A
:1013E0004FF4FA610948FCF7A7FD01280AD1084823
:1013F000C07B401C0649C87300210448FCF79CFDD3
:10140000012010BD0020FCE7A00700208023002061
:101410008823002010B5184890F8380000F001002B
:1014200040B116484079012804D115A0FDF782FD8E
:10143000012010BD104890F8380000F0010038B1CC
:1014400002200E49487114A0FDF774FD0120F0E759
:10145000174908698047022801D00220E9E70A21DC
:101460001448FCF75BFA20B11248FCF76AFA022034
:10147000DFE70020DDE70000C00B00204423002050
:10148000424D535F50524F544F43414C5F4742329D
:101490003031350A0D000000424D535F50524F5419
:1014A0004F43414C5F4742323031310A0D0000005A
:1014B0006C000020DC33002010B515490869804716
:1014C0000446022C16D1134A906E926ED169884759
:1014D00004281AD100201049C8733C210F48F6F7A0
:1014E0006CFE40210E48F6F768FE0EA0FDF722FDC7
:1014F000012010BD012C08D140210948F6F75DFEFE
:101500000DA0FDF717FD0220F3E70020F1E7000032
:101510006C000020A007002088230020C00B0020C2
:10152000D4330020BDF8C8EBD6B1C1F7B3E4B5E7BA
:10153000C1F7B3CC0D0A0000BDF8C8EBBDBBC1F7C5
:10154000B3E4B5E7C1F7B3CC0D0A000010B5094804
:10155000008F00F4804018B1F9F7A6FE012010BDFD
:10156000054908698047022801D00220F7E70020DA
:10157000F5E70000C00B00206C00002010B50D48FE
:10158000C078AA2804D10CA0FDF7D4FC012010BD1E
:10159000FCF742F820B90FA0FDF7CCFC0220F6E7DB
:1015A0001A4908698047022801D00320EFE700208C
:1015B000EDE70000C00B002052455620445F434435
:1015C0005A5F48414E44494E475F43524D20414186
:1015D0000A0D000052656164792D537461746520B1
:1015E0005265636569766564205468652043686167
:1015F0007267696E672050696C652041626F727412
:10160000204D6573736167650A0D00006C00002052
:1016100010B5FCF701F820B909A0FDF78BFC0320F9
:1016200010BDFCF7D7FA08B90120F9E7134908699A
:101630008047022801D00320F2E70020F0E70000F5
:1016400052756E6E696E672D5374617465205265B4
:1016500063656976656420546865204368617267D4
:10166000696E672050696C652041626F7274204D0D
:101670006573736167650A0D000000006C0000204F
:1016800010B5FBF7C9FF20B924A0FDF753FC0220D9
:1016900010BD2820F9F746FE98B90620F9F742FE5A
:1016A00078B91C20F9F73EFE58B92120F9F73AFE27
:1016B00038B90920F9F736FE18B90A20F9F732FED1
:1016C00008B10320E4E7234908698047022801D0D4
:1016D0000520DDE70A212048FCF720F938B1FDF7A5
:1016E00023FB20B91C48FCF72CF90320D0E71B484A
:1016F000807EAA2804D11AA0FDF71CFC0120C7E7B0
:101700003C2115480838FCF709F928B11248083877
:10171000FCF717F90520BBE70020B9E753746172A5
:10172000742D5374617465205265636569766564D0
:1017300020546865204368617267696E672050694C
:101740006C652041626F7274204D657373616765CB
:101750000A0D00006C000020FC330020C00B0020AC
:1017600043445A5F5F43524F20414120746F2043EE
:1017700068617267696E670A0D00000010B50A2182
:101780000548FCF7CBF820B10348FCF7DAF8012054
:1017900010BD0020FCE700000434002070B50446B2
:1017A0000D46002629462046F7F738FA0520FFF7B0
:1017B00097FDFBF7EFFF0646304670BD0146072058
:1017C00070477047014602207047000010B512486C
:1017D000008F00F4804078B100200F498863012019
:1017E0000E49487100BF0E4800880446FEF752FCBF
:1017F0000CA0FDF79FFB0EE040F6B831074808301B
:10180000FCF79AFB38B10CA0FDF794FB00210348CC
:101810000830FCF791FB10BDC00B002044230020D2
:10182000A0070020445F43445A5F48414E44494E5C
:10183000475F43484D0D0A004E4F2048616E647368
:1018400068616B65205369676E616C0A0D0000006A
:1018500001460020704770470146012070477047DD
:10186000014603207047000010B50B48007920B1F5
:10187000012807D002280DD108E002210748F9F716
:1018800015FF07E00548F9F743FF03E00220F9F7E9
:101890004FFF00BF00BF10BD44230020D50001084A
:1018A00001460520704710B5F9F79CFB10BD0146B5
:1018B0000420704770B53548007920B1012807D061
:1018C00002280DD108E006213148F9F7EFFE07E0C4
:1018D0002F48F9F71DFF03E00620F9F729FF00BFA5
:1018E00000BF002605212B48FCF718F888B1F9F74E
:1018F00077FB70B1F7F7F4FA58B1FCF729F840B16B
:10190000254A906E926E516A8847012801D1AA2615
:1019100000E0002635462C46204890F8380000F0BC
:10192000020030B11D48806B20F002001B49886323
:101930002AE01A4890F8380000F00400A8B114B961
:10194000F9F70AFB07E000BF012015494870154868
:10195000FAF706FF00BF2046FEF7F6FC0F48806B43
:1019600020F004000D4988630EE00C4890F8380020
:1019700000F0080040B10CA0FDF7DCFA0748806BCE
:1019800020F008000549886370BD00004423002052
:101990001DFE0008EC330020A0070020C00B002033
:1019A00068060020A409002043445A5F48414E4481
:1019B000494E475F43524D2041410A0D000000004F
:1019C000014606207047000010B500200F494871FD
:1019D00032210F48FCF7B0FA012806D10020FEF7AB
:1019E0006BFD00210A48FCF7A7FAFA2108481030DD
:1019F000FCF7A2FA012807D10020FEF7C1FC002164
:101A000003481030FCF798FA10BD00004423002072
:101A10006C23002070B505460E463046F9F7D6FF18
:101A2000044604B970BD812D26D004DC042D07D0F6
:101A3000802D4DD116E0822D0AD0832D48D128E08B
:101A400094F85400032802DB2046FAF750FA40E0ED
:101A500094F85400032804DBE06C10B18220E16CA0
:101A6000884736E094F85400032804DBE06C10B19A
:101A70008020E16C88472CE094F85400032807DBB1
:101A80002046FAF7D4FAE06C10B18120E16C884767
:101A90001FE094F85400032819DB9120005D022810
:101AA00006D104219120015522780120FFF7F8F892
:101AB000E06C18B18320E16C884708E0207800F0E2
:101AC00009FB207800231A46194600F075FB00E058
:101AD00000BF00BF00BFA5E770B506460D46304603
:101AE000F9F774FF04461CB394F85400022805DC8F
:101AF000E068E8B13046E168884719E094F854009E
:101B0000812808D13DB184F854003246812101205A
:101B1000FFF7C6F80CE094F85400812808D03DB9CE
:101B2000802084F85400324680210120FFF7B8F865
:101B300070BD70B504460D4629462046FFF7CCFF20
:101B400070BD70B505462846F9F740FF04468CB1D4
:101B500094F85400022805DCE06858B12846E16892
:101B6000884707E0832084F854002A468321012017
:101B7000FFF796F870BD00002DE9F04107460D46CD
:101B800090461E463846F9F721FF0446002C39D00E
:101B900094F85400032835DB94F85400802802D1CF
:101BA000032084F8540094F8400000F0010038B19C
:101BB000A06C38B3324641462846A36C984721E0D2
:101BC0001248056006710079002809DD0F48007988
:101BD000082805DC0D4802794146401DF6F7D4FA85
:101BE0000A4904F1580002F0C4FD04F1580002F063
:101BF0008CFD38B1822084F854003A4682210120BD
:101C0000FFF74EF80120BDE8F08100001414002019
:101C100070B506460C463046F9F7D8FE05461DB1AC
:101C2000E1B22846FAF71CFA70BD000010B5142086
:101C3000724981F8660041F288300880012088707E
:101C400001216E48C1700171032141714FF47A7115
:101C5000C18041F268010181422181725921C17222
:101C6000442101735421417300218173C173012107
:101C7000017402214174192181740B21C1740A215C
:101C800001750021417581751021C1750021017612
:101C9000417611225AA11A30F6F776FA57482B30BE
:101CA0005CA10A680260496841604FF4D2705349F0
:101CB000A1F833005A4A5B494FF66A70FDF744F8C1
:101CC0004E49A1F835004FF47A714C48A0F8351010
:101CD0004FF49B71A0F8371041F22431A0F839106D
:101CE0006E2180F83B10142181874FF47A61C187FF
:101CF0000020424981F840004FF47A60A1F8410089
:101D00004FF416713D48A0F84310022180F84510A9
:101D100000203A49A1F8460000213848A0F84810B0
:101D2000B0F84A006FF30B0000F5A2703349A1F838
:101D30004A00084690F84B0020F0F00110312F487F
:101D400080F84B103C21A0F84D1001202B4981F860
:101D50004F006FF0310233490A20FCF7F5FFC1B2A2
:101D6000264880F85010032180F851106FF031029E
:101D70002C490520FCF7E8FFC1B2204880F852103A
:101D8000042180F85310002180F8541080F8551079
:101D900080F8561080F8571080F8581080F85910C5
:101DA00080F85A100120154981F85B000021134882
:101DB000A0F85C1080F85E106420104981F85F0084
:101DC00040F259110D48A0F8601040F26311A0F8DC
:101DD00062106FF0310213491920FCF7B5FFC1B250
:101DE000064880F864106FF031020E491C20FCF7A1
:101DF000ABFFC1B2014880F8651010BDA0070020FC
:101E00004C4656324132314B364133303932333918
:101E100039000000533030314830303100000000CC
:101E200070FEFFFFCDCCCC3D07480068401C05216B
:101E300090FBF1F201FB120004490968884201D1CC
:101E4000012070470020FCE778080020740800207B
:101E500070B504460D4618480078B0B929462046AA
:101E6000FFF79CFC154909680844144908601448A8
:101E700001780078401C124A1070092902DB012009
:101E80000D4908700F48008870BD00200A4908708D
:101E90000A4800680C4908600020084908600849A1
:101EA0000870094800680A21B0FBF1F00549088074
:101EB00008460088E8E70000E1000020D800002084
:101EC000E0000020D4000020DC00002086B0FBF7FA
:101ED00017FF4FF400410803FAF744FDFBF7CEFE6D
:101EE00001A8FBF789FAFAF7F4FCFAF777FAFAF7A0
:101EF000C9F9F6F7DDFEF6F7B5FE4FF47A3002F0D9
:101F000065FC4FF4E13002F0BBFC40F2CF2140F21F
:101F1000F310FBF763FFFFF789FEFDF719FDFBF7F1
:101F2000DFFBF8F759FFF9F745FB01203D498873BE
:101F300000BF00203C49C8703C48FAF711FC00BFC4
:101F40000120394988703A48FAF735FC69E0FCF716
:101F500029F8FDF79BFC37480078012813D10020B1
:101F600034490870F6F754FFF7F7B8F932490868B2
:101F700080473149486880472F49886880472E4903
:101F8000C86880474DE02B484078012807D10020E1
:101F900028494870FBF782FCFAF768F941E02548C8
:101FA0008078012808D10020224988700220F9F7A2
:101FB00033FD2249C86034E01E48C078012803D1AF
:101FC00000201C49C8702CE01A480079012805D16E
:101FD000002018490871FAF743FC22E015484079BF
:101FE000012803D10020134948711AE01148C07933
:101FF000012816D100200F49C871F7F7D5F9FBF772
:1020000055F8FBF763FB044621460DA0FCF792FF51
:1020100000BF1148FAF7B9FB044621460FA0FCF7B0
:1020200089FF94E74423002068060020F40900207B
:10203000CC0900208814002080000020380B0020EC
:102040005254435F476574436F756E7465722069BF
:10205000732025640D0A0000E40A002048696768BF
:102060002025640D0A000000F0B50B30154D20F05E
:1020700007010024144A0FE003688B420BD38B4204
:1020800005D95E1A43184768C3E9006700E0436852
:10209000136002C004E0021D10680028ECD1204645
:1020A000002802D1286808B10020F0BD064A074880
:1020B0001060074A121A22F00702C0E9002401202A
:1020C0002860D7E7100B00200C0B002024340020E0
:1020D0002054002070B505462846F9F777FC0446E1
:1020E0001CB194F85400022801DC002070BD0220CD
:1020F00084F85400E06810B12846E16888479120D0
:10210000005D002834D0D4F8A800B0B19120005D63
:10211000052804D10021D4E92902904728E0912024
:10212000005D042804D10121D4E9290290471FE071
:102130000321D4E9290290471AE0206DC0B1912013
:10214000005D052805D10021226DD4F8A400904738
:102150000EE09120005D042805D10121226DD4F804
:10216000A400904704E00321226DD4F8A400904716
:1021700015E004F1940104F1700002F0DDFA70B191
:10218000D4F8A80020B10321D4E92902904706E041
:10219000206D20B10321226DD4F8A400904704F1F2
:1021A000700002F0A9FA0028E3D0202104F1900089
:1021B000F6F703F8012099E72DE9F04105460E46B0
:1021C000174698462846F9F701FC04461CB194F8D6
:1021D0005400012802DC0020BDE8F081606848B3AB
:1021E00043463A4631462846D4F804C0E04708B38F
:1021F000D4F88C0040B194F84530182204F17000F6
:10220000D4F88C1002F08AFA94F8400000F0010033
:1022100058B9D4F8880040B194F84530102204F140
:102220005800D4F8881002F079FA032084F854009A
:102230000120D1E70020CFE770B5054600242846ED
:10224000F9F7C4FB044614B194F8540070BD0020A3
:10225000FCE72DE9FF4180460E4615461F464046E5
:10226000F9F7B4FB04464CB194F85400022805DD9C
:1022700025B194F8400000F0010018B1002004B02E
:10228000BDE8F08104F1580002F036FA08B10020F0
:10229000F5E7694604F1580002F04EFA08B900204B
:1022A000EDE7009830609DF8040038709DF8040058
:1022B00000280ADD9DF80400082806DC9DF80420AB
:1022C0000DF105012846F5F75FFF94F854008228C8
:1022D00002D1032084F854000120D0E72DE9F04713
:1022E00086B080460F4615461E46DDE90E9A00244C
:1022F0004046F9F76BFB044654B194F854000228A9
:1023000006DD082E04DC04F1700002F0FEF918B1BD
:10231000002006B0BDE8F087FBF7BBFA94F8540044
:10232000832803D094F85400032803DAFBF7B3FAA8
:102330000020EEE7CDF814A000978DF80560CDF8E9
:10234000109015B900208DF805009DF805000028B3
:102350000ADD9DF80500082806DC9DF805202946C1
:102360000DF10600F5F710FFFF208DF80400694617
:1023700004F1700002F0FDF99120005D10B92046D3
:10238000F9F7B5FDFBF787FA0120C2E70346002005
:1023900070470000F0B54FF480541B4A0023072714
:1023A00002EA070600256E406D402E4307D0D21D7D
:1023B0006FF0070602EA0602134D551B641B114617
:1023C000124D29604FF00005104E75600A19083A49
:1023D0006FF0070602EA06020D4D2A604FF0000575
:1023E0000B4E366875600A4E366835600846151A19
:1023F0004560074D2D680560064E45683560064E00
:1024000045683560F0BD0000D4230020EC0A0020B0
:10241000F40A0020FC0A0020F80A002010B501464A
:10242000184800E0006803688B42FBD3024643680B
:1024300013448B4205D143684C68234443600146F2
:1024400000E000BF0A464B6813440468A34211D160
:102450000D4C03682468A34208D04B680468646884
:1024600023444B6003681B680B6005E0064B1B6848
:102470000B6001E003680B60884201D0016000E05E
:1024800000BF10BDEC0A0020F40A00202DE9F0473F
:1024900005464FF000093848006810B9FFF77AFF89
:1024A00000E000BF7DB105F00700C0F11008C8F1E1
:1024B000FF30A84201D2012000E0002008B94544C5
:1024C00002E0002500E000BF012000EBE5700028DD
:1024D0004CD0002D48D029480068854244D8284E69
:1024E0003046046801E0264624686068A84202D2AB
:1024F00020680028F7D120480068844232D0306834
:1025000000F10809206830606068401B10280AD973
:10251000671900BF00BF6068401B7860656038467F
:10252000FFF77CFF00E000BF144960680968081AE3
:10253000124908600846006812490968884204D2B6
:102540000E4800680F49086000E000BF606840F076
:1025500000406060002020600B480068401C0A4971
:10256000086004E000BF02E000BF00E000BF00BF61
:1025700000BF4846BDE8F087F40A0020F80A0020B2
:10258000EC0A0020FC0A0020000B00202DE9F04F8F
:1025900099B0834600201890402106A8F5F70DFE5B
:1025A000002005904FF6FF7004905C460020F14932
:1025B0000874B4F8050048F22001884204D0B4F849
:1025C0000500491C884243D1CDF80CB0B4F802A0F4
:1025D000B4F8050002906088B0F5967F04DC62884C
:1025E000E11DE548F5F7D0FD5146E348FEF750FE02
:1025F000AAF1020003990A5C401C085C42EA002030
:102600001690AAF1020081B20398F6F7E3FD179045
:10261000DAA0DDE91612FCF78DFCDDE9160188422F
:1026200005D0DCA0FCF786FC19B0BDE8F08F0020D7
:10263000D04948740299E031C8B25246CE49FCF7FD
:102640007FF86420DB4908800420CA498870EBE7E2
:10265000B4F80500B0F5004F5FD034DCB0F5D06FB2
:1026600001F0C38714DCB0F5607F72D009DC8028EC
:1026700054D0B0F5C07F79D0B0F5207F41F0E68727
:1026800083E0B0F5906F66D0B0F5B06FF6D1AAE0F8
:10269000B0F5286F01F0D2870CDCB0F5F06F01F0D7
:1026A000B787B0F5086F01F0B887B0F5186FE5D1BE
:1026B00001F0B8BFB0F5025F01F0C587B0F5065F65
:1026C000DCD101F0C2BF48F20702811A904201F04A
:1026D0009E870DDC6FF400410844062881F0B68720
:1026E000DFE810F043005200610066008000820FB6
:1026F000062901F09C8709DC012901F08D87022958
:1027000001F08F870329B9D101F090BF192901F099
:1027100099871A29B2D101F097BF00BFE07901284B
:102720001ED194498870A44981F87600084600219A
:10273000C1660167A0F874100146A268CA66E06825
:10274000086701208B4988709C4908709A496C3150
:1027500002E029E00AE02CE099A0FCF7EBFB02E0A4
:102760009FA0FCF7E7FB01F072BF00BFE0790128F2
:1027700006D102207F4988709EA0FCF7DBFB02E0B7
:10278000A1A0FCF7D7FBEEE700BFE179A2A0FCF720
:10279000D1FBA649D4F809200A60B4F80D208A803C
:1027A000E07B8871DFE700BFA1A0FCF7C3FBDAE79D
:1027B00000BFA5A0FCF7BEFB207A012801D1A8A08C
:1027C00000E0A9A00146AAA0FCF7B4FB207A40B91A
:1027D0000120AA490870AA48007810B90420A84925
:1027E0000870C0E700BF0120A6490870E07918B959
:1027F000A5A0FCF79FFB02E0A7A0FCF79BFBE079FC
:10280000012841F07786267A3146A7A0FCF792FB93
:10281000012E14D1607A40B9012098490870984877
:10282000007810B9042096490870607A012801D117
:10283000A1A000E0A2A00146A3A0FCF77BFB022E12
:1028400009D1607A012803D1A3A0FCF773FB02E051
:10285000A5A0FCF76FFB042E1BD104F10900F5F7CE
:10286000C9FC85B2102D0FD22A4604F10901524845
:102870001030F5F789FC04F109019FA0FCF75AFB21
:1028800001204E49087004E004F109019FA0FCF703
:1028900051FB072E0AD1657A2946A3A0FCF74AFB13
:1028A0004548A0F86950012044490870062E0ED111
:1028B000657A2946A3A0FCF73DFB3F48A0F84D50A0
:1028C000A0F84F50A0F8515001203C490870082E44
:1028D00003D1657A012039490870092E1DD104F110
:1028E0000900F5F787FC85B2102D0ED22A4604F1B7
:1028F00009013148F5F748FC04F1090197A0FCF7FC
:1029000019FB01202D49087004E004F1090199A088
:10291000FCF710FB0120294908700A2E14D1657AB2
:10292000012D07D10120244981F8870098A0FCF7E8
:1029300001FB06E00020204981F8870094A0FCF705
:10294000F9FA01201D4908700B2E00D1657A0C2E72
:102950000FD1657A012D07D10120174981F889002F
:1029600091A0FCF7E7FA32E10020134981F88900D1
:102970002AE12FE1041F00200A2000200A0D4463F1
:102980007263202530782C56637263202530780AD4
:102990000D0000000A0D20284463726320213D20B1
:1029A00056637263292072657475726E212121212C
:1029B000210A0D003805002098140020FC01002099
:1029C00072656769737465726564207375636365A6
:1029D000737365642C436F64652025730A0D0000D2
:1029E00072656769737465726564206661696C6598
:1029F000640A0D004C6F67696E20537563636573DD
:102A00007365640A0D0000004C6F67696E204661B3
:102A1000696C65640A0D0000686561727420636FFB
:102A2000756E742025640A0D00000000B50B0020AF
:102A3000726563656976652073746174652064618D
:102A40007461200A0D000000726563656976652077
:102A50006368617267652064617461200A0D00001B
:102A6000456E61626C65000044697361626C65006B
:102A70006368617267652025730A0D0035050020C3
:102A80000C02002036050020706172616D207265B5
:102A900061640A0D00000000706172616D20777240
:102AA0006974650A0D000000706172616D206164D7
:102AB00064722025780A0D00656E61626C65000005
:102AC00064697361626C65006368617267696E67EF
:102AD0002025730A0D000000636C6F73652072651A
:102AE0006C61790A0D0000006F70656E2072656C74
:102AF00061790A0D00000000626C7565746F6F7477
:102B000068206E616D652025730A0D00626C756525
:102B1000746F6F7468206E616D65206D6973746188
:102B20006B652025730A0D0048656172742042654B
:102B300061742054696D6520256420207365630AE3
:102B40000D0000004F76657254656D7056616C75AE
:102B5000652025642020200A0D0000005379735061
:102B600061726150696C65442E736E3A25730A0D6B
:102B7000000000005379735061726150696C6544C4
:102B80002E736E206661756C742025730A0D00002B
:102B9000517569636B2043686172676520456E619A
:102BA000626C650A0D000000747269636B6C6520CD
:102BB0004368617267696E6720536F6320456E6179
:102BC000626C6520310A0D00F3A0FCF7B3F9012017
:102BD000F94908700D2E14D1657A642D07DAF7498A
:102BE00081F88A502946F6A0FCF7A4F906E0FAA07D
:102BF000FCF7A0F95A20F14981F88A000120EE493A
:102C000008700E2E15D1657A0A2095FBF0F100FBB5
:102C1000115001900A2095FBF0F000900146F4A0BD
:102C2000019AFCF787F9E54880F88B500120E249CA
:102C300008700F2E0ED1657A2946F3A0FCF77AF9B9
:102C400005EB85004006000EDC4981F88C00012070
:102C5000D9490870102E37D1617AA07A41EA00254F
:102C60002946EFA0FCF766F9D448B0F8590005EB07
:102C70008501B0EB410F0CDD05EB85004FF6FF71D0
:102C800001EA4000CD49A1F883000120CA4908703B
:102C90001AE0CA48B0F8592005EB85004100E4A0CD
:102CA000FCF748F9C548B0F859001438C349A1F8F1
:102CB00083000846B0F883000A2190FBF1F001463A
:102CC0000190E2A0FCF736F9112E25D1617AA07AA5
:102CD00041EA00252946E2A0FCF72CF9B748B0F8F4
:102CE0005B0005EB8501B0EB410F0CDD05EB8500CA
:102CF0004FF6FF7101EA4000B049A1F885000120BC
:102D0000AD49087008E0AD48B0F85B2005EB8500E0
:102D10004100D8A0FCF70EF9122E13D1617AA07AE7
:102D200041EA00252946D9A0FCF704F905EB850006
:102D30004FF6FF7101EA4000A049A1F859000120B7
:102D40009D490870132E13D1617AA07A41EA0025BB
:102D50002946D3A0FCF7EEF805EB85004FF6FF718E
:102D600001EA40009549A1F85B00012092490870F2
:102D7000142E19D1657A2946CEA0FCF7DBF8D2488B
:102D80008078202802DD2020CF498870CE488078C6
:102D900000EBC001CC48C01C00EB41008580CA4854
:102DA0008078401CC8498870162E18D1617AA07AA4
:102DB00041EA00258148A0F863500A2095FBF0F114
:102DC00000FB115001900A2095FBF0F000900146A5
:102DD000BEA0019AFCF7AEF80120774908701D2EBD
:102DE00017D1657A012D01D0022D0FD1734981F8D9
:102DF0008D50012D01D1BBA000E0BBA00146BBA0BE
:102E0000FCF798F801206C49087002E0BCA0FCF7C0
:102E100091F81E2E20D1657A05EB85004FF6FF71E3
:102E200001EA40006549A1F853000846B0F8530094
:102E30000A2190FBF1F201FB120001905F48B0F80B
:102E4000530090FBF1F000900146B3A0019AFCF70B
:102E500071F80120584908701F2E50D1657A5748E3
:102E6000B0F890005549B1F85310884227DD534817
:102E7000B0F853000A2190FBF1F001904F48B0F8F0
:102E8000900090FBF1F000900146A9A0019AFCF798
:102E900051F84A48B0F853000A384849A1F8900060
:102EA0000846B0F890000A2190FBF1F0014601902D
:102EB000AAA0FCF73FF801203F4908701FE005EB8E
:102EC00085004FF6FF7101EA40003C49A1F89000EF
:102ED0000846B0F890000A2190FBF1F201FB1200C5
:102EE00001903648B0F8900090FBF1F00090014658
:102EF000A0A0019AFCF71EF801202F490870202E8F
:102F00001DD1657A05EB85004FF6FF7101EA40009F
:102F10002A49A1F8B3000846B0F8B300642190FB39
:102F2000F1F201FB120001902448B0F8B30090FBCD
:102F3000F1F00090014696A0019AFBF7FBFF212ECD
:102F400020D1657A05EB85004FF6FF7101EA40005C
:102F50001A49A1F8B1000846B0F8B100642190FB0D
:102F6000F1F201FB120001901448B0F8B10090FB9F
:102F7000F1F0009001468DA0019AFBF7DBFF0120E4
:102F80000D490870222E06D1657A0C48A0F8B7507A
:102F9000B0F8B71018E11DE1747269636B6C6520BD
:102FA0004368617267696E6720536F6320456E6185
:102FB000626C6520300A0D00FC010020981400208E
:102FC000747269636B6C654368617267696E67539D
:102FD0006F6325640A0D0000747269636B6C65434E
:102FE00068617267696E67536F632039300A0D003C
:102FF000747269636B6C6520706F776572202564ED
:103000002E25646B770A0D00747269636B6C652002
:1030100063757272656E742564410A0D00000000CC
:10302000426D734D6178566F6C742564200A0D00F3
:10303000256420426D734D6178566F6C7420256451
:10304000206661696C640A0D00000000426D5265E3
:103050007175697265566F6C74202564200A0D00C5
:10306000426D734D617843757272656E742025648C
:10307000200A0D00726571202564206F766572202C
:103080006D6178202564200A0D000000426D734DAB
:103090006178566F6C74202564200A0D00000000D2
:1030A000426D734D617843757272656E742564204C
:1030B0000A0D000073657474696E6720736F63286E
:1030C0002564290A0D000000F41600207542617481
:1030D0004D6178456E657267792025642E25640AF6
:1030E0000D00000043430000435600004368617236
:1030F00067696E674D6F64653A2573200A0D00009D
:103100004368617267696E674D6F646520466175DB
:103110006C740A0D000000004F766572506F776581
:1031200072203A25642E25646B77680A0D00000032
:1031300052657175697265506F77657220256420DC
:103140006B77204F766572506F776572203A2564F1
:103150006B772C6661756C740A0D00005265717591
:10316000697265506F776572202564206B77200A3D
:103170000D00000052657175697265506F77657258
:10318000203A25642E25646B77680A0D0000000044
:103190004261745261746564566F6C746167652036
:1031A0003A25642E2564560A0D0000004261744DD4
:1031B0006178436861726765566F6C203A25642EAA
:1031C0002564560A0D000000EDA0FBF7B3FE0120B8
:1031D000EF490870232E1CD1617AA07A41EA0025BC
:1031E000EC48A0F85F50B0F85F000A2190FBF1F2C4
:1031F00001FB12000190E748B0F85F0090FBF1F08E
:1032000000900146E4A0019AFBF794FE0120E049FA
:103210000870242E1CD1617AA07A41EA0025DD488D
:10322000A0F85950B0F859000A2190FBF1F201FBC7
:1032300012000190D748B0F8590090FBF1F00090CF
:103240000146DCA0019AFBF775FE0120D049087009
:10325000252E0CD1657A2946DBA0FBF76BFE05F124
:103260003200CC4981F8B5000120C9490870262EEA
:103270000CD1657A2946DBA0FBF75CFE05F1320034
:10328000C44981F8B6000120C1490870272E33D106
:10329000657AC04880F8B050012D02D1D8A0FBF764
:1032A00049FE022D02D1DCA0FBF744FE032D02D122
:1032B000DFA0FBF73FFE042D02D1E4A0FBF73AFEAE
:1032C000052D02D1E7A0FBF735FE062D02D1EBA0BC
:1032D000FBF730FE072D02D1EEA0FBF72BFE082DE9
:1032E00002D1F4A0FBF726FEFF2D02D1F7A0FBF7D9
:1032F00021FE0120A6490870282E13D1617AA07AF8
:1033000041EA0025A348A0F85D50B0F85D000A210D
:1033100090FBF1F001460190F2A0FBF70BFE0120BB
:103320009B490870292E19D1657A0A2D0BDB642D73
:1033300009DC984981F89350084690F89310EEA064
:10334000FBF7F8FD07E02946F4A0FBF7F3FD0020AA
:10335000904981F8930001208D4908702A2E1FD1D1
:10336000617AA07A41EA0025B5F57A7F11DB40F653
:10337000AC5085420DDC8748A0F8A650B0F8A600F6
:103380000A2190FBF1F001460190EAA0FBF7D2FD83
:1033900003E02946EFA0FBF7CDFD01207C49087032
:1033A0002B2E19D1657A012D03D17A4981F8A850C5
:1033B00003E00020774981F8A800764890F8A8003B
:1033C000012801D1EDA000E0EEA00146EFA0FBF73F
:1033D000B1FD01206E490870302E1CD1617AA07AAF
:1033E00041EA00256B48A0F86350B0F863000A2159
:1033F00090FBF1F201FB120001906648B0F8630007
:1034000090FBF1F000900146E7A0019AFBF792FDD6
:1034100001205F490870312E23D1617AA07A41EAF8
:10342000002505EB85004FF6FF7101EA4000594980
:10343000A1F88E000846B0F88E000A2190FBF1F248
:1034400001FB120001905348B0F88E0090FBF1F0A0
:1034500000900146DAA0019AFBF76CFD01204C496F
:103460000870322E0BD1657A4A48A0F84D50B0F85A
:103470004D10DAA0FBF75EFD012045490870332EA0
:103480000BD1657A4348A0F84F50B0F84F10D9A03F
:10349000FBF750FD01203E490870342E0BD1657AB0
:1034A0003C48A0F85150B0F85110D8A0FBF742FDAD
:1034B000012037490870352E1BD1657A012D03D1C3
:1034C000344981F8925003E00020324981F892009B
:1034D000304890F89200012802D1AFF67C2001E03C
:1034E000AFF67C200146CFA0FBF724FD0120284940
:1034F0000870362E18D1112126489530F4F75DFE5C
:1035000024481D30D4F809208267D4F80D20C26702
:10351000B4F81110A0F8801004F10901C7A0FBF75E
:1035200009FD01201A490870372E12D1194895302B
:10353000D4F80920C0F80A20B4F80D20C281E17B3C
:10354000017404F10901C3A0FBF7F4FC0120104948
:103550000870502E11D1657A012D03D10D4981F8E3
:10356000745103E000200B4981F87401094890F878
:103570007401012802D1BFA085E18BE182E1000046
:10358000426174436F756E74203A25640A0D000021
:10359000FC01002098140020546F74616C4361702A
:1035A0006163697479203A25642E256441480A0DC7
:1035B00000000000426D734D6178566F6C743A25BF
:1035C000642E2564760A0D00754261744D6178544D
:1035D000656D70506C75733530203A2564200A0D86
:1035E00000000000754261744D696E54656D705045
:1035F0006C75733530203A2564200A0D00000000F8
:103600007563426174547970653AC7A6CBE1B5E73A
:10361000B3D8200A0D0000007563426174547970BC
:10362000653AC4F8C7E2B5E7B3D8200A0D00000038
:103630007563426174547970653AC1D7CBE1CCFAB5
:10364000EFAEB5E7B3D8200A0D0000007563426104
:1036500074547970653AC3CCCBE1EFAEB5E7B3D81B
:10366000200A0D007563426174547970653AEEDC8E
:10367000CBE1EFAEB5E7B3D8200A0D007563426128
:1036800074547970653AC8FDD4AAEFAEB5E7B3D8E3
:10369000200A0D007563426174547970653ABEDB8F
:1036A000BACFCEEFEFAEC0EBD7D3B5E7B3D8200A91
:1036B0000D0000007563426174547970653AEED173
:1036C000CBE1EFAEB5E7B3D8200A0D0075634261D8
:1036D00074547970653AC6E4CBFBB5E7B3D8200AD9
:1036E0000D000000546F74616C566F6C74616765F7
:1036F0003A256420200A0D0052657175697265567D
:103700006F6C74616765446966666572656E636552
:103710002825642956200A0D000000002028256471
:103720002956206F7665722072616E6765200A0DDA
:103730000000000053696D756C61746564437572B7
:1037400072656E74426174566F6C74202564560AFB
:103750000D00000053696D756C617465644375728A
:1037600072656E74426174566F6C74202564562DB8
:103770002D3130302D333530560A0D004F50454E27
:1037800000000000434C4F534500000025732044C7
:10379000656275675F506167655F66756E637469C2
:1037A0006F6E200A0D000000754261744D6178450E
:1037B0006E65726779202564202E2564200A0D002D
:1037C00053746F70566F6C74616765203A25642E70
:1037D0002564205620200A0D000000004F766572F7
:1037E00054656D703056616C75653A256420200A09
:1037F0000D0000004F76657254656D703156616C36
:1038000075653A256420200A0D0000004F76657228
:1038100054656D703256616C75653A256420200AD6
:103820000D0000005369676E616C4C6F7373466CDA
:10383000616720257320200A0D0000005665686925
:1038400063686C65496E666F28302D39293A257397
:103850000A0D00005665686963686C65496E666F9D
:103860002056494E2831302D3137293A25730A0D1B
:103870000000000070726F66657373696F6E616C33
:1038800000000000F4A00146F5A0FBF753FB012067
:10389000F8490870512E2DD1617AA07A41EA0025AD
:1038A000302D0CDBB5F5967F09DA05EB85004FF678
:1038B000FF7101EA4000F049A1F8750103E02946D3
:1038C000EEA0FBF737FBEC48B0F875010A2190FB3E
:1038D000F1F201FB12000190E748B0F8750190FB8E
:1038E000F1F000900146EEA0019AFBF723FB0120C6
:1038F000E0490870522E2CD1617AA07A41EA002565
:103900000A2D0BDD642D09DA05EB85004FF6FF71FA
:1039100001EA4000D849A1F8770103E02946E7A071
:10392000FBF708FBD448B0F877010A2190FBF1F2CD
:1039300001FB12000190D048B0F8770190FBF1F044
:1039400000900146E7A0019AFBF7F4FA0120C9496B
:103950000870532E23D1657A0A2D05DD962D03DAE2
:10396000C548A0F8795103E02946E4A0FBF7E2FA44
:10397000C148B0F879010A2190FBF1F201FB120075
:103980000190BD48B0F8790190FBF1F0009001463C
:10399000E2A0019AFBF7CEFA0120B6490870542E36
:1039A0000BD1657AB44880F87B5190F87B11E1A087
:1039B000FBF7C0FA0120AF490870552E0BD1657A8C
:1039C000AD4880F87C5190F87C11E0A0FBF7B2FA8A
:1039D0000120A8490870562E2CD1617AA07A41EABC
:1039E0000025302D0BDBFA2D09DA05EB85004FF6AB
:1039F000FF7101EA4000A049A1F87D0103E02946DA
:103A0000D7A0FBF797FA9C48B0F87D010A2190FBFC
:103A1000F1F201FB120001909748B0F87D0190FB94
:103A2000F1F000900146D7A0019AFBF783FA01203C
:103A300090490870572E2CD1617AA07A41EA00256E
:103A4000142D0BDB6E2D09DA05EB85004FF6FF71A7
:103A500001EA40008849A1F87F0103E02946D0A08F
:103A6000FBF768FA8448B0F87F010A2190FBF1F275
:103A700001FB120001908048B0F87F0190FBF1F04B
:103A800000900146CFA0019AFBF754FA0120794932
:103A90000870582E0ED1657A962D02DA764981F893
:103AA0008151754890F88111CDA0FBF743FA0120B0
:103AB00070490870592E0ED1657A962D02DA6E493A
:103AC00081F882516C4890F88211CBA0FBF732FA52
:103AD0000120684908705A2E1AD1657A012D03D148
:103AE000654981F8905103E00020634981F8900115
:103AF000614890F89001012801D1C44801E0C34811
:103B000008300146C2A0FBF715FA01205949087098
:103B1000602E1AD1657A012D03D1574981F887515A
:103B200003E00020544981F88701534890F8870149
:103B3000012801D1B54801E0B44808300146BAA0D7
:103B4000FBF7F8F901204B490870612E1AD1657A0C
:103B5000012D03D1484981F8885103E000204649EE
:103B600081F88801444890F88801012801D1A748CC
:103B700001E0A64808300146AFA0FBF7DBF90120C1
:103B80003C490870622E25D1657A032D03DC3A4941
:103B900081F8895103E00020374981F889013648CE
:103BA00090F88901012802D1A8A0FBF7C3F9324897
:103BB00090F88901022802D1A9A0FBF7BBF92E4891
:103BC00090F88901032802D1AAA0FBF7B3F90120DC
:103BD00028490870632E24D1617AA07A41EA002531
:103BE000254890F88901012803D12946A6A0FBF7B2
:103BF000A1F9214890F88901022803D12946A8A0FB
:103C0000FBF798F91C4890F88901032803D129464D
:103C1000A9A0FBF78FF91848A0F88A51012015498F
:103C20000870642E02D1012012490870652E11D14E
:103C3000657A012D03D1104981F88C5103E00020F1
:103C40000D4981F88C010C4890F88C01012802D1B3
:103C50006E483EE144E13BE165617379000000009C
:103C6000576F726B4D6F64656C20257320200A0DB1
:103C700000000000FC01002098140020444352651D
:103C80007175697265566F6C742025643A4F76655C
:103C9000722834382D333030292020200A0D0000BE
:103CA000444352657175697265566F6C743A256448
:103CB0002E2564205620200A0D0000004443526542
:103CC000717569726543757272656E742564413AE7
:103CD0004F7665722831302D313030412920202037
:103CE0000A0D00004443526571756972654375722F
:103CF00072656E74256441200A0D000044434D61D5
:103D000078506F7765722564203A4F766572283156
:103D10002D31356B2909200A0D00000044434D6107
:103D200078506F7765723A25642E2564206B770989
:103D30000A0D000044435F496E64756374616E63ED
:103D40006554656D70202564200A0D0044435F4969
:103D500047425454656D70202564200A0D00000010
:103D600044434D6178566F6C74202564563A4F7603
:103D700065722834382D32303056292020200A0D23
:103D80000000000044432044434D6178566F6C743A
:103D90003A25642E2564205620200A0D00000000DC
:103DA00044432044434D617843757272656E7425B7
:103DB000643A4F7665722832302D31313029202017
:103DC000200A0D0044432044434D617843757272CC
:103DD000656E743A25642E2564204120200A0D006A
:103DE00043617061636974616E636554656D7031C0
:103DF000202564200A0D00004443426F7854656D0D
:103E00007032202564200A0D00000000602A01089D
:103E1000446F75626C65426174746572794D6F644C
:103E2000652025730A0D000056494E205472616EBC
:103E3000732025730A0D0000426C75655369676E27
:103E4000616C4C6F737325730A0D000043686172D7
:103E500067654D6F64652D2D6B77680A0D00000056
:103E60004368617267654D6F64652D2D74696D657A
:103E70000A0D00004368617267654D6F64652D2D02
:103E8000534F430A0D0000004368617267654D6F30
:103E900064652D6B7768282564290A0D00000000F1
:103EA0004368617267654D6F64652D74696D65283F
:103EB0002564290A0D0000004368617267654D6F33
:103EC00064652D534F43282564290A0D0000000026
:103ED000F9480146F9A0FBF72DF80120FE490870CA
:103EE0006D2E1ED1657A012D06D10120FB4981F886
:103EF0009701FBA0FBF71EF8022D06D10220F7491F
:103F000081F89701FBA0FBF715F8032D06D10320DC
:103F1000F24981F89701FCA0FBF70CF80120EE496B
:103F200008706E2E1DD1617AA07A41EA0025EB4817
:103F3000A0F89851C82D0BDDB5F53E7F08DA05EBEA
:103F400085004FF6FF7101EA4000E449A1F85900ED
:103F5000E248B0F89811F1A0FAF7ECFF0120DE4931
:103F600008706F2E1CD1617AA07A41EA0025C82D15
:103F70000BDDB5F53E7F08DA05EB85004FF6FF71E6
:103F800001EA4000D549A1F85D00D448A0F89A5153
:103F9000B0F89A11E9A0FAF7CDFF0120CE490870D8
:103FA000702E0DD1617AA07A41EA0025CB48A0F8A5
:103FB0009C512946E9A0FAF7BDFF0120C6490870C7
:103FC000712E0DD1617AA07A41EA0025C348A0F88C
:103FD0009E512946EBA0FAF7ADFF0120BE490870BB
:103FE000722E0DD1617AA07A41EA0025BB48A0F873
:103FF000A0512946E3A0FAF79DFF0120B6490870B9
:10400000732E0DD1617AA07A41EA0025B348A0F859
:10401000A2512946E3A0FAF78DFF0120AE490870AE
:10402000742E0DD1617AA07A41EA0025AB48A0F840
:10403000A4512946DBA0FAF77DFF0120A6490870AC
:10404000752E0DD1617AA07A41EA0025A348A0F827
:10405000A6512946D3A0FAF76DFF01209E490870AA
:10406000762E0DD1617AA07A41EA00259B48A0F80E
:10407000A8512946CBA0FAF75DFF012096490870A8
:10408000772E0DD1617AA07A41EA00259348A0F8F5
:10409000AA512946C3A0FAF74DFF01208E490870A6
:1040A000782E0DD1617AA07A41EA00258B48A0F8DC
:1040B000AC512946BBA0FAF73DFF012086490870A4
:1040C000792E0DD1617AA07A41EA00258348A0F8C3
:1040D000AE512946B3A0FAF72DFF01207E490870A2
:1040E0007A2E0DD1617AA07A41EA00257B48A0F8AA
:1040F000B0512946ABA0FAF71DFF012076490870A0
:104100007B2E0DD1617AA07A41EA00257348A0F890
:10411000B2512946A3A0FAF70DFF01206E4908709D
:104120007C2E0DD1617AA07A41EA00256B48A0F877
:10413000B45129469BA0FAF7FDFE0120664908709C
:104140007D2E0DD1617AA07A41EA00256348A0F85E
:10415000B651294693A0FAF7EDFE01205E4908709A
:104160007E2E0DD1617AA07A41EA00255B48A0F845
:10417000B85129468BA0FAF7DDFE01205649087098
:104180007F2E0DD1617AA07A41EA00255348A0F82C
:10419000BA51294683A0FAF7CDFE01204E49087096
:1041A000802E0DD1617AA07A41EA00254B48A0F813
:1041B000BC51294683A0FAF7BDFE0120464908708C
:1041C000812E0DD1617AA07A41EA00254348A0F8FA
:1041D000BE51294681A0FAF7ADFE01203E49087084
:1041E000822E0DD1617AA07A41EA00253B48A0F8E1
:1041F000C051294679A0FAF79DFE01203649087082
:10420000832E0DD1617AA07A41EA00253348A0F8C7
:10421000C251294671A0FAF78DFE01202E4908707F
:10422000842E0DD1617AA07A41EA00252B48A0F8AE
:10423000C451294669A0FAF77DFE0120264908707D
:10424000852E0DD1617AA07A41EA00252348A0F895
:10425000C651294661A0FAF76DFE01201E4908707B
:10426000862E0DD1617AA07A41EA00251B48A0F87C
:10427000C851294659A0FAF75DFE01201649087079
:10428000872E0DD1617AA07A41EA00251348A0F863
:10429000CA51294651A0FAF74DFE01200E49087077
:1042A000882E07D1617AA07A41EA00250B48A0F850
:1042B000CC519FE0A6E00000682A010868696768A1
:1042C00020766F6C74616765206D6F64756C652016
:1042D00025730A0D00000000FC0100209814002046
:1042E000536F6353696D756C61547970652D310A34
:1042F0000D000000536F6353696D756C61547970E4
:10430000652D320A0D000000536F6353696D756CA3
:1043100061547970652D330A0D0000000A0D205399
:104320006F6353696D756C614D6178566F6C742065
:10433000202564205620200A0D0000000A0D20537D
:104340006F6353696D756C614D696E566F6C742047
:10435000202564205620200A0D0000000A0D20535D
:104360006F6343616C6962726174696F6E566F6CE2
:1043700074202025642028302E31295620200A0D53
:10438000000000000A0D20536F6343616C69627284
:104390006174696F6E566F6C7420202564205620FE
:1043A000200A0D00536F6343616C69627261746926
:1043B0006F6E566F6C7420202564205620200A0DE5
:1043C00000000000536F6343616C6962726174693D
:1043D0006F6E2020256420200A0D0000536F634378
:1043E000616C6962726174696F6E2020256420209F
:1043F000200A0D002946AFF21C00FAF79BFD0120B0
:1044000095490870892E0ED1617AA07A41EA00257B
:104410009248A0F8CE512946AFF24000FAF78AFD43
:1044200001208D4908708A2E0ED1617AA07A41EA66
:1044300000258A48A0F8D0512946AFF26000FAF76B
:1044400079FD0120844908708B2E0ED1617AA07A03
:1044500041EA00258148A0F8D2512946AFF28400F4
:10446000FAF768FD01207C4908708C2E0ED1617A24
:10447000A07A41EA00257948A0F8D4512946AFF244
:10448000A400FAF757FD0120734908708D2E0ED154
:10449000617AA07A41EA00257048A0F8D6512946F1
:1044A000AFF2C800FAF746FD01206B4908708E2E66
:1044B0000ED1617AA07A41EA00256848A0F8D85167
:1044C0002946AFF2E800FAF735FD0120624908708D
:1044D0008F2E0ED1617AA07A41EA00255F48A0F8BC
:1044E000DA512946AFF20C10FAF724FD01205A499F
:1044F000087078E0E079E8BB94F80880414658A05D
:10450000FAF718FD5B4880F8008000780D2804D188
:104510000020584908705849488000205649488072
:1045200000F00EFA00273BE0B81CE11D0E5C4FF0D6
:10453000000930E0514810F83900B04227D14F4807
:1045400000EBC900427831464DA0FAF7F3FC08F1C0
:104550000203DFF824C1BCF802C09C44464BDB1DBB
:104560000CEB0300454B03EBC9035A78434B03EBB9
:10457000C90300E037E05968F3F706FE3E4840887B
:104580003E4901EBC901497808443B49488009F19B
:10459000010000F0FF09B9F1610FCBD3781CC7B25D
:1045A0004745C1DB3448418808F1020008443249DC
:1045B000488041F20500A1F80500E079C87108467D
:1045C00080F80880002707E0B81CE11D0A5C2A4932
:1045D000C91D0A54781CC7B24745F5DB05AA06A9D0
:1045E0002548F6F7F3FD32E000BFE07901280DD150
:1045F00000201A4981F8B90078211848BA30F3F739
:10460000DCFDF9F76FFB27A0FAF794FC1FE000BF71
:104610002AA0FAF78FFC1AE000BF28A0FAF78AFC5C
:1046200015E000BF25A0FAF785FC10E000BF2AA026
:10463000FAF780FC00202F49087408E01FA0FAF761
:1046400079FC04E000BF02E000BF00E000BF00BF53
:1046500000BFFDF7E9BF0000FC0100209814002016
:104660005265616420706172616D206E756D2025E8
:10467000640A0D00340500207E1D00202C0200205D
:104680007265616420706172616D20616464722082
:104690003078257820706172616D206C656E202500
:1046A000640A0D0052656365697665207265636F03
:1046B0007264732061636B0A0D00000052656365CC
:1046C00069766520444344432073746174652061B6
:1046D000636B0A0D00000000526563656976652012
:1046E000444542554720444344432061636B0A0DCF
:1046F00000000000041F00200146488808B18868B7
:1047000008B9012070470020FCE7014648880A8864
:10471000904201DB012070470020FCE710B50380C8
:10472000002444808160828002FB0314C46084689A
:1047300004618468446110BD70B504460D4660880C
:1047400008B1A06808B9002070BDA2882846616938
:10475000F3F71AFDA188606908446061E168606947
:10476000884201D3A06860616088401E6080A08894
:10477000EAE770B504460D4660882188884201DA70
:10478000A06808B9002070BDA28829462069F3F707
:10479000FBFCA188206908442061D4E90310884209
:1047A00001D3A06820616088401C60800120EAE796
:1047B000026811BA426812BA02604160704702682A
:1047C00011BA426812BA02604160704710B586B0F3
:1047D000044601210420F8F7F9FD01214804F8F707
:1047E000D5FD0420ADF8140003208DF81600182024
:1047F0008DF8170005A92048F6F7CAFF0820ADF884
:10480000140048208DF8170005A91B48F6F7C0FFD3
:1048100026208DF8000001208DF801008DF802009F
:104820008DF803006846F8F75BF801940020ADF8B6
:104830000800ADF80A00ADF80C00ADF810000C202F
:10484000ADF80E0001A90D48F9F704FF012240F26E
:1048500025510A48F9F7D9FE012240F224410748C0
:10486000F9F7D3FE01210548F9F78CFE80210348B2
:10487000F9F770FE06B010BD00080140004400408A
:1048800010B586B0044601211120F8F79FFD0121E3
:10489000C804F8F77BFD4FF48060ADF814000320E6
:1048A0008DF8160018208DF8170005A92248F6F794
:1048B0006FFF4FF40060ADF8140048208DF817002A
:1048C00005A91D48F6F764FF34208DF80000032089
:1048D0008DF801008DF8020001208DF80300684674
:1048E000F7F7FEFF01940020ADF80800ADF80A00CC
:1048F000ADF80C00ADF810000C20ADF80E0001A9C9
:104900000E48F9F7A7FE01210C48F9F73BFE0122FA
:1049100040F225510948F9F778FE012240F226615C
:104920000648F9F772FE012240F224410348F9F7E4
:104930006CFE06B010BD000000100140004C0040AD
:104940003848B0F859000A2190FBF1F03649088048
:104950003448B0F85B000A2190FBF1F032494880FE
:104960003048B0F883000A2190FBF1F02E4908820C
:104970002C48B0F853000A2190FBF1F02A49088333
:104980002848B0F88E000A2190FBF1F02649888271
:104990002448B0F885000A2190FBF1F022494882B2
:1049A000204890F88B000A2190FBF1F01E49887690
:1049B0001C4890F88C000A2190FBF1F01A49C87647
:1049C0001848B0F890000A2190FBF1F01649C8820F
:1049D0001448B0F8B1000A2190FBF1F01249888325
:1049E0001048B0F8B3000A2190FBF1F00E49C883DB
:1049F0000C48B0F8B1000A2190FBF1F00A49888315
:104A0000084890F8B600323881F82100054890F83F
:104A1000B500323881F82000024890F8790181F819
:104A20002200704798140020E61F002070B505464C
:104A3000002462E004EB440000EBC400304901EBC9
:104A4000001090F85400032800DA54E004EB44000E
:104A500000EBC4002A4901EB001090F891000128F6
:104A60000AD104EB440000EBC40001EB0010027813
:104A700004210120FCF714F904EB440000EBC4000E
:104A80001F4901EB001090F89100022832D104EB8D
:104A9000440000EBC40001EB001090F8AC00401C97
:104AA000C1B204EB440000EBC400154A02EB001055
:104AB00080F8AC1004EB440000EBC400114601EB9D
:104AC000001090F8AC00022814DB032104EB440032
:104AD00000EBC40002EB001080F8911004EB4400DE
:104AE00000EBC400114601EB001002780421012004
:104AF000FCF7D6F800BF601CC4B2022C9ADB70BD74
:104B0000B4120020D8FF0000F8339F43D9FF000003
:104B100058699543DAFF0000BA298C43DBFF000097
:104B2000C77B8343DCFF000071BD7643DDFF0000DF
:104B3000A09A6743DEFF000000805943DFFF0000BA
:104B4000E75B4C43E0FF0000E71B4043E1FF000050
:104B50001BAF3443E2FF00005A042A43E3FF000086
:104B60008B0C2043E4FF00001DBA1643E5FF000054
:104B700042000E43E6FF0000B6D30543E7FF000006
:104B80007B54FC42E8FF0000C3F5ED42E9FF000062
:104B90005879E042EAFF000068D1D342EBFF000001
:104BA000E6EEC742ECFF0000AFC5BC42EDFF0000DF
:104BB000C749B242EEFF00002E70A842EFFF00008E
:104BC000B22E9F42F0FF0000C07B9642F1FF000032
:104BD0008A4E8E42F2FF0000AB9E8642F3FF000039
:104BE0009AC87E42F4FF000007307142F5FF0000D2
:104BF000FE656442F6FF0000645D5842F7FF000066
:104C0000230A4D42F8FF0000C5604242F9FF000050
:104C10006D563842FAFF000048E12E42FBFF0000CB
:104C2000B5F72542FCFF000000911D42FDFF00008A
:104C3000DDA41542FEFF00009F2B0E42FFFF000087
:104C4000011E0742000000005A75004201000000EA
:104C5000A156F441020000005474E8410300000032
:104C60005238DD4104000000FC98D24105000000EC
:104C70004A8CC84106000000D509BF41070000006A
:104C8000CE08B64108000000D881AD4109000000FF
:104C9000916DA5410A00000039C59D410B0000003F
:104CA000758296410C0000008A9F8F410D00000024
:104CB000F01689410E00000088E382410F000000D9
:104CC00069007A4110000000B7D16E411100000068
:104CD0006132644112000000CE195A4113000000F5
:104CE0006F815041140000007C61474115000000B5
:104CF00039B43E4116000000197336411700000018
:104D0000F6972E41180000004F1E274119000000A1
:104D1000000020411A000000DA3819411B00000091
:104D200028C412411C000000939D0C411D0000008E
:104D300020C106411E000000022B01411F0000009F
:104D400025AFF74020000000D786ED40210000008D
:104D5000A1D6E340220000009E98DA402300000024
:104D6000E7C6D14024000000145CC94025000000C3
:104D70001153C14026000000DFA6B9402700000003
:104D8000FC52B240280000001153AB402900000043
:104D9000DBA2A4402A000000963E9E402B000000AB
:104DA0007D2298402C0000000A4B92402D0000000C
:104DB000E1B48C402E000000E65C87402F0000002C
:104DC00010408240300000002CB77A4031000000D3
:104DD0006059714032000000D0616840330000002B
:104DE00092CB5F4034000000109257403500000025
:104DF000DEB04F4036000000E2234840370000009C
:104E00002EE740403800000027F739403900000005
:104E1000DF4F33403A00000063EE2C403B000000BF
:104E20006CCF26403C000000B3EF20403D00000066
:104E3000984C1B403E00000054E315403F0000002A
:104E40001CB1104040000000D0B30B4041000000F6
:104E5000A7E8064042000000D34D02404300000096
:104E6000BEC1FB3F44000000FB3FF33F4500000094
:104E70001B12EB3F460000002B35E33F47000000CC
:104E8000E8A4DB3F480000005F5ED43F490000001B
:104E90004A5ECD3F4A000000B6A1C63F4B0000006D
:104EA0000326C03F4C0000003EE8B93F4D00000023
:104EB00075E5B33F4E000000041CAE3F4F000000FC
:104EC000A488A83F50000000062AA33F510000001C
:104ED00037FD9D3F520000009300993F53000000B2
:104EE0002332943F54000000EF8F8F3F55000000A5
:104EF00001188B3F5600000008C9863F570000008C
:104F000062A1823F580000002D3E7D3F5900000005
:104F1000AE81753F5A0000004E0B6E3F5B000000F3
:104F20001FD7663F5C0000002AE35F3F5D00000082
:104F3000CF2C593F5E00000018B2523F5F000000C6
:104F400065704C3F600000001765463F610000003F
:104F5000DE8E403F620000001CEB3A3F6300000021
:104F6000D977353F640000006E34303F65000000A3
:104F7000931D2B3F66000000A032263F6700000013
:104F80009F71213F6800000040D91C3F690000006C
:104F90008C67183F6A000000331B143F6B00000051
:104FA000E5F20F3F6C00000052ED0B3F6D0000007A
:104FB0002D09083F6E000000CC45043F6F00000043
:104FC00038A1003F700000009335FA3E71000000E8
:104FD0006362F33E720000008FC7EC3E7300000076
:104FE0007862E63E740000007F30E03E750000000D
:104FF000A531DA3E76000000FA61D43E7700000069
:105000007FC1CE3E78000000944DC93E790000007B
:105010003A06C43E7A00000082E7BE3E7B000000F4
:105020006BF1B93E7C0000005721B53E7D000000C9
:105030009678B03E00000000710B0108210C0108B9
:10504000B509010800000000000000000000000099
:105050000000000001000000710B0108210C010894
:10506000B509010800000000000000000000000079
:105070000000000030003000300030003000C6007A
:1050800041343055303400000000000001000000C1
:105090003C5401086910010801000000D8530108C0
:1050A000B711010801000000D0530108B511010833
:1050B0000100000030540108B9110108010000008E
:1050C000285401081D120108010000001C540108A9
:1050D0001B12010801000000E05301081912010829
:1050E00001000000405401083D11010801000000CA
:1050F000C8530108211201080100000050540108A2
:105100004111010801000000485401081110010874
:1051100001000000B8530108BD11010801000000A2
:10512000645401086D100108010000005854010882
:10513000D11001080100000070540108A50F0108FA
:1051400001000000045401085DC6000801000000D1
:10515000EC53010835C60008010000001054010896
:105160009DC9000801000000F8530108D5AE0008F1
:1051700000C1814001C0804101C0804100C1814027
:1051800001C0804100C1814000C1814001C0804117
:1051900001C0804100C1814000C1814001C0804107
:1051A00000C1814001C0804101C0804100C18140F7
:1051B00001C0804100C1814000C1814001C08041E7
:1051C00000C1814001C0804101C0804100C18140D7
:1051D00000C1814001C0804101C0804100C18140C7
:1051E00001C0804100C1814000C1814001C08041B7
:1051F00001C0804100C1814000C1814001C08041A7
:1052000000C1814001C0804101C0804100C1814096
:1052100000C1814001C0804101C0804100C1814086
:1052200001C0804100C1814000C1814001C0804176
:1052300000C1814001C0804101C0804100C1814066
:1052400001C0804100C1814000C1814001C0804156
:1052500001C0804100C1814000C1814001C0804146
:1052600000C1814001C0804101C0804100C1814036
:1052700000C0C101C30302C2C60607C705C5C404F6
:10528000CC0C0DCD0FCFCE0E0ACACB0BC90908C866
:10529000D81819D91BDBDA1A1EDEDF1FDD1D1CDC56
:1052A00014D4D515D71716D6D21213D311D1D010C6
:1052B000F03031F133F3F23236F6F737F53534F4B6
:1052C0003CFCFD3DFF3F3EFEFA3A3BFB39F9F83826
:1052D00028E8E929EB2B2AEAEE2E2FEF2DEDEC2C16
:1052E000E42425E527E7E62622E2E323E12120E086
:1052F000A06061A163A3A26266A6A767A56564A476
:105300006CACAD6DAF6F6EAEAA6A6BAB69A9A868E5
:1053100078B8B979BB7B7ABABE7E7FBF7DBDBC7CD5
:10532000B47475B577B7B67672B2B373B17170B045
:105330005090915193535292965657975595945435
:105340009C5C5D9D5F9F9E5E5A9A9B5B99595898A5
:10535000884849894B8B8A4A4E8E8F4F8D4D4C8C95
:105360004484854587474686824243834181804005
:10537000A55A00000D0A3737375570642D2D747902
:1053800070653A253078202C7665723A2530782C75
:1053900054627974653A2530782C204372633A253B
:1053A00030782C5061673A2530782C506C656E3A15
:1053B0002530780D0A0000005265616C79486967F4
:1053C00068343030000000004B43353600000000E8
:1053D0004F464644434443004F4E44434443000039
:1053E00053455441504E50574400000041435F72B2
:1053F00045634C4F53450000414352656C61794F02
:105400004646000041435F72454F50454E00000044
:10541000414352656C61794F4E0000005345544141
:10542000504E55534552000054455354424D53007D
:10543000524541444D415353000000005345540030
:105440005265736574000000414363757400000089
:105450004443637574000000434332434352656123
:105460006C79000043433143505265616C79000010
:1054700047554E54656D705265616C7900000000AF
:1054800048414E440000000049444C4500000000E3
:1054900052554E4E494E470053544F5000000000A5
:1054A000494E49540000000053544152540000003A
:1054B0006368617267655F4D6F64655F3132560086
:1054C0005245414459000000526573657276656427
:1054D000000000005265736572766174696F6E5FDB
:1054E00041435F6368617267655F6D6F646500006B
:1054F00044435F6368617267655F6D6F6465000058
:1055000041435F6469736368617267655F6D6F646F
:105510006500000044435F64697363686172676596
:105520005F6D6F64650000004E6F726D616C5F6D42
:105530006F64650052656D6F74655F636F6E747242
:105540006F6C5F6D6F6465006368617267655F6251
:105550006174746572795F686561745F6D6F6465AD
:105560000000000052656D6F74655F626174746560
:1055700072795F686561745F6D6F6465000000003B
:1055800044656661756C745F6D6F64650000000052
:1055900041435F4368617267000000004B43310084
:1055A000595831004B433200595832004B433300B5
:1055B0004B4335004B4338004B43390043414E3198
:1055C0005F5354420000000043414E325F53544247
:1055D00000000000454C535F4F46460048565F446C
:1055E00053475F434845434A0000000043414E3261
:1055F0005F454E00454C535F4F4E00004D43555F95
:1056000052554E005057335F3356000050573556B1
:10561000000000003456010800000020140B0000B8
:105620003C8A0008605B0108140B00200C69000034
:105630008CEF00088133E80384A24A0400092C019E
:10564000020304060708091AFF0181B0089EC97FFA
:105650007F1EAB8252A61389BE140855BC1B08617D
:10566000041AAD0C1309A914086DDD140859B914F6
:105670000805C8027008024301180E111C0108D960
:105680001A0108331B010843041A79044123140347
:10569000B2641AE8109AF47100091CD5FBB3B5D0B6
:1056A000ADD2E963030A1E150901085104092A3421
:1056B00001501A02BC132A025B2001085A03082376
:1056C000051013B8141B2004081AA8082306021A90
:1056D000E5081A07081301151B2008281A03081AE1
:1056E00009201A98181A0A101A1F101A0F081A24DB
:1056F000081A0E081A23081A0D081A22081A0C088C
:105700001A21085A0B601A13481AF3381A12081A89
:10571000F1081A11081A1D201A10081A1B081A1469
:105720000829281A16081AFB201A18381A48181AB5
:105730001F0813FC1F1B201E081AFE081A1D081A3A
:1057400025181A20081304201B2021081A02081A01
:1057500022081A4F185A24601A23081AF7085A27E1
:10576000481A26081A07281A25081A06081A28208F
:105770001AF5201A29101A2B20197C111A3E081A22
:105780002B101A40085A30881A31081AFA781A323F
:10579000181AE5101A33081AE7081A34081AE90823
:1057A0002A35E0193023360A1A2D082337071A370D
:1057B000081A5018130C161B2051401A0D081A52C3
:1057C000081A0F081A53181A11081A54081A13083D
:1057D0001A55081A14081A56201A15081A57081AC2
:1057E00017081A58181A19081A59081A1A081A5AAA
:1057F000081A28081A60081A1F081A61081A2008CF
:105800001A62081A21081A63381A22081A65101A2F
:1058100024081A66081A25081A6D081A2F081A6E25
:10582000201A30081A6F081A32081A70081A340839
:105830001A71081A36081A72081A38081A73081AE0
:105840003A081A74081A3C081A75081A3E081A769B
:10585000081A40081A77081A42081A78081A4408E1
:105860001A79081A46081A7A081A48081A7B081A78
:105870004A081A7C081A4C081A7D081A4E081A7E23
:10588000081A50081A7F081A52081A80081A540871
:105890001A81081A56081A82081A58081A83081A10
:1058A0005A081A84081A5C081A85081A5E081A86AB
:1058B000081A60081A87081A62081A88081A640801
:1058C0001A89081A66081A8A081A68081A8B081AA8
:1058D0006A081A8C081A6C081A8D081A6E081A8E33
:1058E000081A70081A8F081A7208012E1AFF01018F
:1058F0001A036FE8032D01020304043009060708A8
:105900000902040608133DFB240804011315CA1BF1
:105910000809081A75081A57981AAD081A58081A6B
:10592000E1081A59081331CB1B085D081A71081ACF
:105930005F081A9508239B051AB9081AE6101ADDA4
:10594000081AE7081375CC1B0880181AC1082A1119
:105950005012D02967511751180108D9AB8C08791A
:10596000AC14411A59181AF114DA611817C5170145
:10597000080DADDB0845181A61301A2518DAA51C88
:105980001AAF181A3D141AFD645A155029201AA18D
:10599000181A55181A8D049A2D301EC11901086D58
:1059A0001401101ABD78DAB974411A57481A5F0405
:1059B0001ACD201A69081AB5041AA7041AC9482A68
:1059C000C33418091401084D15010815081A7D087B
:1059D0001E8116010811041A7D1C7CD1130150137D
:1059E000E1DA14083FBC140805DB140895BE1B0857
:1059F000B5101A1F101AC5081A25081AA5081A1179
:105A00000801681370071F2088540108A0041A8039
:105A1000041AC0041AA8041A90042A98081A5518DF
:105A200019041A28041AE0101119081AF0081A1497
:105A3000081AD4081AB0041A340C1A48041A640458
:105A40001AC81032281353B93308144B15C2080B67
:105A500010F9C1D413A5C71B084D041A7D04391DC4
:105A6000350C0140012904290C419A020C118A804D
:105A70000C39055A0818290669249A0418293D6921
:105A80000C293C3C100140502912690C2905593C55
:105A90009A108439851924390C2924190C5129119B
:105AA00059549A209C29777954013B13BDC5140899
:105AB00084081B2090041398094808209C5501086D
:105AC0009DC6141A9C041AAC149AA4141AA8041A99
:105AD000C0149AAC141AB4041AD4149AB0141AC08C
:105AE000041AE8149AB4141ACC041AFC149AB814C0
:105AF0001AD80413100A4808200C56010801C714CC
:105B00001AE4041A24141AFC285AD3141AF0041A9A
:105B100038149AA0141AFC041A4C149AA8501A08A3
:105B2000601A60141A045069141A14141A74149A1E
:105B3000C8281A20141A88149AEC141A2C141A9CC7
:105B4000149AF4142A38D819149AD4141A44141A2A
:105B5000C4149ABC141A50141AD8141ADC1401284C
:04000005080081511D
:00000001FF
